:100000000C94C0300C94E8300C94E8300C94E83038
:100010000C94E8300C94E8300C94E8300C94E83000
:100020000C94E8300C946AAE0C9475AE0C94E830E5
:100030000C94E8300C949DB40C94E8300C94E830A7
:100040000C9480AE0C94E8300C94E8300C94E830BA
:100050000C94BAC60C94E8300C94E8300C94E83058
:100060000C942B500C94E8300C94E8300C94E8304D
:100070000C94A9C50C94E0C50C94E8300C94E830BD
:100080000C94E8300C94E8300C94E8303A333E336A
:10009000423346334A3389335E33623366336E33D9
:1000A0007233F7320E33123316331A331E332233C0
:1000B00026332A332E33323336330A337A338533B9
:1000C000474157415C41664174417B4181419541C3
:1000D00098417F6386638D63926397639E63A56394
:1000E000AA63B163B863BD63C463D263CB63517564
:1000F00054755C7559755F756275657568756D7554
:100100007075757578757B757E75817589758C755B
:100110009175947599759E75A37535987D993B98E1
:1001200045984F985D986D9879987D99C498E59811
:100130003C994A995D998C987D996C9905A84CCD0C
:10014000B2D44EB93836A9020C50B9918688083C11
:10015000A6AAAA2ABE000000803F4F4B000D0A004D
:10016000720A00496E717569727920456E64000DDE
:100170000A00496E717569727920526573756C74E5
:10018000733A0D0A002E004552524F520D0A004F8D
:100190004B0D0A000D004154423F004154533100C1
:1001A00041544E3D004154523100415452300041BF
:1001B000544F300041544F31004154463F004154A8
:1001C000443D0041544430004154480041544100F2
:1001D000415400415445310041545130004154458F
:1001E0003000415451310041544C350041544C349D
:1001F0000041544C330041544C320041544C3100C6
:1002000041544C300041544C2A0041545A30004172
:1002100054503D0054696D65206F75742C466169BA
:100220006C20746F20636F6E6E6563742100434FA2
:100230004E4E45435400444953434F4E4E4543545C
:10024000000D0A0042544D32323220496E6974204A
:100250004F4B0042544D323232206E6F7420666F25
:10026000756E642100425420696E697469616C691D
:1002700073696572656E2E2E007365617263682006
:100280006572726F7200666F756E64002E2E2E2E70
:10029000002E2E2E002E2E002E0031313532303021
:1002A00000353736303020003338343030200031DC
:1002B00039323030200039363030202000343830A8
:1002C00030202000323430302020007365617263AA
:1002D0006820776974683A00736574204563686FB5
:1002E000206F6666004572726F72207365742045D8
:1002F00063686F0073657420426175647261746530
:10030000204572726F720073657420426175647269
:10031000617465206F6B004572726F723120736576
:10032000742042617564726174652E2E00425420FF
:10033000736574206E6577204261756472617465BF
:100340002E2E00504B54004576616C756174696FB8
:100350006E20283836384D487A29202000526164B2
:10036000696F74726F6E69782057692E3233324428
:10037000545300555342202D3E2057692E323332BC
:10038000004D4B2D55534200555342202D3E2053D6
:100390005632204B6162656C004B6162656C206176
:1003A0006E7363686C69657373656E2E20200050F0
:1003B0004B542065696E2067656B7265757A74654C
:1003C00073202020005A7769736368656E204D4B57
:1003D0002D55534220756E642020004D4B2D5553F2
:1003E0004220616E20504320616E7363686C2E2042
:1003F000004643203E204D4B2D555342203E204287
:10040000544D2D3232320042544D2D323232204B77
:100410006F6E6669677572696572656E00424C45FC
:1004200020457874656E646572003136392E323538
:10043000342E312E313A3230303000574C414E207C
:10044000457874656E646572004254204578746521
:100450006E646572004254202D3E20535632204B6C
:100460006162656C004F4B002121436865636B201E
:10047000506172616D657465722121200000003148
:1004800036392E3235342E3030312E303031003284
:1004900035352E3235352E3030302E30303000317B
:1004A00036392E3235342E3030312E303031003165
:1004B0003233343536373800504B5400303030301A
:1004C00000303030302D30302D3030303030300092
:1004D000504B540030303030005374616E646172A0
:1004E0006477657274652067657365747A740077E4
:1004F000657264656E206175660020454550524FF7
:100500004D20506172616D6574657220202020005D
:10051000202020577269746520454550524F4D2068
:10052000202020004F4B00636865636B2073657467
:1005300074696E677321006E657720566572736902
:100540006F6E00454550726F6D2075706461746503
:100550006420746F0000003136392E3235342E306D
:1005600030312E303031003235352E3235352E30A7
:1005700030302E303030003136392E3235342E3096
:1005800030312E30303100313233343536373800A7
:10059000504B54006D002E002E006B6D2F68002E06
:1005A00000636D002020006F6B00200044006E6F20
:1005B0000032440033440020002D00780058004FE2
:1005C00000416C742020202020203A20004C6174CF
:1005D0002020202020203A20004C6F6E6720202011
:1005E00020203A20005370656564202020203A20A6
:1005F0000050444F5020202020203A2000416363C7
:100600007572616379203A200053617420202020A4
:1006100020203A20004669782054797065203A20DD
:10062000004E7572206D6974204E4320210048579A
:1006300020332E3978202831312E323031322900C2
:10064000485720332E396D202830392E3230313141
:100650002900535632205061746368000000000086
:100660000000781514157800205554557800384549
:10067000444538003049484930003C4140413C0045
:100680003841402178007E1515150A0022170F17F2
:100690002200008482FF82841C141C0000000007DA
:1006A0000507000010385410101E180C1800000028
:1006B0001010101010101010107C101008100800EE
:1006C00000000814000014081008040408100810A2
:1006D00020201008000814224100004122140800C4
:1006E00004027F02040010207F20100010385410F4
:1006F000101010101054381010181C1C1810081866
:100700003838180800081C3E7F00007F3E1C080097
:100710000609090906001020100804020000000064
:10072000000000002F000000000700070000147FF9
:10073000147F1400242A6B2A120023130864620019
:10074000364955225000000503000000001C2241DC
:1007500000000041221C000014083E081400080894
:100760003E08080000503000000008080808080093
:100770000060600000002010080402003E5149455E
:100780003E0000427F400000426151494600214145
:10079000454B31001814127F10002745454539009C
:1007A0003C4A49493000030171090700364949496B
:1007B0003600064949291E00003636000000005662
:1007C0003600000008142241000014141414140010
:1007D0000041221408000201510906003249794102
:1007E0003E007E1111117E007F49494936003E418D
:1007F000414122007F4141221C007F49494941007B
:100800007F09090901003E4149497A007F0808082B
:100810007F0000417F4100002040413F01007F08F0
:10082000142241007F40404040007F020C027F00C4
:100830007F0408107F003E4141413E007F090909C5
:1008400006003E4151215E007F09192946004649B4
:100850004949310001017F0101003F4040403F0014
:100860001F2040201F003F4038403F006314081401
:1008700063000708700807006151494543007F4144
:10088000410000000204081020000041417F0000E8
:100890000402010204004040404040000001020404
:1008A00000002054545478007F48444438003844B1
:1008B00044442000384444487F00385454541800BD
:1008C000087E090102000C5252523E007F080404C7
:1008D000780000447D4000002040443D00007F102F
:1008E0002844000000417F4000007C041804780088
:1008F0007C08040478003844444438007C14141400
:100900000800081414187C007C08040408004854EB
:1009100054542000043F444020003C4040207C00D0
:100920001C2040201C003C4038403C00442810283B
:1009300044000C5050503C004464544C44000008A7
:100940003641000000007F00000000413608000032
:1009500008082A1C0800081C2A0808006E6F74206A
:10096000617661696C61626C6521007468697320ED
:1009700066756E6374696F6E206973002A2A204F52
:100980005554204F462052414D202A2A0020202E27
:1009900020202E2020202000201A202020201B2074
:1009A00020202020457869740020203031323334F3
:1009B00035363738394142434445460D0A005375B0
:1009C000636865204D696B726F6B6F707465720040
:1009D000736561726368204B6F70746572004F536A
:1009E0004420446174656E004F5344204461746137
:1009F00000504B54205370657A69616C00504B5421
:100A0000205370656369616C00504B5420436F6ED6
:100A10006E65637400504B542053657475700050BC
:100A20004B5420496E666F004D4B20496E666F0037
:100A30004D4B2053657474696E6773004D4B2044B1
:100A40006973706C6179004D4B20446174656E0070
:100A50004D4B2044617461004F5344004D4B20477F
:100A6000505320496E666F00425420202045787410
:100A7000656E64657200424C452020457874656E51
:100A800064657200574C414E20457874656E64650C
:100A9000720055534220202D3E20576932333200D8
:100AA00055534220202D3E205356320042542020E0
:100AB000202D3E2053563200504B5420436F6E6E13
:100AC000656374004D4B204D6F746F727465737461
:100AD00000547261636B696E67004A6F7973746961
:100AE000636B00504B54205370657A69616C00FB56
:100AF0000EFB0E060F1C0F320F480F5E0F700F8299
:100B00000F8C0F960FA00FAA0FB10FB80FC80FD5FB
:100B10000FE10FEF0FFF0F0D10211036104C106179
:100B20001071107F109410A810AD10B110B410B750
:100B300010BE10C410CA10D010DA10DF10F310FD70
:100B40001007110F1118111D1123112A113311391A
:100B5000113F11431158116B117E118C1195112AFF
:100B60001133119E11B211C711CB11D011D711DD64
:100B700011E511ED11F311F911FF1105120512091B
:100B8000121A12281232123C12461250125F126CC4
:100B90001281129312A612B812C812D712ED1203C4
:100BA0001319132F134413581365137213881394D6
:100BB00013A713BA13CB13D513EB13FE1314142678
:100BC000143C14461459146514781484149814AC05
:100BD00014BC14CB14DD14EF1405151B152B153E96
:100BE000154E155E155E1574158A15A015B615CC33
:100BF00015E215F815F8150E161E162C1642165885
:100C0000166A1679168F16A516A516BB16D116E705
:100C100016FD16131729173F1755175D1763176928
:100C2000176917721772177A1782178A17A017B2E7
:100C300017BF17C717D117DB17EC17FA1704180DD2
:100C4000181918251831183D18491855186B1881AE
:100C5000189218A318AE18B918C818D818E518F1C2
:100C600018FF180D190D191C192A193719371941B0
:100C7000194119501950195F195F196E196E197DB4
:100C8000197D198D199F19B119C719D619E119EBD9
:100C900019F019F519FA19FF19151A2B1A411A52D8
:100CA0001A5D1A671A791A8B1AA11AB71AC51AD3BC
:100CB0001AD31AE31AF91A0D1B201B2D1B3D1B49D1
:100CC0001B491B571B591B5B1B5D1B5F1B5F1B617C
:100CD0001B611B631B631B661B661B691B6C1B6F05
:100CE0001B851B961BA61BB21BBC1BC61BDC1BF269
:100CF0001BF91B001C0B1C141C1E1C281C3E1C4E2C
:100D00001C5E1C691C791C871C981CA51CBB1CD173
:100D10001CE41CF11C071D1D1D331D491D5F1D75A5
:100D20001D8B1DA11DB61DCB1DE11DF71D0D1E2325
:100D30001E341E451E531E611E6F1E7D1E8B1E9986
:100D40001EA71EB51EC31ED11EDF1EED1EFB1E09F3
:100D50001F091F111F111F191F281F371F4B1F5E4F
:100D60001F691F741F7F1F8A1F951FA01FAB1FB60F
:100D70001FB61FC01FC01FCA1FCA1FCF1FCF1FD43F
:100D80001FD41FD91FE51FF11FFD1F0920092015C2
:100D90002015201F202920332033203D20472051BB
:100DA000205B2065206F20792083208D20A320B92F
:100DB00020C820D820E620F4200421142124213446
:100DC000214421542162217021802190219F21B052
:100DD00021B021BF21BF21D221D221E221F3210460
:100DE000220422152226223722482259226A227BF7
:100DF000229122A622B422C222D822EE22FF221061
:100E0000231023262326233C233C2345234C235312
:100E1000235B2362236923712384239723AA23BDA1
:100E200023D023E323F62309241C242F2442245512
:100E30002468247B247B248E249924A424B724CAE8
:100E400024DD24F0240325162529253C2549255693
:100E5000256325702581258F25A225B525BC25C3B1
:100E600025CA25D125E725FD251026232630263D38
:100E7000264F2660266F267C268B269926A926B724
:100E800026C226CB26D426DC26ED26FD260A2716EA
:100E90002726273627462756276627762776277E52
:100EA000277E2789278927922792279C279C27A579
:100EB00027A527AD27AD27B827B827BD27BD27C24F
:100EC00027C227C727DB27EF27F627FC270A281585
:100ED0002826283A284F2863286E28732877287CEC
:100EE0002881288428842888288F289728A628B134
:100EF00028C228D028DF28EA28EA286C6E672E202E
:100F00006572726F7200201A20202020201B202082
:100F10002020456E64652020204F4B00201A2020A1
:100F20002020201B20202020656E64202020204FC0
:100F30004B00201820202020201920202020456E42
:100F400064652020204F4B002018202020202019ED
:100F500020202020656E64202020204F4B00201888
:100F600020202020201920202020456E64652000AC
:100F7000201820202020201920202020656E6420A9
:100F80002000456E64652020204F4B00656E642074
:100F90002020204F4B00456E646520496E666F002F
:100FA000656E642020696E666F0020416262722E59
:100FB0000043616E63656C00546173746520312079
:100FC00053656B756E64650070726573732062752E
:100FD00074746F6E006665737468616C74656E21FD
:100FE00000666F722031207365636F6E6421004C60
:100FF00065747A746520506F736974696F6E006CE4
:1010000061737420706F736974696F6E00427265EA
:101010006974656E677220204CE46E67656E677256
:10102000006C617469747564652020206C6F6E6754
:101030006974756465006CF6736368656E202020C2
:10104000202020202020204E65696E0064656C659C
:1010500074652020202020202020202020204E6F7A
:1010600000476F6F676C652045696E676162653A1E
:1010700000476F6F676C6520496E7075743A007336
:1010800075636865204D696B726F6B6F7074657204
:101090002E2E2E00736561726368696E67204B6F38
:1010A000707465722E2E2E00456E646500656E6448
:1010B000004F4B006F6B004665686C65720065728F
:1010C000726F7200616B7469760061637469760097
:1010D00073706569636865726E0073617665007729
:1010E0006972642067657370656963686572742EE0
:1010F0002E2E00736176696E672E2E2E0056657255
:1011000077657266656E0064697363617264004B33
:101110006F70696572656E00636F707900737563D7
:1011200068650073656172636800676566756E6403
:10113000656E00666F756E64007365747A65007322
:101140006574004D6F746F72656E206175737363A3
:1011500068616C74656E2100737769746368206DD3
:101160006F746F7273206F666621004643206E694C
:1011700063687420676566756E64656E210046431A
:10118000206E6F7420666F756E64210065727761E2
:101190007274657400657870656374656400766F59
:1011A0006C6C206B6F6D7061746962656C206E751C
:1011B000720066756C6C20636F6D70617469626C2F
:1011C00065206F6E6C79006D6974007769746800D2
:1011D0004645484C4552004552524F5200574152E5
:1011E0004E554E47005741524E494E470045696E95
:1011F0002020004F6E202020004175732020004FDA
:10120000666620200045534300504B54206175739F
:10121000736368616C74656E3F0073687574646FA6
:10122000776E20504B543F004A612020204E656964
:101230006E00796573202020206E6F004E65696E08
:101240002020204A61006E6F2020202079657300E5
:10125000446174656E206CF6736368656E3F00646C
:10126000656C65746520646174613F0056657262E7
:10127000696E646520504B54206D69742050432181
:1012800000436F6E6E65637420504B5420746F2062
:101290005043004472FC636B652027537461727481
:1012A000272066FC720050726573732027537461A7
:1012B00072742720666F72006D696E2E2032205383
:1012C000656B756E64656E006D696E2E20322073DD
:1012D00065636F6E64730020202020202020202072
:1012E0002020456E646520537461727400202020B4
:1012F0002020202020202020456E6420205374616F
:101300007274002050432D517569636B2D566572C0
:1013100062696E64756E6720002050432D517569B7
:10132000636B2D436F6E6E656374696F6E2000563C
:10133000657262696E64652064617320504B54204D
:101340006D697400436F6E6E65637420504B54205A
:1013500077697468204D4B0064656D204D4B20FC0F
:101360006265723A002020206F766572202020206E
:101370003A0064656D204D4B20FC6265723A202076
:101380004B6162656C2C20006F7665723A204B6170
:1013900062656C00657320697374206B65696E20EB
:1013A00057692E3233320074686572652069732084
:1013B0006E6F2057692E323332004D6F64756C208A
:1013C00065696E6765626175742E006275696C741B
:1013D00020696E2E0057656E6E20646F63682C2046
:1013E00064616E6E20626974746500696620796557
:1013F000732C207468656E20666972737400646172
:1014000073204D6F64756C207A75657273742069F2
:101410006D2020006163746976617465206D6F646E
:10142000756C20696E0053657475706D656EFC2077
:10143000616B746976696572656E2E0053657475AB
:10144000706D656E7500536965206DFC7373656E14
:101450002064617320504B5400596F752068617689
:101460006520746F006A65747A74206E65752073E8
:1014700074617274656E2100726573746172742098
:10148000504B5400457320697374206B65696E205E
:1014900042544D2D323232005468657265206973B2
:1014A000206E6F2042544D2D323232004D6F6475E4
:1014B0006C2065696E676562617574004D6F647557
:1014C0006C206275696C7420696E00204D4B2D553F
:1014D00053422046756E6B74696F6E2000204D4B31
:1014E0002D5553422046756E6374696F6E2000203F
:1014F0004254202D2D3E204B6162656C20616E2090
:101500004643202000204254202D2D3E204B616276
:10151000656C20746F2046432020005043206D6985
:101520007420425420766572622E00636F6E6E6581
:101530006374205043207769746820425400504BF4
:10154000542D4B6162656C20616E20464300504B08
:10155000542D4B6162656C20746F2046430020421D
:1015600054202D2D3E2057692E323332202020204A
:101570002020200057692E32333220616E204643EE
:101580002020202020202020200057692E323332B6
:1015900020746F204643202020202020202020007F
:1015A00020555342202D2D3E204B6162656C2061F9
:1015B0006E204643200020555342202D2D3E2063AF
:1015C00061626C6520746F20464320005043206D9B
:1015D0006974205553422076657262696E64656E47
:1015E0002000636F6E6E65637420504320776974CA
:1015F000682055534220200020555342202D2D3E77
:101600002057692E323332202020202020004D4BDD
:101610002D546F6F6C207374617274656E007374F7
:10162000617274204D4B2D546F6F6C002057692EE2
:10163000323332204B6F6E66696775726965726509
:101640006E002057692E32333220436F6E66696711
:1016500075726174696F6E0050726F6772616D6D43
:10166000207374617274656E2E00737461727420DD
:1016700070726F6772616D200042544D2D323232AC
:10168000204B6F6E6669677572696572656E0042A0
:10169000544D2D32323220636F6E66696775726108
:1016A00074696F6E004643203E204D4B2D555342CA
:1016B000203E2042544D2D323232004D4B2D555399
:1016C0004220616E20504320616E7363686C2E204F
:1016D00000636F6E6E65637420504320746F204DFD
:1016E0004B2D55534220005A7769736368656E200D
:1016F0004D4B2D55534220756E64202000636F6E54
:101700006E6563742063726F7373656420636162D6
:101710006C6500504B542065696E2067656B72657F
:10172000757A746573202020006265747765656E34
:10173000204D4B2D55534220616E64202020004BDC
:101740006162656C20616E7363686C696573736553
:101750006E2E202000504B5420535632004B6162B5
:10176000656C006361626C6500536C617665202076
:1017700020004E6F726D616C200052657665727349
:101780006500696E7665727365004E61636820C49A
:101790006E646572756E672064617320504B5400EF
:1017A0007265737461727420504B54206166746565
:1017B00072006E6575207374617274656E210063CA
:1017C00068616E67652100456E64652020204F4B7F
:1017D00000456E64202020204F4B0020454550726C
:1017E0006F6D207769726B6C696368002052656168
:1017F0006C792064656C65746500206CF6736368B1
:10180000656E3F0020454570726F6D3F00646575E1
:101810007473636820202020006765726D616E20FC
:101820002020202000656E676C697363682020208B
:1018300000656E676C6973682020202000686F6CFB
:101840006CE46E6469736368006475746368202077
:101850002020202000416E7A656967652045696E09
:101860007374656C6C756E67656E00204469737087
:101870006C61792053657475702020202020202011
:1018800000496E666F7320626569205374617274DB
:101890003A00496E666F20617420737461727475CA
:1018A00070200053707261636865203A20004C61BB
:1018B0006E67756167653A20004C696368742061E2
:1018C0007573206E616368004C69676874206F6689
:1018D00066206166746572004C43442048656C6CF8
:1018E00069676B2E00204272696768746E65737356
:1018F000004C4344204B6F6E74726173743A004C19
:10190000434420636F6E74726173743A004C4344B5
:10191000204E6F726D2F496E763A2000524320465A
:1019200065686C657270696570005243204572721B
:101930006F726265657000446562756720504B5434
:101940000057692054582F5258204368616E3A005E
:101950005769204E6574572E204772702E3A0057F3
:1019600069204E6574572E204D6F64653A005769A3
:101970002054582054696D656F75743A005769207A
:1019800055415254204D54552020203A0057692E7D
:101990003233322065696E6765626175743A00574B
:1019A000692E323332206275696C7420696E203A78
:1019B000004973742065696E2057692E3233322DC9
:1019C0004D6F64756C2000497320576932333220A3
:1019D0006D6F64756C0065696E6765626175743FF3
:1019E000006275696C7420696E3F004A61202000B6
:1019F00079657320004E65696E006E6F20200020AF
:101A000042544D3232322045696E7374656C6C7588
:101A10006E67656E00202042544D2D3232322073A5
:101A2000657474696E6773202020004973742065A3
:101A3000696E2042544D2D3232322D4D6F64756CDB
:101A40000049732042544D2D323232204D6F64755F
:101A50006C0065696E6765626175743F00627569E7
:101A60006C7420696E3F0042544D323232206569F9
:101A70006E6765626175743A0042544D32323220AD
:101A80006275696C7420696E203A0020504B5420B6
:101A9000416B6B752045696E7374656C6C756E6710
:101AA0000020504B5420416363752053657475705A
:101AB00020202020202000504B5420416B6B757457
:101AC00079703A2000504B542041636375747970EB
:101AD0003A2000416B6B752055204F666673657424
:101AE0003A20004F6666736574207665727374657C
:101AF0006C6C656E206269730061646A7573742032
:101B00006F666673657420756E74696C00646965D0
:101B1000205370616E6E756E672070617373740010
:101B2000766F6C746167652066697473007A6569A5
:101B30006765205A656C6C656E73702E0073686FF4
:101B4000772043656C6C2055004C6F7742617420A0
:101B50005761726E20560056004600480042004C05
:101B60000052004E6900526F004B6F00436F0046F9
:101B700045484C45523A20446174656E7665726CF6
:101B800075737420004552524F523A20446174617B
:101B9000206C6F7374004C65747A74652062656B99
:101BA000616E6E7465004C617374206B6E6F776E3E
:101BB0002000506F736974696F6E2000706F7369D5
:101BC00074696F6E20002045696E7374656C6C7566
:101BD0006E67656E20202020202020002053657431
:101BE00074696E67202020202020202020202020C3
:101BF0002000E46E6465726E006368616E67650064
:101C0000416B746976696572656E006163746976AB
:101C100061746500616B74697669657274006163F3
:101C200074697661746564002053657474696E67C5
:101C300020782073706569636865726E3F00207359
:101C4000746F72652073657474696E673F004765D1
:101C500073706569636865727420756E640073746F
:101C60006F72656420616E64004B6F7069657265A8
:101C70002053657474696E6700636F7079207365B3
:101C80007474696E67730020766F6E202078202050
:101C90006E616368202079002066726F6D20782065
:101CA000746F207900766F6E2020206E616368204B
:101CB00020456E64652020204F4B0066726F6D20BA
:101CC00020746F20202020656E64202020204F4B40
:101CD000005769726B6C696368206B6F706965721D
:101CE000656E3F007265616C6C7920636F70793F3F
:101CF000004B6F706965727420756E6420616B743F
:101D000069766965727400636F7069656420616EDD
:101D100064206163746976617465642000E46E64B4
:101D20006572652045696E7374656C6C756E676568
:101D30006E20002020206368616E676520736574E3
:101D400074696E6773202020002057E4686C65205A
:101D5000506172616D657465722020202020002022
:101D600073656C65637420706172616D6574657212
:101D700073202020002057E4686C65205365697447
:101D8000652020202020202020200020202020202E
:101D900073656C6563742070616765202020202066
:101DA000002057E4686C652053657474696E673A67
:101DB0002020202020002073656C656374207365EB
:101DC0007474696E67202020202000202047505323
:101DD0002045696E7374656C6C756E67656E202046
:101DE00000202020204750532073657474696E676B
:101DF00073202020202000676577E4686C74657389
:101E00002047505320476572E47420200073656CAE
:101E10006563746564204750532064657669636523
:101E200020200047505320456D70662E616B746909
:101E3000763F3A00726563656976652047505320A6
:101E40006F6E3F3A006D61782048F668652020206B
:101E5000203A006D617820616C7469747564653A2C
:101E6000006D6178204765736368772E203A006DB6
:101E700061782073706565642020203A006D617878
:101E800020456E746665726E2E3A006D617820642E
:101E9000697374616E63653A006D696E2053706199
:101EA0006E6E756E673A006D696E20766F6C746148
:101EB0006765203A006D6178205A6569742020209A
:101EC000203A006D61782074696D65202020203AE9
:101ED000006D6178205374726F6D2020203A006D80
:101EE00061782063757272656E74203A00456E7475
:101EF0002E4B6170617A69742E3A005573656443A4
:101F0000617061636974793A004C6F6E672E203A94
:101F1000004C61742E20203A004E7572206D697459
:101F2000204E4320212020004F6E6C792077697469
:101F300068204E432021004B65696E65205365740F
:101F400074696E67732021212020004E6F20736515
:101F50007474696E6773207265616421210048F6AC
:101F6000686520206175732000416C74692E206FB4
:101F70006666200048F6686520626567722E00413B
:101F80006C74692E4C696D697400566172696F20BA
:101F90006175732000566172696F206F666620005C
:101FA000566172696F2048F6686500566172696F04
:101FB00020416C742E002020202020202020200092
:101FC0004361726520467265650020202020004C28
:101FD000454431004C454432004E61766920206111
:101FE00075732020004E61766920206F6666202080
:101FF00000506F732E2068616C74656E00506F73B3
:102000002E20486F6C64202000436F6D696E67203E
:10201000486F6D6500202020202020202020004ACD
:10202000757374696572656E0043616C6962726193
:10203000746500537461727420202020004265741E
:102040007269656220200052756E202020202020B9
:1020500000466C696567656E202000466C7920201B
:1020600020202020004C616E64756E672020004C9B
:10207000616E64696E67202000416B6B75206C6532
:102080006572004C6F77204261742E200020204F33
:10209000534420416E7A6569676520536574757095
:1020A00020200020204F53442073637265656E200A
:1020B0007365747570202020004F7574312F3220A5
:1020C0006E656769657274004F7574312F322069CF
:1020D0006E766572746564004F7574312F322046D8
:1020E0006F726D6174004F7574312F3220666F729C
:1020F0006D6174004E6176696461746120616E2067
:10210000535632004E6176696461746120746F20A9
:10211000535632006D2E2053696E6B7261746520C8
:102120006D2F73006D2E66616C6C73706565642035
:102130006D2F7300566172696F6D65746572204210
:1021400065657000766172696F6D65746572206295
:10215000656570006D4168205761726E756E67200D
:102160003E006D4168207761726E696E67203E00A7
:102170004F534420416E7A656967657661723A0013
:102180004F53442073637265656E6D6F64653A00EA
:102190004D4B20566F6C742042616C6B656E004D28
:1021A0004B20766F6C742062617267726170680098
:1021B000426175642057693233322F42543A00200D
:1021C000466F6C6C6F77204D652053657475702079
:1021D0002000202020202052656672657368202030
:1021E0003A00476573636877696E6469676B656910
:1021F000743A002020202053706565642020202040
:1022000020203A00546F6C6572616E7A20526164CE
:102210006975733A00546F6E61757367616265200A
:102220004572772E3A00736F756E64206578746519
:102230006E73696F6E3A00486172647761726520EF
:102240005069657065723A006861726477617265A1
:10225000206265657020203A004C6175747374E4E7
:10226000726B6520202020203A00766F6C756D65BA
:102270002020202020202020203A007365726965EC
:102280006C6C65204B616EE46C65205365747570F1
:102290000073657269616C206368616E6E656C20A5
:1022A0007365747570004C69706F204D657373753C
:1022B0006E673A004C69706F20636865636B20201D
:1022C0003A004B616E616C202020202020202020CD
:1022D00020202020202020004368616E6E656C2045
:1022E0002020202020202020202020202000536596
:1022F00072766F73636872697474653A2020007334
:102300006572766F73746570732020203A20200008
:102310002020202020202020536572766F2031203D
:102320002020202020002020202020202020536555
:1023300072766F20322020202020200052657665A2
:102340007273653A004C696E6B733A006C65667423
:10235000683A005265636874733A0072696768741A
:102360003A004D697474653A006D6964646C653A4D
:1023700000546573742050756C736CE46E6765204F
:102380002020200074657374206672616D65776922
:102390006474682020200020536572766F207A755F
:1023A0006D2054657374656E200020736572766FBE
:1023B00020746F207465737420202020002020205A
:1023C000202020506572696F646520202020200045
:1023D0002020202020206672616D65202020202092
:1023E0002020005465737420666F72746C6175668A
:1023F000656E642020007465737420636F6E746969
:102400006E756573202020200045696E7A656C73B7
:1024100063687269747420202020200073696E67DD
:102420006C652073746570202020202020200041DE
:102430006E7A61686C20202020202020202020201F
:1024400020007465737420636F756E7420202020E3
:102450002020202000506175736520456E64706FE8
:10246000736974696F6E2000706175736520656EA5
:1024700064706F736974696F6E2000506175736565
:102480002070726F20496E632E202020200047505C
:1024900053204D617573203A00475053206D6F757E
:1024A00073653A00475053204254204D61757320A4
:1024B00031202020202000475053204254204D6FCF
:1024C0007573652031202020200047505320506F25
:1024D000732E20766F6D204D4B20202000475053E7
:1024E00020706F732E2066726F6D204D4B20200080
:1024F000537469636B206D696E2E20576572743A50
:10250000202000737469636B206D696E2E207661E4
:102510006C75653A2000537469636B206D61782E89
:1025200020576572743A202000737469636B206DC4
:1025300061782E2076616C75653A20005269636877
:1025400074756E673A20202000646972656374694F
:102550006F6E3A202000537469636B747970653A2A
:10256000202000737469636B747970653A202000D1
:102570004E65757472616C6973696572656E643AF3
:10258000006E65757472616C697A696E673A004CA9
:1025900069706F204D657373756E673A2020202037
:1025A00020004C69706F206D6561737572656D6593
:1025B0006E743A2000506F7469202000706F746947
:1025C00020200054617374657200737769746368C6
:1025D00000202020504B54205A65697420205365F8
:1025E00074757020202000202020504B54207469E6
:1025F0006D6520736574757020202020005A656910
:10260000747A6F6E652020285554432B2D293A008B
:1026100074696D65207A6F6E6520285554432B2DA3
:10262000293A00536F6D6D65727A656974203A00BE
:1026300073756D6D65722074696D653A004F534412
:102640002D20756E6420424C2D446174656E004FE0
:1026500053442D20616E6420424C2D44617461000E
:102660004D4B204665686C65726C69737465004DEE
:102670004B206572726F726C69737400557365726A
:10268000204750532D446174656E00557365722068
:102690004750532D64617461006C65747A746520D1
:1026A000506F736974696F6E006C61737420706F22
:1026B000736974696F6E00414C4C452044617465C8
:1026C0006E00414C4C2064617461006CF673636869
:1026D000656E3F0064656C6574653F007A65696787
:1026E00065204D4B2D53657474696E670073686F78
:1026F00077204D4B2073657474696E670057694687
:102700006C79204D6F6475733A005769466C792077
:102710006D6F64653A005750412076657277656E3B
:1027200064656E203A007573652057504120202063
:10273000202020203A0053696368657268656974D7
:10274000202020203A007365637572697479202017
:10275000202020203A004B616E616C202020202038
:10276000202020203A006368616E6E656C20202076
:10277000202020203A0047656E6572616C004E6132
:102780007669676174696F6E00456C656374726920
:1027900063004D4B2D5374617475730055736572EE
:1027A00020475053003344204C61676500537461E7
:1027B00074697374696373004F534430004F53441A
:1027C00031004F534432006B65696E656E204D4B8E
:1027D00020676566756E64656E2100202020206E7E
:1027E0006F204D4B20666F756E64212020200046BF
:1027F00045484C4552004552524F52004461746561
:102800006E7665726C757374210044617461206C1E
:102810006F737421006C6164652053657474696E14
:1028200067732E2E2E006C6F6164696E672073656E
:102830007474696E67732E2E2E00616B74697669ED
:102840006572652053657474696E672E2E2E006163
:10285000637469766174652073657474696E672E3C
:102860002E2E004265617262656974656E00656452
:10287000697400766F6E0066726F6D006E616368DA
:1028800000746F00504B5400414B54495621004195
:1028900043544956452100424C4520766F72686189
:1028A0006E64656E3A00424C452065786973743AEF
:1028B000004D6F64756C20766F7268616E64656E32
:1028C0003F004D6F64756C652065786973743F00D7
:1028D000496E697469616C6973696572656E0049F6
:1028E0006E697469616C697A65004C6173747269B0
:1028F0006E670052656672657368004D4B205365C4
:102900007474696E67004E433A00205265762D4517
:102910005252210025303375005265763A00464305
:102920003A004D4B20496E666F00257500257520D5
:102930002573002D206572726F72202D0025317570
:102940002E253032752563002D2D2D2D2D0025319E
:10295000752E253032752563004552524F523A206C
:102960006E6F2064617461004E430046430045521F
:10297000524F523A206E6F20646174610020200033
:10298000416E616C6F67204E616D65733A20005235
:10299000656164696E673A004665686C65723A20E5
:1029A0004B65696E6520446174656E0018202020B7
:1029B000201920202020201B202020201A004469DC
:1029C00073706C6179004643004E4300ACCC610DDE
:1029D0003300000F331333ADCC610D3300001C33D3
:1029E0001C33AACC610D33000021332133ABCC6101
:1029F0000D33000026332633AECC612B3300003379
:102A0000333333AFCC612B3300003A333A33B0CC9D
:102A1000612B33000041334133B1CC612B330000D3
:102A200048334833B2CC612B3300004F334F33B3BC
:102A3000CC612B33000056335633B4CC612B3300BA
:102A4000005D335D33B5CC612B33000064336433F8
:102A50005ACC616B33000071338733DFCC619B3319
:102A600000009E339E33CBCC619B330000AD33C35B
:102A700033E2CC619B330000D933E733E6CC619B72
:102A8000330000F133FF33EBCC619B3300000E3495
:102A90000E34E9CC619B33000018342634EACC6153
:102AA0009B33000034344034ECCC619B3300004C49
:102AB000345E34EDCC619B3300006D348134E8CC5E
:102AC000619B330000943494340DCC61A134001424
:102AD000A334A3340ECC61A1340014AF34AF340F4F
:102AE000CC61BB3400F7BE34BE3457CC61BB34007C
:102AF000F7C534D434D2CC619B330000E134EE34DA
:102B0000D3CC619B330000F9340735D4CC619B33BF
:102B1000000014352235D5CC619B3300002F353EA3
:102B20003531CC61BB3400F74C355E3532CC61A118
:102B30003400F77235833533CC61A13400F7963514
:102B4000A03537CC61A13400F7AB35BC3538CC614A
:102B5000A13400F7CA35DB35E6CC619B330000F1C8
:102B600033FF33C8CC619B330000E935F935C9CC5C
:102B7000619B3300000B361636E7CC619B330000B7
:102B800023363136CACC619B3300003F363F3606D0
:102B9000CC614C3600005336613604CC61A1340060
:102BA000F77036793607CC61BB3400F787368E363E
:102BB00005CC61BB3400F79936A53609CC61BB342E
:102BC00000F7B236B2365ECC61BB3400F7B836CE11
:102BD0003608CC61A13400F7E436F3360ACC61A1A3
:102BE0003400F7FD3609370BCC61BB3400F71937D9
:102BF00019370CCC61A13400A01F37313762CC618A
:102C00004337000047375C3763CC61A13400F7726B
:102C100037723723CC61BB3400F78837993724CC1F
:102C200061BB3400F7A937BB37E3CC619B330000AD
:102C3000CC37DB37BECC619B330000F137FF37C0A8
:102C4000CC619B3300001338203825CC61A13400BF
:102C5000F72D382D3826CC61A13400F740384038A4
:102C600060CC61A134001953385F3827CC61BB3484
:102C700000F76B387C3828CC61BB3400F78D389F67
:102C800038BFCC619B330000B138BF3829CC61A17B
:102C90003400F7D338D3382ACC61A13400F7E038B8
:102CA000E03861CC61A1340019ED38F9382BCC61E2
:102CB000A1340208053913392CCC61A13400F72165
:102CC000392F392ECC613D3900F5413941392FCCAE
:102CD000613D3900F54939493930CC61BB3400F7E1
:102CE00051395139EBCC619B3300000E340E34471F
:102CF000CC61593900006139753948CC61BB340069
:102D0000F786399C3951CC61A13400F7B239BF390B
:102D100050CC61A13400F7D339DD3949CC61BB34E3
:102D200000F7EE39EE394ACC61BB3400F7F439F4E0
:102D3000394BCC61BB3400F7FA39FA394CCC61BB62
:102D40003400F7003A003A4DCC61BB3400F70C3A3E
:102D50000C3A4ECC61BB3400F7183A183A4FCC61AC
:102D6000BB3400F7243A243A52CC61BB3400F72C30
:102D70003A423A53CC61BB3400F7583A693A54CCE2
:102D800061BB3400F77A3A863A55CC61BB3400F720
:102D9000923A9F3A56CC61A13400F7AB3AC13ACE91
:102DA000CC619B330000D73AD73ADDCC619B33002E
:102DB00000E23AE23A5CCC61A13400F7F13A073B19
:102DC0006FCC61BB3400F71D3B1D3B40105E000023
:102DD00000002D3B3C3B41CC61BB3400F74A3B4AF1
:102DE0003BD6CC619B330000603B723BD7CC619BF0
:102DF000330000853B923BE1CC619B330000A43B58
:102E0000B93B46CC61BB3400F7CF3BCF3B6DCC61C7
:102E1000BB3400F7CF3BCF3B6ECC61BB3400F7E552
:102E20003BE53B42105E00000000FB3B0A3C43CC0C
:102E300061BB3400F74A3B4A3BD9CC619B3300006D
:102E4000603B723BD8CC619B330000853B923B4496
:102E5000105E00000000183C273C45105E0000009A
:102E6000003B3C4A3C10CC61A13400F75E3C673C1F
:102E700011CC61A13400F7753C7E3C13CC61BB34AE
:102E800000F78C3C9B3C641A5D00000000AA3CAA41
:102E90003CF0006000000000C03CC03C59CC614CDC
:102EA000360000D33CE63CCFCC619B330000F73CBE
:102EB000F73C1ACC61A13400F7043D1A3D66CC61A1
:102EC000A13400F7303D303D65CC61A13400F746B8
:102ED0003D463D1CCC61A13400F75C3D723DDECC2B
:102EE000619B330000883D9B3D1BCC61A13400F702
:102EF000AE3DB63D5DCC61A13400F7C53DDB3D5F25
:102F0000CC61A1340010F13D073ECDCC619B330074
:102F1000001D3E2F3ED0CC619B330000423E583E08
:102F2000DCCC619B3300006D3E803EE0CC619B3386
:102F30000000953EA73E14CC61BB3400F7BC3EBCFC
:102F40003E17CC61BB3400F7BE34BE3415CC61BB38
:102F50003400F7C33EC33E18CC61BB3400F7CA3E11
:102F6000CA3E16CC61BB3400F7D13ED13E3BCC61AA
:102F7000BB3400F7D83EEE3EEDCC619B3300006DD4
:102F800034813412CC61A13400F7FF3EFF3E39CCCE
:102F900061A13400F70F3F253F1ECC61BB3400F721
:102FA0003B3F493F3ACC61A13400F7503F633F19A2
:102FB000CC61A13400F7763F763F5BCC61A1340051
:102FC000F7813F903F1FCC61BB3400F79D3F9D3F91
:102FD00020CC61BB3400F7A93FA93F21CC61BB34B1
:102FE00000F7B53FB53F22CC61BB3400F7C13FC10C
:102FF0003F3CCC61BB3400F7CD3FCD3F3DCC61BB06
:103000003400F7D93FD93F3ECC61BB3400F7E53FF0
:10301000E53F3FCC61BB3400F7F13FF13FECCC61C1
:103020009B3300004C345E3434CC61BB3400F7FD7C
:103030003F104035CC61BB3400F72340364036CCDE
:1030400061BB3400F749405840FF00000000000019
:10305000000000004E4F2052414D21004B616EE4B4
:103060006C65004368616E6E656C004B6F6E6669DF
:103070006775726174696F6E00436F6E666967751C
:10308000726174696F6E00537469636B004C6F6F8B
:1030900070696E670048F6686500416C7469747504
:1030A0006465004B616D6572610043616D657261BD
:1030B000004E6176692D4374726C0041757367E44C
:1030C0006E6765004F757470757473005665727322
:1030D0006368696564656E6573004D697363656CEB
:1030E0006C616E656F7573004779726F0042656E33
:1030F00075747A6572005573657200416368736B0D
:103100006F70706C756E6700436F75706C204178DE
:1031100065730045617379205365747570006E693D
:103120006368742076657266FC67626172002120B4
:103130004552524F52202100767374723A20257303
:1031400000767374723A2025730076616C75653A67
:10315000257500666F726D61743A202573002553E2
:10316000006E696368742076657266FC67626172DE
:10317000004E4121003E2025336400C46E64657218
:103180006E00253364003E202531385300C46E6440
:1031900065726E003D2025303375001200284269AB
:1031A00074313D49646C6529001800302F312020AE
:1031B000201920202020202020202020204F4B00DC
:1031C000C46E6465726E0025303375003E20253173
:1031D000387300C46E6465726E0056616C75653A32
:1031E0002025337500436F6465203A204525303231
:1031F00075006D6B706172616D65746572732E63BD
:1032000000204552524F522000452530327500258E
:1032100033750020204E004E65696E004E6F002011
:10322000204A00202059004A61005965730020504F
:10323000257500506F74692025750043253275008F
:103240004B616E616C202575004368616E6E656C24
:103250002025750053253275005365722E204B6171
:103260006E616C202575005365722E204368616E77
:103270006E656C20257500417573004F66660057BA
:1032800050450057502D4576656E74004D696E00AF
:103290004D696E696D756D004D6964004D6974749A
:1032A00065004D6964646C65004D6178004D61781E
:1032B000696D756D0020416E00204F6E004672658D
:1032C00000467265650020434800436F6D696E6774
:1032D00020486F6D65202843482900205048005041
:1032E0006F736974696F6E20486F6C642028504852
:1032F00029004469730044697361626C6564004F1E
:1033000075253175004F75742025317500430047D0
:103310006173007468726F74746C650047656172E4
:10332000004E69636B00526F6C6C004143535755FC
:103330004D5800506F7469203100506F746920320D
:1033400000506F7469203300506F7469203400504E
:103350006F7469203500506F7469203600506F74A7
:1033600069203700506F7469203800444353574F29
:10337000004D6F746F7220536963686572682E53D5
:103380006368616C742E006D6F746F722073616678
:1033900065747920737769746368003031004D6F0C
:1033A000746F72205377692E4D6F64650045727794
:1033B0002E20456D70662E5369672E5072FC66751F
:1033C0006E6700656E682E207265632E20736967D4
:1033D0006E2E20636865636B00416C6C65732041E1
:1033E0006E736167656E00737065616B20616C6CF4
:1033F0000048F668656E726567656C756E67006893
:10340000656967687420636F6E74726F6C004750F3
:103410005320416B746976004B6F6D70617373203C
:10342000416B74697600636F6D7061737320616BBB
:10343000746976004B6F6D70617373204669780014
:10344000636F6D70617373206669780041636873A0
:1034500028656E74296B6F70706C756E67002844F8
:103460006529436F75706C204178657300447265FF
:1034700068726174656E62656772656E7A756E6793
:1034800000726F746172792072617465206C696D6D
:1034900069742E0048656164696E6720486F6C64CA
:1034A0000076004E69636B2F526F6C6C2050004E9B
:1034B00069636B2F526F6C6C204400765000476933
:1034C00065722050004578742E204B6F6E74726FB9
:1034D0006C6C65006578742E20636F6E74726F6C0F
:1034E000004C6F6F70696E67204F62656E006C6F85
:1034F0006F70696E67207570004C6F6F70696E67D2
:1035000020556E74656E006C6F6F70696E67206415
:103510006F776E004C6F6F70696E67204C696E6BD1
:1035200073006C6F6F70696E67206C656674004C19
:103530006F6F70696E6720526563687473006C6F9B
:103540006F70696E67207269676874004C6F6F7086
:10355000696E6720476173204C696D6974006C6FF8
:103560006F70207468726F74746C65206C696D691B
:103570007400416E73707265636873636877656C1D
:103580006C6500726573706F6E7365207468726528
:1035900073686F6C64004879737465726573650055
:1035A00068797374657265736973004E69636B2023
:1035B000556D6B65687270756E6B74006E69636BC8
:1035C000207475726E6F76657200526F6C6C205548
:1035D0006D6B65687270756E6B7400726F6C6C20C9
:1035E0007475726E6F7665720048F668656E626516
:1035F0006772656E7A756E670068656967746820C2
:103600006C696D69746174696F6E00566172696F7F
:103610002D48F6686500766172696F206865696794
:10362000746800536368616C7465722048F668655D
:1036300000686569676874207377697463680061FE
:103640006B7573742E20566172696F004443535733
:103650004F4E0048F6686520536F6C6C7765727446
:1036600000686967687420736574706F696E7400B0
:103670004D696E2E20476173006D696E2E2074684F
:10368000726F74746C650048F66865205000616C58
:103690007469747564652050004C75667464727545
:1036A000636B2044006261726F6D657472696320A0
:1036B00044005A2D414343004D61782E2048F6685E
:1036C000652020202020202020205B6D5D006D6182
:1036D000782E20616C746974756465202020202028
:1036E0005B6D5D005665727374E4726B2E2F5261D0
:1036F0007465006761696E20726174650053636868
:10370000776562652D47617300686F6F766572201B
:103710007468726F74746C6500475053205A00537C
:103720007469636B204E657574722E50756E6B7480
:1037300000737469636B206E657574722E706F69A7
:103740006E7400444353004175746F20537461726A
:10375000744C616E64204B616E616C006175746FB6
:103760002073746172742F6C616E64206368616E83
:103770002E004C616E64696E67205370656564202D
:1037800020302E316D2F73004E69636B20416E73B4
:103790007465756572756E67006E69636B2073651D
:1037A00072766F206374726C004E69636B204B6F8E
:1037B0006D70656E736174696F6E006E69636B2006
:1037C000736572766F20636F6D702E004E69636B48
:1037D000204B6F6D702E20417573006E69636B20F6
:1037E000636F6D70656E736174696F6E206F66666E
:1037F000004E69636B20556D6B656872656E006E77
:1038000069636B20696E762E2064697265637469E2
:103810006F6E004E69636B2052656C61746976004F
:103820006E69636B2072656C61746976004E6963C2
:103830006B20536572766F204D696E696D756D00F2
:103840004E69636B20536572766F204D6178696DA8
:10385000756D004E69636B2046696C746572006E0D
:1038600069636B2066696C74657200526F6C6C20C2
:10387000536572766F20416E73742E00726F6C6C9C
:1038800020736572766F206374726C2E00526F6CB9
:103890006C204B6F6D70656E736174696F6E007232
:1038A0006F6C6C20636F6D70656E736174696F6EA1
:1038B00000526F6C6C20556D6B656872656E0052BE
:1038C0006F6C6C20696E762E206469726563746912
:1038D0006F6E00526F6C6C204D696E696D756D0076
:1038E000526F6C6C204D6178696D756D00526F6C14
:1038F0006C2046696C74657200726F6C6C2066692E
:103900006C74657200416E73742E20476573636832
:10391000772E00736572766F2072656672657368C4
:10392000004D616E752E204765736368772E006DBC
:10393000616E75656C6C20537065656400765450DB
:1039400000536572766F203300536572766F2034B2
:1039500000536572766F20350044435357464851F3
:1039600000475053204D6F6475732053746575651F
:1039700072756E6700475053206D6F646520636FEA
:103980006E74726F6C00475053205665727374E406
:10399000726B756E672020205B255D0047505320B9
:1039A0006761696E202020202020202020205B25B8
:1039B0005D004750532053742D536368772E0047A2
:1039C000505320737469636B207468726573686FF9
:1039D0006C64004D696E2E205361742E006D696E0B
:1039E000696D756D20736174656C6974650047500D
:1039F000532D50004750532D49004750532D44003C
:103A00004750532D50204C696D6974004750532D19
:103A100049204C696D6974004750532D44204C690E
:103A20006D69740047505320416363004750532031
:103A300057696E646B6F7272656B747572205B256B
:103A40005D004750532077696E6420636F72726522
:103A500063742E205B255D00414343204B6F6D70E6
:103A6000656E736174696F6E0041434320636F6DCF
:103A700070656E736174696F6E006D61782E20528F
:103A80006164697573006D61782E20726164697577
:103A9000730057696E6B656C204C696D69740061C9
:103AA0006E676C65206C696D6974005048204C6FBE
:103AB00067696E205A65697420202020205B735D41
:103AC000005048206C6F67696E2074696D65202016
:103AD0002020205B735D0044796E616D6963205026
:103AE00048004D61782E52616469757320645048B6
:103AF00000436F6D2E486F6D652048F66865202085
:103B00002020205B6D5D00636F6D696E6720686FBC
:103B10006D6520616C74692E205B6D5D0053696E6C
:103B2000676C65205750205370656564004C4544B0
:103B3000313A204269746D61736B65004F75743161
:103B40003A206269746D61736B0054696D696E67C8
:103B50002020202020202020205B31306D735D004C
:103B60006E75722077656E6E204D6F746F72204196
:103B70006E006F6E6C792077697468206D6F746F5A
:103B800072206F6E00201920736F666F727420614F
:103B90006E00201920696D6D6564696174656C79CA
:103BA000206F6E006D69742057502D4576656E74D8
:103BB00020207665726B6E2E00636F6D62696E6594
:103BC00020776974682057502D4576656E740041E2
:103BD00075746F20547269676765722044697374E5
:103BE0002E5B6D5D004175746F2054726967676567
:103BF0007220416C742E205B6D5D004C4544323A5E
:103C0000204269746D61736B65004F7574323A20A0
:103C10006269746D61736B004C4544312057617269
:103C20006E2055426174004F75743120756E646565
:103C300072766F6C74207761726E004C454432204E
:103C40005761726E2055426174004F757432207551
:103C50006E646572766F6C74207761726E004D6968
:103C60006E2E20476173006D696E2E207468726F2E
:103C700074746C65004D61782E20476173006D612E
:103C8000782E207468726F74746C65004B6F6D7061
:103C90006173737769726B756E6700636F6D7061C6
:103CA00073732065666665637400436F6D7061733E
:103CB00073204F6666736574202020205B0B5D00C7
:103CC00044697361626C65204465636C2E204361B6
:103CD0006C63004361726546726565205374657557
:103CE0006572756E67006361726546726565206313
:103CF0006F6E74726F6C00546561636861626C65AD
:103D000020434600556E7465727370616E6E756EF9
:103D10006720205B302E31565D00756E64657276CB
:103D20006F6C746167652020205B302E31565D001A
:103D3000436F6D696E6720482E20566F6C74205B50
:103D4000302E31565D004175746F6C616E642E20AB
:103D5000566F6C74205B302E31565D004E4F542DE3
:103D6000476173205A6569742020205B302E3173BF
:103D70005D00456D6572672E5468726F2E54696DD3
:103D8000655B302E31735D004E4F542D47617320BB
:103D9000566172696F2048F6686500456D65726707
:103DA0002E7468722E766172696F20682E004E4FF5
:103DB000542D47617300456D6572672E5468726FAC
:103DC00074746C65004661696C732E204348205AF8
:103DD000656974202020205B735D006661696C73E7
:103DE0002E2043482074696D65202020205B735D80
:103DF000004661696C732E204368616E6E656C20AD
:103E000020303D417573006661696C732E206368D4
:103E1000616E6E656C2020303D6F6666006B2E53C0
:103E2000756D6D6572206F2E53656E646572006EE0
:103E30006F206265657020776974686F75742054AF
:103E400058004B6F6D70617373204665686C6572C6
:103E50002069676E6F722E0069676E6F72652063EE
:103E60006F6D70617373206572726F72006B2E5389
:103E700074617274206F2E53442D4B61727465000F
:103E80006E6F20737461727420772F6F2053442DEE
:103E900063617264006B2E5374617274206F2E47DD
:103EA000505320466978006E6F20737461727420DD
:103EB000772F6F2047505320466978004779726FFB
:103EC0002050004779726F20490047696572204988
:103ED000004779726F20440044796E616D697363A5
:103EE00068652053746162696C6974E47400647974
:103EF0006E616D69632073746162696C69790041F8
:103F000043432F4779726F2046616B746F72004193
:103F100043432F4779726F204B6F6D702E20205BCB
:103F2000312F785D004143432F4779726F20436FF3
:103F30006D702E20205B312F785D004861757074A4
:103F40007265676C65722049006D61696E20490079
:103F500044726966742D4B6F6D70656E7361746920
:103F60006F6E00647269667420636F6D70656E7346
:103F70006174696F6E004779726F20737461622E8D
:103F8000004D6F746F7220476CE47474756E670037
:103F90006D6F746F7220736D6F6F74680050617213
:103FA000616D65746572203100506172616D657478
:103FB0006572203200506172616D657465722033E4
:103FC00000506172616D65746572203400506172D9
:103FD000616D65746572203500506172616D657444
:103FE0006572203600506172616D657465722037AC
:103FF00000506172616D65746572203800476965B3
:104000007220706F732E204B6F70706C756E67002E
:104010006769657220706F732E20636F75706C69AD
:104020006E67004E69636B2F526F6C6C204B6F7024
:10403000706C756E67006E69636B2F726F6C6C20AD
:10404000636F75706C696E670047696572204B6FAE
:104050007272656B747572006769657220636F7246
:1040600072656374696F6E004D4B2053657474699B
:104070006E67730025313573004E4F2052414D213C
:1040800000FE6F6B0CFE01FF00FE706B0CFE01FF6B
:1040900000FE726B0CFE01FF000101020C03010423
:1040A00001050106010701080109010A010B010CC4
:1040B000010D010E010F0110011101120113011474
:1040C00001150116011701180119011A011B011C24
:1040D000011D011E011F01200121012201230124D4
:1040E00001250126012701280129012A012B012C84
:1040F000012D012E012F0130013101320133013434
:1041000001350136013701380139013A013B013CE3
:10411000013D013E013F0140014101420143014493
:1041200001450146014701480149014A014B014C43
:10413000014D014E014F01500151015201530154F3
:1041400001550156015701580159015A015B015CA3
:10415000015D015E015F0160016101620163016750
:1041600001680169016A016B0C6C01FF0001010229
:104170000C03010401050106010701080109010AF8
:10418000010B010C010D010E010F011001110112B3
:104190000113011401150116011701180119011A63
:1041A000011B011C011D011E011F01200121012213
:1041B0000123012401250126012701280129012AC3
:1041C000012B012C012D012E012F01300131013273
:1041D0000133013401350136013701380139013A23
:1041E000013B013C013D013E013F014001410142D3
:1041F0000143014401450146014701480149014A83
:10420000014B014C014D014E014F01500151015232
:104210000153015401550156015701580159015AE2
:10422000015B015C015D015E015F01600161016292
:10423000016301640165016701680169016A016B3D
:104240000C6C01FF000101020C03010401050106D1
:10425000010701080109010A010B010C010D010E02
:10426000010F0110011101120113011401150116B2
:10427000011701180119011A011B011C011D011E62
:10428000011F012001210122012301240125012612
:10429000012701280129012A012B012C012D012EC2
:1042A000012F013001310132013301340135013672
:1042B000013701380139013A013B013C013D013E22
:1042C000013F0140014101420143014401450146D2
:1042D000014701480149014A014B014C014D014E82
:1042E000014F015001510152015301540155015632
:1042F000015701580159015A015B015C015D015EE2
:10430000015F016001610162016301640165016691
:10431000016701680169016A016B0C6C01FF000112
:1043200001020C030104010501060107010801094E
:10433000010A010B010C010D010E010F0110011109
:1043400001120113011401150116011701180119B9
:10435000011A011B011C011D011E011F0120012169
:104360000122012301240125012601270128012919
:10437000012A012B012C012D012E012F01300131C9
:104380000132013301340135013601370138013979
:10439000013A013B013C013D013E013F0140014129
:1043A0000142014301440145016D014701480149B2
:1043B000014A014B014C014D014E014F0150015189
:1043C0000152015301540155015601570158015939
:1043D000015A015B015C015D015E015F01600161E9
:1043E00001620163016401650166016E016F01678D
:1043F00001680169016A016B0C6C01FF00FE7B6BB7
:104400000CFE01FF000101020C030104010501067D
:10441000010701080109010A010B010C010D010E40
:10442000010F0110011101120113011401150116F0
:10443000011701180119011A011B011C011D011EA0
:10444000011F012001210122012301240125012650
:10445000012701280129012A012B012C012D012E00
:10446000012F0130013101320133013401350136B0
:10447000013701380139013A013B013C013D013E60
:10448000013F014001410142014301440145016DE9
:10449000014701480149014A014B014C014D014EC0
:1044A000014F015001510152015301740155015650
:1044B0000175015701580159015A015B015C015D09
:1044C000015E015F016001610170017101720173A0
:1044D00001620163016401650166016E016F01679C
:1044E00001680169016A016B0C6C01FF00BE680183
:1044F000010000BF6801020000C06801040000C89C
:104500006901010000C96902010000CA69010200D5
:1045100000CB6901040000CC6901080000CD6901ED
:10452000100000CE6901200000CF6901400000D0DA
:104530006901800000D26701010000D36701020019
:1045400000D46701040000D56701080000D66701A8
:10455000100000D76701200000D86701400000D993
:104560006701800000DC6A01010000DD6A010200D1
:1045700064DE6A01040000DF6A01080000E06A01ED
:10458000100000E16A01200000E26A01400000E33F
:104590006A01806000E60301010000E703010200F8
:1045A00000E80301040000E90301080000EA030138
:1045B000100000EB0301200000EC0301400000EDBF
:1045C0000301800000AA0203000000AB0203010007
:1045D00000AC0203020000AD0203030000AE0203C0
:1045E000040000AF0203050000B00203060000B1A2
:1045F0000203070000B20203080000B3020309002F
:1046000000B402030A0000B502030B0000F06403CB
:10461000000000FF00000000001D00200020001D21
:1046200000416C6C001D001A201B0056616C756502
:104630003A20202030004D6F746F723A20202031D4
:104640000020424C2D4374726C20546573742020FA
:10465000202020202020000A481348254839484DB2
:10466000486148764888489748A748BB48C848D515
:1046700048E148ED48F948024912491949244930AE
:10468000493F49484955496349714980498B499E89
:1046900049AC49B949C449D849E449F449034A04F1
:1046A0004A054A064A074A084A0E0F0E4E0E0F0EDA
:1046B0004F0E0F0E530E0F0E570E0F0E4E0E0F0E07
:1046C0004F0E0F0E530E0F0E570E0F0E4E0E0F0EF7
:1046D0004F0E0F0E530E0F0E57144A174A1A4A1D4B
:1046E0004A204A234A264A294A496E666F0055479E
:1046F0007073006C6F6E672070726573733A003A66
:10470000002A2A204D4B2D4572726F7220202020E6
:104710002A2A004D4B2053657474696E6700504B14
:1047200054204F5344000B43006D617820424C20CD
:104730002054656D703A006D617820424C20204312
:104740007572723A006D41680020202030006B6D58
:104750006800730041006D4168006D4168006D00A4
:1047600055475053006D00486F6D653A00416C74B9
:104770003A00206B6D68002020493A004469723A83
:1047800000416C743A00206D41005750006D730079
:104790006D202D005A69656C0020536174005043F0
:1047A000002020006D202D00486F6D65004B6D6866
:1047B000006D0041006D41680056005600760053C0
:1047C000006D0048F66865004D4300545200534C9C
:1047D00000524C00465200544400545500532100EE
:1047E000475000465300454C004659004D52005377
:1047F00054004341004241006F32006F3100434892
:10480000004346005048004148004E6F20457272F8
:104810006F72004643206E6F7420636F6D70617419
:1048200069626C65004D4B334D6167206E6F74207B
:10483000636F6D706174692E006E6F204643206354
:104840006F6D6D756E69636174696F6E006E6F2058
:104850004D4B334D616720636F6D6D756E69632ECF
:10486000006E6F2047505320636F6D6D756E6963E6
:104870006174696F6E0062616420636F6D70617353
:10488000732076616C7565005243205369676E61D1
:104890006C206C6F737400464320737069207278CB
:1048A000206572726F72006E6F204E4320636F6DD1
:1048B0006D756E69636174696F6E004643204E6961
:1048C000636B204779726F00464320526F6C6C20F7
:1048D0004779726F00464320596177204779726F9C
:1048E000004643204E69636B20414343004643200A
:1048F000526F6C6C20414343004643205A2D414384
:10490000430050726573737572652073656E736FC3
:10491000720046432049324300426C204D69737354
:10492000696E67004D69786572204572726F72001A
:104930004361726566726565204572726F720047E9
:104940005053206C6F7374004D61676E6574204521
:1049500072726F72004D6F746F7220726573746142
:10496000727400424C204C696D69746174696F6E99
:1049700000576179706F696E742072616E676500AF
:104980004E6F2053442D43617264005344204C6F9A
:104990006767696E672061626F7274656400466C58
:1049A00079696E672072616E676521004D617820BC
:1049B000416C746974756465004E6F2047505320D4
:1049C00046697800636F6D70617373206E6F742039
:1049D00063616C6962722E00424C2073656C667470
:1049E000657374006E6F206578742E20636F6D7030
:1049F00061737300636F6D706173732073656E73A1
:104A00006F72000000000000504B54205258206C80
:104A10006F7374004E45004520005345005320003D
:104A20005357005720004E57004E20004F5344204C
:104A3000446174656E004F534420646174610042A8
:104A40004C2020446174656E00424C2020646174E7
:104A500061004D4B20204665686C65726C6973740B
:104A600065004D4B20206572726F72736C697374B0
:104A7000004750532042656E75747A65726C697395
:104A800074650047505320757365726C69737400C8
:104A9000475053206C65747A746520506F732E00F4
:104AA000475053206C61737420506F732E004CD6A6
:104AB0005343484520616C6C6520446174656E0009
:104AC00044454C45544520616C6C20646174610020
:104AD0004F534420446174656E0044656C00253278
:104AE00030530020436F6465202530327500253037
:104AF00032753A253032753A25303275202025300E
:104B000032752E253032752E2530347500204D4BF0
:104B1000204572726F72730025332E366C64253314
:104B20002E366C6400253764206D4725352E3164A0
:104B3000206D4200253032752E253032752E2530FD
:104B400034752020253032753A253032753A2530BB
:104B50003275002055736572204750530020202580
:104B60006354656D702E2538752025634300202021
:104B7000256343757272656E7425342E317520413C
:104B8000002531643A256343757272656E7425346D
:104B90002E317520410020424C2044617461002573
:104BA00063424C2531642054656D702E2025357587
:104BB00020256343002563424C25316420437572F0
:104BC00072656E7425322E31752041002563437560
:104BD0007272656E7425362E316420410025634360
:104BE000757272656E7425362E3164204100204244
:104BF0004C20537461746973746963002563526F48
:104C00006C6C25313164202563002563526F6C6C18
:104C1000253131642025630025634E69636B25319E
:104C200031642025630025634E69636B253131644F
:104C300020256300256352432D5175616C69747999
:104C400025356400256352432D5175616C69747973
:104C5000253564002563566F6C7461676525362EB3
:104C600031642056002563424C2531642054656D23
:104C7000702E2025357520256343002563424C2581
:104C8000316420437572722E25342E317520410017
:104C9000256343757272656E7425362E316420412A
:104CA00000256343757272656E7425362E3164205B
:104CB0004100204361706163697479253764206D18
:104CC0004168002563566572742E537065656425CE
:104CD000332E3164206B6D6800256347726E642E3D
:104CE000537065656425332E3164206B6D68002533
:104CF0006344697374616E6365253775206D0025A3
:104D000063416C746974756465253764206D002097
:104D10004C61737420466C792020253032753A2519
:104D2000303275206D696E00204F534420537461FA
:104D300074697374696300456E643A2020202530DD
:104D400032753A253032752020253032752E2530C7
:104D500032752E00426567696E3A20253032753A09
:104D6000253032752020253032752E253032752EB3
:104D70000020202020206E6F20646174612E2E2E72
:104D800000323030382054686F6D6173204B616998
:104D900073657200323030392D3230313020506539
:104DA000746572204D61636B003230313020536581
:104DB0006261737469616E20426F65686D003230A4
:104DC00031322067656261640032303132204D61DA
:104DD0007274696E2052756E6B656C002020202005
:104DE00020486172616C6420426F6E676172747AF0
:104DF0000032303132204368722E204272616E647C
:104E0000746E65720032303133204F6C6976657292
:104E10002047656D6573690020437265646974732A
:104E20000000466F6E742042696700493243204D8E
:104E30006F746F7274657374004A6F797374696309
:104E40006B00466F6C6C6F77204D65005472616328
:104E50006B696E6700536F756E64004F5344205347
:104E60007461746973746963004F53442033442D33
:104E70004C616765004F534420557365724750532A
:104E8000004F5344204D4B537461747573004F535E
:104E90004420456C656374726963004F5344204E2F
:104EA000617669676174696F6E004F5344204F6C7F
:104EB000642053637265656E73004F53442D4461E3
:104EC0007461004D4B20446973706C6179004D4BE7
:104ED0002044656275672044617461004D4B205326
:104EE000657474696E677300574C414E205779465C
:104EF0006C7900426C7565746F6F746800204D6F3B
:104F000064756C657320696E7374616C6C656400A4
:104F100025313553202534530000202020204E4FCA
:104F20002057415252414E54590028432920474EA0
:104F3000552047504C204C6963656E736500003303
:104F40002E382E30610020504B54207625385320C7
:104F5000257300504B5420557064617465002532F0
:104F60003073002532305300332E382E306100501C
:104F70004B5420760056657262696E64756E6720C8
:104F80004D4B00636F6E6E656374696F6E204D4BA1
:104F900000504B5420616C6C67656D65696E005004
:104FA0004B542067656E6572616C0057692E323311
:104FB0003200426C7565746F6F746800426C756581
:104FC000746F6F746820424C4500574C414E205717
:104FD00069466C79004F534420416E7A6569676574
:104FE000004F53442073637265656E004750532031
:104FF0004D61757300475053206D6F757365005494
:105000007261636B696E6720536572766F730074AB
:105010007261636B696E6720736572766F73004AA5
:105020006F79737469636B00504B542055706461E1
:10503000746500454550726F6D205265736574004C
:105040004F53442053637265656E7300504B542078
:1050500053657475700053707261636865006C61AC
:105060006E6775616765005A6569747A6F6E650071
:1050700074696D65207A6F6E6500536F6D6D657232
:105080007A6569740073756D6D65722074696D65FC
:10509000004C434420617573206E6163682E2E2E90
:1050A000004C4344206F6666206166746572004C54
:1050B00043442048656C6C69676B656974004C43B8
:1050C00044206272696768746E657373004C434470
:1050D000204B6F6E7472617374004C434420636F95
:1050E0006E7472617374004C4344204E6F726D6134
:1050F0006C2F496E76657273004C4344206E6F725C
:105100006D616C2F696E76657274004861726477A8
:105110006172652042656570657200416B6B7574E4
:105120007970004163637574797000416B6B752011
:105130004D657373756E6700416363754D6561738B
:1051400075726500504B5420616C6C67656D6569C4
:105150006E0054582F5258204B616E616C005458A9
:105160002F5258204368616E6E656C004E6574570F
:105170002E20477275707065004E6574572E20475B
:10518000726F7570004E6574572E204D6F64650008
:1051900054582054696D656F7574005458204D54EF
:1051A000550042617564726174652057693233320B
:1051B0002F425400496E697469616C697369657244
:1051C000656E00696E697469616C697A65004B6F20
:1051D0006E6669672E206D697420504300636F6EA0
:1051E0006669672E20776974682050430057692EDE
:1051F00032333220536574757000424C452053653C
:10520000747570002052452D4944204E6F74697AA0
:10521000003A004D41433A002042544D2D32323283
:10522000204D41432D4164726573736520004254E3
:1052300020496E6974204572726F72004254204991
:105240006E6974206F6B0020426C7565746F6F74AB
:10525000682050696E0020426C7565746F6F7468C9
:10526000204E616D65004D6F64756C2065696E67D9
:1052700065626175743F006D6F64756C6520627561
:10528000696C7420696E3F004E616D65006E616DE2
:10529000650050696E0070696E00426C7565746FD0
:1052A0006F7468204D41430052452D494400426CC3
:1052B0007565746F6F7468205365747570005375ED
:1052C00063686520475053204D61757300736561B5
:1052D00072636820475053206D6F757365005A657F
:1052E00069676520476572E474656C69737465006D
:1052F00073686F77206465766963656C69737400A1
:105300005A6569676520475053204465766963652F
:105310000073686F77204750532064657669636532
:1053200000475053204D61757320547970004750E9
:1053300053206D6F7573652074797000475053204A
:105340004D61757320616B7469763F00475053203F
:105350006D6F7573652061637469763F00475053C4
:1053600020446174656E004750532064617461008D
:10537000475053204D6F75736520536574757000E9
:105380004F53442053637265656E73004F5344203E
:10539000536574757000566F6C743A00204645482A
:1053A0004C45522120312E205A65696368656E2173
:1053B0002000201720202020201620202020201927
:1053C000202020204F4B00202020202020202020A3
:1053D000202020204300200025005769323332006E
:1053E000576932333200253853004164486F6300F7
:1053F00041502D4D6F646500756E6B6E6F776E005A
:1054000062697474652077617274656E2E2E2E0049
:10541000475053207472656E6E656E006C6F7374C6
:105420002042542064617461006D0020202D2D2DD8
:1054300000416C743A2000204C6174697475646595
:105440002020204C6F6E6769747564650048444F76
:10545000503A20004669783A2000584572723A2046
:10546000005361743A20004F4B004572726F7220F6
:10547000636F6E6E656374696E6721007472792064
:10548000746F20636F6E6E656374006B6F6E666918
:105490006775726965727421006B65696E65204776
:1054A0005053204D617573007375636865204254D5
:1054B00020446576696365004254204465766963DB
:1054C00065732073756368656E3F00616B74756505
:1054D0006C6C6573204254204465766963653A209C
:1054E0000042542073656C6563742044657669637B
:1054F000650073756368656E210042697474652088
:10550000657273742042542D446576696365730037
:105510004D41433A004465766963653A0065696EBA
:1055200067656261757421006B65696E2042544D38
:10553000323232004F4B0042542D4D6F757365313E
:10554000004D696B726F6B6F7074003234303020B5
:105550002000393630302020003139323030200000
:105560003338343030200035373630302000313198
:105570003532303000343830302020004C69496FEB
:105580006E004C69706F2000194F1800207365720F
:1055900069656C6C6520506F74697320312D3520FE
:1055A00000DC62657273696368740073756D6D61A8
:1055B000727900537469636B203100537469636BB3
:1055C000203200537469636B203300537469636B3A
:1055D000203400537469636B203500504B54204CC9
:1055E00069706F6D657373756E6700504B54204C16
:1055F00069706F206D6561737572652E004A6F79F1
:10560000737469636B205365747570004D696E69BE
:105610006D616C2057657274006D696E696D616CA7
:105620002076616C7565004D6178696D616C2057FD
:10563000657274006D6178696D616C2076616C755E
:10564000650054797065007479706500526963680B
:1056500074756E6700646972656374696F6E004E7D
:1056600065757472616C69736965726564006E65F5
:10567000757472616C697A696E67004A6F797374C8
:1056800069636B004F4B00504B54204C69706F6D39
:10569000657373756E672020200059004E005265B7
:1056A00076004E6F726D005461737400506F7469B0
:1056B0000053204D696E204D617820547970202070
:1056C00044697220204E002020204A6F797374694B
:1056D000636B20536574757020202020005556F7A9
:1056E00032EE1AAB0DDC066F03B801DC006E00373A
:1056F000001B000E0007000300020001005365724A
:10570000766F736368726974746500736572766F1F
:1057100020737465707300536572766F2031005387
:105720006572766F203200536572766F746573749C
:1057300000547261636B696E6720536572766F7394
:1057400000546573742050756C736CE46E6765006B
:10575000746573742070756C732077696474680065
:105760005465737420666F72746C66642E00746581
:10577000737420636F6E742E00536572766F0050E1
:105780006572696F6465006672616D65005365726C
:10579000766F74657374005374617274205465730A
:1057A0007400737461727420746573740045696E5B
:1057B0007A656C736368726974740073696E676C80
:1057C00065207374657000416E7A61686C20546561
:1057D0007374006E756D626572206F6620746573F8
:1057E0007400506175736520456E64706F736974E1
:1057F000696F6E00706175736520656E6420706FEF
:10580000730050617573652070726F20496E632E4E
:105810000070617573652070726F6320696E632E0E
:1058200000536572766F7465737420436F6E742EC7
:105830000052657665727365007265766572736590
:10584000004C696E6B73006C65667400526563682A
:105850007473007269676874004D69747465006DD3
:105860006964646C6500536572766F2041646A7583
:10587000737400536572766F203200536572766FD1
:10588000203100536572766F3A00010000000A0073
:10589000000064000000E803000010270000A0865C
:1058A000010040420F008096980000E1F50500CA13
:1058B0009A3B456E64650020547261636B696E6744
:1058C000204D696B726F6B6F7074657200547261FA
:1058D000636B696E6720426C7565746F6F746820C6
:1058E0002020006C6F73742057692E32333220648D
:1058F00061746100475053206F6B2C207374617288
:1059000074206F6B202000202020202020202020C9
:10591000202020202020202020005768616974204A
:10592000666F72204750532046697820005768619F
:10593000697420666F7220475053204669782000B2
:1059400053204C6174697475646520204C6F6E67D8
:105950006974756465004665686C65722062656986
:105960006D205472656E6E656E007377697463683E
:10597000206F6E204254204D6F75736521210045C4
:1059800072726F7220617420636F6E6E65637469EA
:105990006E6700475053207472656E6E656E006CC2
:1059A0006F737420425420646174610048444F5006
:1059B0003A004669783A005361743A004D00480055
:1059C00053204C6174697475646520204C6F6E6758
:1059D0006974756465004641494C00204F4B2000B6
:1059E000203F3F200054696C743A0050616E203AA9
:1059F000006D00446973743A001E00426561723A9A
:105A00000025632563253137732000256325632531
:105A100031367325632000256325632531375320F4
:105A20000025632563253136532563200025632532
:105A30006325313453202533730000256325632506
:105A4000313853002535530025345300202532309A
:105A50007300202532305300202025313973002077
:105A600020253139530020202020206E6F742070B3
:105A70006F737369626C65202020200020455252AC
:105A80004F525F4E4F4954454D2020002045525201
:105A90004F525F4D41584954454D200020455252C8
:105AA0004F525F4D41584D454E55200020455252B2
:105AB0004F525F4E4F4D454E55202000206D656E74
:105AC000756374726C2E6320212120002020202019
:105AD000004E6F206D6F72652052414D004572720D
:105AE0006F723A205363726F6C6C426F7800576923
:105AF0002E323332204E414B005769323332204927
:105B00006E69744572726F722020005769323332A9
:105B100020496E6974206F6B2E2E2E2E005769322D
:105B2000333220496E69744572726F722020002EE4
:105B3000002E002E002E002E002E002E002E002EF5
:105B4000002E002E002E002E002E002E002E002EE5
:105B5000002E002E00496E697420576932333220BE
:105B6000776169742E2E2E2E0056657273696F6EE2
:105B70003A004572726F72207365742052414D2055
:105B800020202020004572726F7220736574204EB1
:105B9000562D52414D0057692E3233322077726FA5
:105BA0006E672042617564726174650057692E32B8
:105BB000333220666F756E64200057692E3233329F
:105BC0002053797461786572726F72202020006EA4
:105BD0006F2057692E32333220666F756E64007302
:105BE00065617263682057692E323332204D6F64CD
:105BF000756C003131353230300020353736303079
:105C00000020333834303000203139323030002039
:105C1000203936303000202032343030002077698F
:105C200074682020202020202020426175640076A6
:105C3000657273696F6E2067657400636F6D6D6167
:105C40006E646D6F646520656E7465720052657375
:105C50006574204641494C21005265736574204F9C
:105C60004B210025533F00526573657420576946E8
:105C70006C7900322E33382E3300342E34310055F7
:105C80007064617465204F4B2100557064617465C8
:105C9000204641494C2100555044415445204F4B2A
:105CA0000066747020757064617465207769666C35
:105CB00079372D3434312E696D6700555044415485
:105CC00045204F4B006674702075706461746520C8
:105CD0007769666C79372D323338332E696D6700FA
:105CE000555044415445204F4B00667470206375F5
:105CF0007064617465207769666C79372D3434314E
:105D00002E696D6700555044415445204F4B006645
:105D100074702063757064617465207769666C794E
:105D2000372D323338332E696D6700736574206602
:105D300074702074696D656F75742038303000732D
:105D40006574206674702070617373205061737382
:105D50003132330073657420667470207573657218
:105D600020726F76696E67007365742066747020A8
:105D7000646972207075626C696300736574206673
:105D800074702061646472657373203139382E3108
:105D900037352E3235332E313631004654502055AA
:105DA00070646174650073657420776C616E206344
:105DB00068616E6E656C20300073657420776C616D
:105DC0006E2070687261736500736574206970205D
:105DD0006468637020310076657262696E64652064
:105DE0004865696D6E65747A005265736574002547
:105DF000533F0025533A207625530025533A207609
:105E0000257300557064617465205769466C79008C
:105E1000496E6974204F4B2100496E6974204641D8
:105E2000494C210025533F0025533A204F4B005742
:105E300069466C79207625730056657273696F6EBA
:105E4000206E6F20255321004552524F5200576952
:105E5000466C79207625730041502D4D6F646500A6
:105E60004164486F6300496E6974205769466C79D4
:105E7000003136392E3235342E312E31003136395B
:105E80002E3235342E312E31003235352E32353525
:105E90002E302E30007365742061706D6F64652044
:105EA0006C696E6B5F6D6F6E69746F72203000731A
:105EB00065742069702070726F746F636F6C20302E
:105EC00078330073657420776C616E206368616E4F
:105ED0006E656C007365742061706D6F6465207011
:105EE000617373007365742061706D6F64652073F6
:105EF0007369640073657420776C616E20726174DD
:105F000065203300736574206970206E65746D615F
:105F1000736B0073657420697020676174657761C5
:105F200079007365742069702061646472657373AD
:105F30000073657420697020646863702034007396
:105F4000657420776C616E206A6F696E203700730C
:105F5000657420776C616E206368616E0073657490
:105F600020776C616E2073736964007365742069B7
:105F700070206E65746D61736B0073657420697059
:105F8000206761746577617900736574206970209A
:105F90006164647265737300736574206970206452
:105FA00068637020300073657420776C616E206ABE
:105FB0006F696E203400494E49540056657273690A
:105FC0006F6E204641494C210056657273696F6EB1
:105FD0003A20762573005769466C792056657273AE
:105FE000696F6E005769466C79206E6F7420666F1A
:105FF000756E640073657420752062203537363005
:106000003000255320256C7520426175640072654F
:10601000626F6F74004173736F63696174656400CC
:106020006A6F696E0053746F72696E670073617690
:10603000650044656661756C747300666163746FB6
:10604000727920524553455400414F4B00676574A7
:106050002076657273696F6E002424240025642FF6
:10606000256400576C616E2050617373776F7264A2
:1060700000576C616E205353494400576C616E2089
:1060800050617373776F726400576C616E20535365
:1060900049440054455354005769466C79204D6F6C
:1060A000647573005769466C79206D6F646500579D
:1060B00069466C792056657273696F6E3F00535361
:1060C00049440050617373776F7274005061737349
:1060D000776F7264004B616E616C004368616E6E35
:1060E000656C00486F6D65205353494400486F6DDF
:1060F000652050617373776F727400486F6D65200F
:1061000050617373776F7264005769466C792065CC
:10611000696E736368616C74656E005769466C796B
:1061200020706F776572206F6E0052455345543A68
:10613000205769466C79005550444154453A2057E0
:1061400069466C7900494E49543A204164486F636E
:1061500000494E49543A2041502D4D6F6465005717
:1061600069466C79005769466C79204164486F63D1
:10617000005769466C792041502D4D6F64650000D1
:1061800014BE88E10FB6F89480936000109260000E
:106190000FBE11241FBEC0E0D0E4DEBFCDBF14E0AF
:1061A000A0E0B1E0EAE3FCED01E00BBF02C0079024
:1061B0000D92AA3BB107D9F718E2AAEBB4E001C0EF
:1061C0001D92AA3DB107E1F70E94DA500C941BEE34
:1061D0000C940000EBE3FFE08191882319F08E32EC
:1061E000D9F706C080913B0F803211F0882331F43B
:1061F0008BE39FE063E473E00E948FEC8BE39FE00E
:106200000C9476D820E030E048E853E105C0FA016C
:106210003197F1F72F5F3F4F28173907C4F30895DF
:106220008091350F813019F41092BB04089581E0FC
:106230008093BB04089523C00E9452C6BC018070A5
:1062400022E08030920789F022E08130920728F422
:1062500021E08030920779F4089524E0803092079D
:1062600021F028E08030920731F48091BE048F5FE6
:106270008093BE04089580EC94E00E94EF3980EC96
:1062800094E00E94C4398823B9F20895A1E0B0E0F7
:10629000ECE4F1E30C94BFE9682E562E062D192F7D
:1062A0006E010894C11CD11C28E8A22E23E1B22E55
:1062B00094EF892E91E0992E4FC0F80180810E94C1
:1062C0006CC6009709F44DC080911201882341F4F7
:1062D00084EF91E0F4013197F1F70197D9F734C0D9
:1062E000813021F4C5010197F1F72EC0823061F5AC
:1062F0008091BB04813041F522C09DDF81E090E0B8
:1063000081DF0894E11CF11CFAECEF16F10431F086
:1063100080EC94E00E94BB39882379F780EC94E00C
:10632000B6010E94CF39F80180819981981791F0C8
:106330000E946CC60097A9F07A9419F40BC083E010
:10634000782EEE24FF24DDCF76DF80EC94E0B601DA
:106350000E94CF390F5F1F4F802F8619851508F4D3
:10636000ACCF2196EFE00C94DBE9CF93DF93C0E054
:10637000D0E004C060DF81E090E044DF2196C433C8
:10638000D105C1F780EC94E061E472E00E94193A13
:10639000DF91CF9108951F93182F80E061E04BECBF
:1063A00052E020E00E945947143041F1153038F492
:1063B0001230D1F01330E8F4113061F510C016300E
:1063C00049F0163000F1173029F58EE061E044EC19
:1063D00052E01DC08EE061E04DEB52E018C08EE04F
:1063E00061E046EB52E013C08EE061E04FEA52E01C
:1063F0000EC08EE061E048EA52E009C08EE061E044
:1064000041EA52E004C08EE061E04AE952E020E057
:106410000E9459471F910895FC0140E021912D32BF
:1064200051F422812D3239F44450262F372FD901CF
:1064300020E030E005C04F5F483281F740E0F5CF03
:10644000FC01E20FF31FE40FF11D50815D3209F4EE
:106450004F5FFC01E20FF31FE40FF11D50815D93CC
:106460002F5F3F4F2E30310559F70895262F372FD4
:10647000D90120E030E040E0FC01E20FF31FE40F1F
:10648000F11D50815D3209F44F5FFC01E20FF31FF3
:10649000E40FF11D50815D932F5F3F4F2E3031058A
:1064A00059F70895CF93DF93E82FF92FDB0180E0B0
:1064B000EF019081903219F49181903231F0319650
:1064C00098819D938F5F823199F78091BC04680F0A
:1064D000711DFB011082DF91CF910895A0E0B1E022
:1064E000E4E7F2E30C94C6E900E010E004C0A3DEA8
:1064F00081E090E087DE0F5F1F4F87E0023D1807C5
:1065000009F44FC080EC94E060E671E092D78823F4
:1065100071F347C080EC94E0B80141D70F5F1F4F83
:1065200080EC94E06DE571E081D7882399F3F80160
:10653000108289818823C9F1CE01019660E071E063
:1065400095DF40E0E42E41E0F42E3BE4C32E3FE033
:10655000D32E90E08701892F66E0F70141917F01FA
:1065600020E0C050DF4F9883C050D1400E9499472F
:10657000F8018081F60181936F01C050DF4F98814F
:10658000C050D1409F5F9D3029F780EC94E06AE5D0
:1065900071E04FD7882381F080EC94E040D781E010
:1065A0000CC07E010894E11CF11C80EC94E0E3D661
:1065B000882311F48701B4CF80E0C050DF4FE8E0BA
:1065C0000C94E2E9A4E1B0E0E8EEF2E30C94C4E953
:1065D000A82E7B01E82FF0E0EA31F10508F0C1C1F7
:1065E000EA5BFF4F8E010F5F1F4F0C94F3E9C80168
:1065F0006FE072E00E948FEC8091360F8D83809166
:10660000370F8E838091380F8F838091390F888761
:10661000198684C0C8016AE072E067C0C80165E0FD
:1066200072E07AC0C80160E072E076C0C8016BEF2A
:1066300071E072C0C80166EF71E06EC0C80161EF21
:1066400071E06AC0C8016CEE71E066C0C80167EE17
:1066500071E062C0C80162EE71E05EC0C8016DED1C
:1066600071E05AC0C80168ED71E056C0C80163ED21
:1066700071E052C0C80160ED71E04EC0C8016CEC21
:1066800071E04AC0C80168EC71E046C0C80163EC23
:1066900071E042C0C8016EEB71E00E948FECF8011E
:1066A00001900020E9F731978E2D9F2DDC018CE0C1
:1066B0000D9001928150E1F7198A30C0C80169EB51
:1066C00071E02AC0C80164EB71E003C0C8016FEA41
:1066D00071E00E948FEC0CEA1DE022C0C8016AEA5A
:1066E00071E003C0C80165EA71E00E948FEC08EB1D
:1066F0001BE016C0C80160EA71E00E948FECC8017F
:106700006BE37FE00E94E8EC09C0C8016BE971E02F
:1067100003C0C80166E971E00E948FEC04E610E056
:106720007E010894E11CF11CC70164E971E00E943C
:1067300084EC81DD80EC94E072D6F70101900020BA
:10674000E9F7BF01615070406E197F09C7019EDDF6
:106750008091BB04882319F0EE24FF24F9C0B8010E
:1067600080E090E00E9456E75B016C0120E030E49D
:106770004CE955E40E9445E8F62E172FE82E092F24
:1067800020E030E040E85FE30E94B6E687FD29C0E4
:106790006F2D712F8E2D902F20E03FEF4FE757E4A4
:1067A0000E9441E81816B4F4C601B50120E030E0BB
:1067B00040E251E40E9445E80E942AE724EF31E0DC
:1067C00005C0C9010197F1F761507040611571056D
:1067D000C1F70CC06F2D712F8E2D902F0E942AE7CC
:1067E00002C061E070E0CB010197F1F70E94B5C6ED
:1067F00080EC94E014D69FC01EDDFA2DF53009F030
:106800004BC0B80180E090E00E9456E75B016C014C
:1068100020E030E44CE955E40E9445E87B018C011E
:106820007F2D912F20E030E040E85FE30E94B6E644
:1068300087FD29C06E2D7F2D802F912F20E03FEF07
:106840004FE757E40E9441E81816B4F4C601B501B9
:1068500020E030E040E251E40E9445E80E942AE74F
:1068600024EF31E005C0C9010197F1F76150704094
:1068700061157105C1F70CC06E2D7F2D802F912FF2
:106880000E942AE702C061E070E0CB010197F1F7B6
:1068900025DE282F30E067C080EC94E06FE871E0DF
:1068A000C8D5882309F44AC0B80180E090E00E946E
:1068B00056E75B016C0120E030E44CE955E40E94AE
:1068C00045E87B018C017F2D912F20E030E040E8EE
:1068D0005FE30E94B6E687FD29C06E2D7F2D802FD5
:1068E000912F20E03FEF4FE757E40E9441E8181650
:1068F000B4F4C601B50120E030E040E251E40E946A
:1069000045E80E942AE724EF31E005C0C90101975C
:10691000F1F76150704061157105C1F70CC06E2D23
:106920007F2D802F912F0E942AE702C061E070E046
:10693000CB010197F1F721E030E015C080EC94E045
:1069400067E871E076D5882361F481E090E05ADC55
:106950000894E11CF11C82EDE81687E0F80609F0C6
:106960004BCF20E030E0C9016496EAE00C94E0E906
:106970000F931F93CF93DF938C01C0E0D0E03CC016
:106980005ADC80EC94E066E372E053D5882349F04A
:10699000ECDC82E08093120180E060E070E012DEC7
:1069A0002FC080EC94E06EE272E043D5882359F06A
:1069B00088EE93E024EF31E0F9013197F1F7019788
:1069C000D9F781E00EC080EC94E064E172E031D54B
:1069D0002196882349F0C9DC80E060E070E0F2DDB8
:1069E00082E0809312010EC081E090E00115110554
:1069F00011F480E090E006DC0C171D0708F0C0CF12
:106A000080911201DF91CF911F910F910895A1E024
:106A1000B0E0EDE0F5E30C94C6E980E090E0A8DF9B
:106A2000823059F1F4E0DF2EEBE2CE2E8E010F5FC3
:106A30001F4F74EFE72E71E0F72EC982C80161E0A5
:106A400025DC80E197E2F7013197F1F70197D9F75B
:106A5000DA9499F782E08093120160E070E0B2DD91
:106A6000009789F083E060E070E0ACDD009759F0BA
:106A700080E197E27DDF823031F480EC94E0CFD486
:106A800021E030E002C020E030E0C9012196E8E0DA
:106A90000C94E2E9CF93DF93EC0180EC94E068EC96
:106AA00074E040E052E059D4C6DB80EC94E0B7D407
:106AB00080E090E05DDF8130F1F080E060E070E048
:106AC00081DD80E060E070E07DDD84E0BE017ADDA4
:106AD000009789F080E060E070E074DD81E060E0C4
:106AE00070E070DD009739F080E29EE441DF21E044
:106AF00030E0813011F020E030E0C901DF91CF912A
:106B000008951F93182F82E080931201812F0E9415
:106B10002BC6812F40DC0E94B5C680EC94E07FD468
:106B20001092BB0480E062E048E952E020E00E945D
:106B3000594780E060E070E045DD80E062E045E9D3
:106B400052E020E00E94594785E160E070E03ADDC4
:106B500080E062E041E952E020E00E94594786E18E
:106B600060E070E02FDD81E08093BB0480E062E0B4
:106B70004CE852E020E00E94594780E060E070E07D
:106B800021DD009749F080E062E046E852E020E035
:106B90000E94594781E008C080E062E049E752E086
:106BA00020E00E94594780E01F91089592E0909361
:106BB00012011092BB04882319F186E160E070E0B5
:106BC00001DD85E160E070E0FDDC80E060E070E028
:106BD000F9DC80E060E070E0F5DC009701F580E032
:106BE00066E045EE52E020E00E94594780E395E7D9
:106BF00024EF31E0F9013197F1F70197D9F70895C2
:106C000080E066E048ED52E020E00E94594784E1D0
:106C100060E070E0D7DC83E160E070E0D3CC089501
:106C20000F931F93182F809113011817A1F11123AF
:106C300099F482E08093120181E0B8DF89E060E09E
:106C400070E0C0DC009701F11092130187E060E072
:106C500070E0B8DCE3D518C01130B1F402E0009365
:106C6000120181E0A3DF88E060E070E0ABDC009718
:106C700059F0109313018AE060E070E0A3DCCAD5FC
:106C800080E094DF0093120181E0909113011917C5
:106C900019F080E001C081E01F910F910895AFEFDE
:106CA000B0E0E5E5F6E30C94C2E980E0B9DF8823C3
:106CB00009F497C080E060E070E084DC86E060E08A
:106CC00070E080DC009709F48CC0CC24DD2420E443
:106CD000A22E2CE9B22E98E8892E93E1992EABDAF8
:106CE0000894C11CD11CC4010197F1F780EC94E019
:106CF0003ED3AC0180E065E025E030E000E0EE242A
:106D00000E943C4D88EEC81683E0D80671F480914D
:106D1000BC04982F9F5F9093BC0461E045E851E06C
:106D200020E00E945947CC24DD2480EC94E02CD351
:106D3000882369F40894A108B108A114B10479F674
:106D400080EC94E062E771E074D3882341F2EE2492
:106D5000FF246E010894C11CD11C84E0A82EB12C24
:106D6000AC0EBD1E37C080EC94E0B80118D30F5FA5
:106D70001F4F80EC94E06FE671E058D3882399F3BD
:106D8000F80110828981882329F1C60163E671E048
:106D90000E94AEEC009731F080EC94E040D321E00B
:106DA00030E021C08701000F111FC701A5E0880F47
:106DB000991FAA95E1F7080F191FB8016050734F8A
:106DC000C50170DBB8016C5E724FC50125DB08940C
:106DD000E11CF11C80EC94E0CED2882311F48601F2
:106DE000C8CF20E030E0C901C150DF4FECE00C9487
:106DF000DEE91F93CF93DF93182F1092BC040E94FB
:106E00005B4380E060E04DE253E020E00E945947A0
:106E100082E0809312010E94B5C680EC94E0FFD21C
:106E200081E0C4DE80E060E070E0CCDB009789F4B4
:106E300080E061E047E153E020E00E94594788E0AC
:106E400092E524EF31E0F9013197F1F70197D9F795
:106E500078C01430A1F1153040F4123011F1133024
:106E600038F5113009F04CC015C0163061F01630FD
:106E700068F1173009F044C08CE060E070E0A2DBFC
:106E8000EC0187E029C08DE060E070E09BDBEC0165
:106E900086E022C08EE060E070E094DBEC0181E0EF
:106EA0001BC08FE060E070E08DDBEC0182E014C07D
:106EB00080E160E070E086DBEC0183E00DC081E101
:106EC00060E070E07FDBEC0184E006C082E160E01E
:106ED00070E078DBEC0185E00E942BC60E94B5C60D
:106EE00080EC94E09CD280E060E070E06BDB80E0BE
:106EF00060E070E067DB009729F011E0209719F05F
:106F000010E001C011E080E051DE112351F480E077
:106F100062E047E053E020E00E94594721E030E082
:106F200012C080E062E044EF52E020E00E94594746
:106F300088E092E524EF31E0F9013197F1F701970C
:106F4000D9F720E030E0C901DF91CF911F9108957A
:106F50001F93CF93DF930E945B4380E060E045E6A0
:106F600052E020E00E94594735D982E00E940D424C
:106F70001092BB0480EC94E068EC74E040E052E0D6
:106F8000ECD18091081EBDDD8823E9F482E0B9DDF3
:106F90008823C9F481E0B5DD8823A9F483E0B1DD5D
:106FA000882389F484E0ADDD882369F485E0A9DDD8
:106FB000882349F486E0A5DD882329F487E0A1DD54
:106FC000882309F46EC082E08093120183E060E0C0
:106FD00070E0F8DAEC018AE060E070E0F3DA009744
:106FE00029F011E0209719F010E001C011E08BE0CA
:106FF00060E070E0E7DA009709F411E088E160E012
:1070000070E0E0DA009709F411E089E160E070E0F7
:10701000D9DA009709F411E085E060E070E0D2DA97
:10702000009739F0112329F48091960FE2DE009742
:1070300009F411E08091960F0E942BC61123F1F400
:1070400080E0B4DD81E08093130180E064E044E4FB
:1070500052E020E00E94594788E893E124EF31E0B4
:10706000F9013197F1F70197D9F7D0D3D3D3D8D815
:1070700081E00E940D4221E030E00EC081E00E94DC
:107080000D4280E29EE424EF31E0F9013197F1F7FF
:107090000197D9F720E030E0C901DF91CF911F912E
:1070A000089580E064E043E552E020E00E94594703
:1070B00081E08093ED061092320F0E940D42809184
:1070C000960F0E942BC6E6CF1F9380EC94E068ECED
:1070D00074E040E052E041D188EE93E024EF31E0EB
:1070E000F9013197F1F70197D9F7A5D880EC94E031
:1070F00096D18091350F813059F412E0109312012E
:1071000055DD80E08DDD882331F01093120103C03E
:1071100082E0809312011F910895A0E6B0E0E3E9B8
:10712000F8E30C94CCE99E01235F3F4F80E090E0B0
:10713000AE014F5F5F4F0BC01192E217F307E1F70B
:1071400001969F01245F3F4F8830910561F0FC015B
:10715000EE0FFF1FE80FF91FEE0FFF1FEE0FFF1FCF
:10716000E40FF51FE9CFCE01019699DD009779F183
:10717000E4E1FDE080E09081992309F59181992374
:10718000F1F492819923D9F493819923C1F49481E4
:107190009923A9F49581992391F49681992379F4FF
:1071A0009781992361F49085992349F491859923D6
:1071B00031F49285992319F49385992331F08F5FE7
:1071C000B2969EE0E432F907B1F68093BD04C05A4E
:1071D000DF4FE2E00C94E8E9A1E0B0E0E2EFF8E391
:1071E0000C94C3E96E010894C11CD11C992493949A
:1071F000FAE6AF2EFCE0BF2E54C08091BA04813075
:1072000009F45FC018D880EC94E0B5D0882329F049
:107210000894E108F1080109110980EC94E0ABD071
:10722000882309F046C080EC94E0B601B8D0809184
:10723000BA048823B1F58981843261F48091110107
:10724000813041F410921101B0921001A0920F010F
:107250001092200F809111018823A1F4E0910F0179
:10726000F0911001898180838091200F8F5F80933E
:10727000200F89818A3031F481E08093110180935D
:10728000BA0420C080910F01909110010196909353
:10729000100180930F018091200F863911F4909294
:1072A0001101E0E8EE2EEAE1FE2EE6E00E2F112DB0
:1072B000A4CFE114F1040105110509F09ECF80E08F
:1072C00001C081E02196EBE00C94DFE9A0E0B0E0A2
:1072D000ECE6F9E30C94C6E9EC016B018A0120E0CD
:1072E00030E019C0C901800F911F8E159F0578F5F8
:1072F0008A819B81800F911F820F931F6C817D81FA
:107300000E9458E9AE81BF81A80FB91F8C918E17DA
:10731000F1F42F5F3F4FF601E20FF31FE491E88095
:10732000F980EE23F9F68A819B81800F911F820FED
:10733000931F6C817D810E9458E99B838A83E01AA8
:10734000F10AE21AF30AF982E88281E001C080E0E2
:10735000CDB7DEB7E8E00C94E2E9FC015583448345
:107360007783668313821282118210820895FC0152
:10737000808191810895FC0181E020813181211576
:10738000310509F080E00895FC0181E044815581D8
:10739000208131814217530709F080E00895FC01F4
:1073A000808191810097C9F0A681B7818281938104
:1073B000A80FB91F8C91DB018C9382819381019678
:1073C000648175810E9458E99383828380819181D1
:1073D00001979183808381E0089580E008951F9351
:1073E000FC01162F248135814081518124173507F6
:1073F00099F082819381840F951FB9010E9458E909
:10740000A681B781A80FB91F1C9380819181019635
:107410009183808381E001C080E01F910895FC0189
:10742000118210821382128281E0089540E050E0C0
:107430004DCFEF92FF920F931F93CF93DF938C0169
:107440007B01C0E0D0E007C0C801B701AE013EDF5C
:10745000882349F42196F80180819181C817D907C2
:1074600098F380E001C081E0CDB7DEB7E6E00C9490
:10747000E4E9429A289A469A459A823051F083303C
:1074800018F48823F9F008958530C1F0863071F53D
:1074900017C08091C9008F7E8093C9008091C90078
:1074A000877F8093C9008091C9008F778093C9003E
:1074B000529853985A985B98429808954598089521
:1074C000469808958091C9008F7E8093C90080916D
:1074D000C900877F8093C9008091C9008F7780930E
:1074E000C900529853985A985B98289808958150EB
:1074F000873068F4E82FF0E0EE0FFF1FEE0FFF1F5C
:10750000EF5DFE4F208131814281538103C020E035
:1075100030E0A901B901CA010895EF92FF920F93DB
:107520001F93CF93DF937C01EB01142F0E945B43E9
:1075300080E060E04FE727E001E00E94724581E0D3
:1075400060E0A70122E00E9459470E947B5082E040
:10755000B70140E020E00DEF0E9437478EEF90E04A
:107560000E940B53BC0183E040E020E001E00E9458
:107570003747112321F48881882371F41DC0CE017F
:107580000E9496EC0097C1F085E0BE0140E020E04B
:1075900001E00E94374707C085E0BE0140E020E0DF
:1075A00001E00E94BF4680E065E24FE72EE001E087
:1075B00092E0E92E0E9492488EE090E00E940B53E8
:1075C000AC018CE067E020E00E945947CDB7DEB700
:1075D000E6E00C94E4E902C00E947B5080E20E9445
:1075E00076B08823C9F384E190E00E940EC68091B2
:1075F000960F0E942BC680912F0F813011F486E0E8
:1076000001C085E036DF81E008C785E594E064E1EC
:1076100071E040E082DF82E000D780E197E224EF72
:1076200031E0F9013197F1F70197D9F78091350FE2
:10763000882311F481E0F4DA82E01BDFCCCF8CE107
:1076400091E066E47FE00E94FCEC89E494E065E16F
:1076500071E040E062DF82E0E0D688E99AE324EF5F
:1076600031E0F9013197F1F70197D9F78091350FA2
:10767000882311F481E0D4DA80E0FBDEACCF8BE329
:1076800094E06AE274E041E048DF83E0C6D680E03F
:10769000F0DEA1CF8DE194E064E171E040E03DDFF8
:1076A00083E0BBD680E0E5DE96CF0E945B4380E0BE
:1076B00060E047E054E022E00E94594780E061E04A
:1076C00041EF53E022E00E94594780E063E04BED38
:1076D00053E020E00E94594780E064E045EC53E02D
:1076E00020E00E94594780E065E04FEA53E020E047
:1076F0000E94594780E066E049E953E020E00E949B
:10770000594783E290E00E940B53AC018CE067E0A4
:1077100020E00E94594782E080D682E0AADE80E223
:107720000E9476B08823D9F380912F0F813011F415
:1077300086E001C085E09DDE81E06FC688E893E0C9
:1077400061E873E041E0E9DE82E093DE44CF83E765
:1077500093E064E171E040E0E0DE80E08ADE3BCF70
:10776000AAD783E490E00E940B53AC0180E060E074
:1077700022E00E94594781E490E00E940B53AC0143
:1077800080E061E022E00E94594780E490E00E949E
:107790000B53AC0180E063E020E00E94594780E099
:1077A00064E04DE553E020E00E94594780E065E049
:1077B00047E453E020E00E94594784E490E00E94AF
:1077C0000B53AC0180E066E020E00E94594783E261
:1077D00090E00E940B53AC018CE067E020E00E9437
:1077E000594780E046DE5E9880E20E9476B08823AA
:1077F000D9F35E9A80912F0F813011F486E001C099
:1078000085E037CE81E08093330F089581E0809347
:10781000340F089581E08093350F08951092350F4D
:10782000089560937E0F70937F0F8093800F9093E5
:10783000810F2093820F3093830F4093840F5093D6
:10784000850F089587E00E94864480E067E040E16C
:1078500055E020E00E94594781E29FE060E070E03F
:1078600049E857E00E94E7ED87E00C94AA440F93A3
:107870001F93CF93DF931FD780E060E04AEF54E07F
:1078800022E00E94594780E061E04FEE54E020E0A2
:107890000E94594780E062E049ED54E020E00E94F8
:1078A000594789E88093220F1092230F85E0809337
:1078B000240F21E02093250F82E48093260F20934C
:1078C000270F80E18093280F80E48093290F209375
:1078D0002A0F10922B0F84E180932C0F84E6809363
:1078E0002D0F10922E0F10922F0F1092300F10921A
:1078F000310F1092320F1092330F1092340F2093E9
:10790000350F1092860F1092870F20938B0F1092D5
:107910008C0F20938D0F10928E0F88E280938F0F23
:107920002093900F2093910F80E197E29093930F13
:107930008093920F1092940F1092950F84E0809391
:10794000960F20938A0F84E391E29093890F80939E
:10795000880F84EF91E09093980F8093970F8EE1BA
:1079600090E090939A0F8093990F85E090E0909328
:107970009C0F80939B0F10929D0F20939E0F10924F
:107980009F0F10927E0F10927F0F1092800F109217
:10799000810F1092820F1092830F1092840F109219
:1079A000850F86E39FE064ED74E00E948FEC8BE32B
:1079B0009FE060ED74E00E948FEC8BE49FE061EC4F
:1079C00074E00E948FEC86E49FE06CEB74E00E9410
:1079D0008FECEAE5FFE011928FE0EE36F807D9F779
:1079E00080E381939FE0EC37F907D9F710927C0F81
:1079F00010927D0F89E88093210F1092AE0F1092A4
:107A0000A00F8DE290E09093A20F8093A10F90932E
:107A1000A40F8093A30F2FE730E03093A60F20939D
:107A2000A50F1092A70F9093A90F8093A80F909382
:107A3000AB0F8093AA0F3093AD0F2093AC0F84E16E
:107A40008093B10F1092B20F81E08093B30F8AE060
:107A50008093B40F1092B50F1092B60F88E2809306
:107A6000B70F1092B80FAF01435C5F4F23EC3FE0BC
:107A70000DEC1FE0C2EDDFE0A7EDBFE080E090E09D
:107A8000BC01625E7F4FFA0161937193AF01BC014B
:107A9000625F7E4FF901619371939F01F80111922A
:107AA0008F0119921D9201968530910549F711E0D9
:107AB0001093DC0F1093DD0F1093DE0F80EE9FE02C
:107AC00068EB74E00E948FEC8BEE9FE06FEA74E04D
:107AD0000E948FEC1092F60F1092DF0F8FEF9FEF46
:107AE000DC018093F70F9093F80FA093F90FB093F8
:107AF000FA0F1092FB0F1092FC0F1093FD0F1093D2
:107B0000FE0F8FEF9FE06FE974E00E948FEC8FE033
:107B100090E16FE874E00E948FEC8FE190E16FE7F5
:107B200074E00E948FEC10922F101092301081E3BD
:107B300090E16FEF70E04AE050E00E94E1EC8BE3EF
:107B400090E16EE774E00E948FEC86E490E16DE7CF
:107B500074E00E948FEC0E94A2D90E946F6D0E9477
:107B6000DE840E94816D6EDE80E066E048E654E0CF
:107B700020E00E94594782E167E045E654E020E0BA
:107B80000E945947789488EC90E060E870E040E00B
:107B90000E94B7B080E10E9476B08823D9F329987B
:107BA000DF91CF911F910F9108950F9381E29FE094
:107BB00060E070E049E857E00E94D7ED0E94EA30AB
:107BC0008091240F823019F481E08093240F8091FA
:107BD000210F893809F4A7C08757833110F047DE99
:107BE000A2C00E94A2D90E946F6D0E94DE840E94F2
:107BF000816D8091210F813830F481E08093DD0F19
:107C00008093DE0F02C0813821F481E080932A0F37
:107C100002C0823881F41092DF0F1092F60F80EECE
:107C20009FE060E975E00E948FEC8BEE9FE067E8D3
:107C300075E00E948FEC8091210F843860F48FEF03
:107C40009FEFDC018093F70F9093F80FA093F90F4B
:107C5000B093FA0F02C08438D9F41092FB0F10923F
:107C6000FC0F81E08093FD0F8093FE0F8FEF9FE06C
:107C700067E775E00E948FEC8FE090E167E675E0C2
:107C80000E948FEC8FE190E167E575E00E948FEC38
:107C90008091210F873818F410922F1002C0873876
:107CA00059F41092301081E390E16FEF70E04AE0F8
:107CB00050E00E94E1EC02C0883861F48BE390E16F
:107CC00066E575E00E948FEC86E490E165E575E07D
:107CD0000E948FEC89E88093210F7894ECD482E0A5
:107CE00063E475E040E020E000E00E94374783E075
:107CF00067E375E040E020E00E94374785E067E2F7
:107D000075E040E020E00E94374782E167E044E20E
:107D100055E020E00E94594780E10E9476B0882318
:107D2000D9F390DDF8940F910895FC016081609380
:107D3000A61771817093A71782818093A8179381EA
:107D40009093A91708952F923F924F925F926F924E
:107D50007F928F929F92AF92BF92CF92DF92EF92DB
:107D60000F931F93DF93CF930F92CDB7DEB780E8C9
:107D70000E9476B0882329F48091CD06823009F0E4
:107D800040C08091CD068130C9F195D480E060E09B
:107D900045E156E020E00E94594780E061E049E07B
:107DA00056E020E00E94594780E062E04DEF55E048
:107DB00020E00E94594780E063E041EF55E020E079
:107DC0000E94594780E064E045EE55E020E00E94C3
:107DD000594780E065E049ED55E020E00E945947B1
:107DE00080E066E04DEC55E020E00E94594780E0DD
:107DF00067E041EC55E020E00E94594781E0809324
:107E0000CD068091CA06813009F067C08091CB060B
:107E1000803309F062C08091CD06882309F05DC0EF
:107E2000A090AE1683EB96E110E03C0153C01031F8
:107E300009F453C0183010F09BE001C090E0F3014A
:107E40004081892F612F50E023E030E000E0EE24F4
:107E500099830E943C4DF30143819981892F8C5F66
:107E6000612F50E022E030E00E943C4DF30121817F
:107E700030E0A9014370507099814330510531F4CD
:107E8000892F895F612F4FEB55E01DC020FF06C091
:107E9000892F895F612F4DEB55E015C0F3012281D9
:107EA000253030F0892F895F612F4BEB55E00BC0F7
:107EB000892F895F223020F0612F49EB55E003C004
:107EC000612F47EB55E020E0F4D71F5F8CE090E096
:107ED000680E791E1A1508F4AACF8091CD0681305C
:107EE00009F068C18091CA06813009F07DC0809197
:107EF000CB06863009F078C08091B416823049F004
:107F0000823060F0853050F48BE060E044EB55E067
:107F100009C08BE060E041EB55E004C08BE060E01D
:107F20004EEA55E020E0C5D78091B51683708330C6
:107F300029F481E160E04CEA55E004C081E160E0B1
:107F40004AEA55E020E0B5D78091B51680FF05C01C
:107F50008EE060E047EA55E004C08EE060E044EA6D
:107F600055E020E0A6D74091D9168BE061E050E0C3
:107F700022E030E000E0EE240E943C4D82EC96E1ED
:107F8000D4DE9B01AC018BE062E0A90125E030E08A
:107F90000E943C4D81E162E041EA55E020E089D752
:107FA0009091D7168FEF989FC00111242091D6167B
:107FB000820F911D64E670E00E9458E9AB015C01FC
:107FC0008BE063E022E030E00E943C4D8DE063E016
:107FD0004FE955E020E06DD78EE063E0A50122E097
:107FE00030E001E00E943C4D8091CA06813011F5DD
:107FF0008091CB068231F1F48EEB96E196DE20E1A2
:108000003EE040E050E00E942DE920EA36E841E001
:1080100050E00E947FE98BE064E0A90123E030E0BA
:1080200000E0EE240E943C4D8FE064E04AE955E018
:1080300020E03FD78091CA06813009F0BBC0809113
:10804000CB06823009F0B6C08EEA96E16EDE5B01A7
:108050006C0190E8692E96E9792E98E9892E912C89
:10806000C601B501A40193010E947FE98AE065E0A1
:10807000A90122E030E000E0EE240E943C4D8CE0BB
:1080800065E048E955E020E014D7C601B50128EEC7
:1080900033E040E050E00E947FE9CA01B90120E1ED
:1080A00037E240E050E00E947FE99B01AC018DE0A7
:1080B00065E0A90124E030E001E00E943C4DC601EA
:1080C000B5012AE030E040E050E00E947FE984E61C
:1080D000282E312C412C512CCA01B901A201910149
:1080E0000E947FE99B01AC0181E165E0A90122E0EA
:1080F00030E00E943C4D82EB96E117DE5B016C01A3
:10810000A40193010E947FE98AE066E0A90122E0D0
:1081100030E000E00E943C4D8CE066E046E955E02E
:1081200020E0C7D6C601B50128EE33E040E050E0BC
:108130000E947FE9CA01B90120E137E240E050E046
:108140000E947FE99B01AC018DE066E0A90124E07B
:1081500030E001E00E943C4DC601B5012AE030E06C
:1081600040E050E00E947FE9CA01B901A2019101FB
:108170000E947FE99B01AC0181E166E0A90122E058
:1081800030E00E943C4D8AEB96E1CFDD28EE33E0F3
:1081900040E050E00E947FE98BE067E0A90124E025
:1081A00030E000E00E943C4D80E167E044E955E0AA
:1081B00020E07FD60F90CF91DF911F910F91EF902C
:1081C000DF90CF90BF90AF909F908F907F906F90F7
:1081D0005F904F903F902F9008959091C806980F10
:1081E0009093C8068091C906890F8093C9060895A7
:1081F000A2E0B0E0EEEFF0E40C94C6E95CD282E0DD
:108200008093CD068091DF06823099F480E063E0B0
:1082100041E256E020E04DD684E690E09093331E94
:108220008093321E8091321E9091331E0097D1F7B9
:10823000A0C08091E006813011F00E94E5C90E9443
:1082400048CA88EC90E09093331E8093321E1982C6
:10825000CC24DD2420E07E010894E11CF11C08EC14
:1082600010E0C7012A830E9408C82A81882309F4E4
:108270006DC01093331E0093321EE22FF0E0E93000
:10828000F10508F063C0E05AFF4F0C94F3E98981CF
:10829000853B09F05BC01092CC061092CB06109281
:1082A000CA061092C8061092C90621E04FC0898103
:1082B000823609F04AC047C08981813009F045C043
:1082C0008CDF89818093CA0623E040C08981803396
:1082D00031F0863021F0823111F08230B1F5809397
:1082E000CB067BDF24E032C089818B3F70F575DFE0
:1082F000D98025E02BC08981882339F56EDF26E0FF
:1083000025C0DA948981E091CC06F0E0E655F94E7B
:1083100080832A8362DF8091CC068F5F8093CC06B6
:108320002A81DD2099F427E011C0C98028E00EC021
:108330008091C806C81649F499818091C90698179A
:1083400021F401DD02C022E001C020E080E22A83A6
:108350000E9476B02A81882339F48091321E909150
:10836000331E009709F07DCF80EF0E9476B00E9407
:10837000E5C92296E8E00C94E2E911B814B817B800
:108380001AB880B18093BF1783B18093C11786B1AB
:108390008093BE1789B18093AB1717B84798379B66
:1083A00002C081E001C082E08093C0174098309BFA
:1083B00003C01092BD1703C081E08093BD17409A9F
:1083C00008958091C017813009F447988091C017B3
:1083D000823009F45F9808958091C017813009F4C4
:1083E000479A8091C017823009F45F9A089580916E
:1083F000C017813009F45F9A8091C017823009F468
:10840000479A08958091C017813009F45F98809150
:10841000C017823009F4479808959091BD179923A9
:1084200019F098B1947F98B9823051F0833001F1FE
:10843000813009F58091BD17439A1092CE060895B8
:108440008091BD17882311F0409A01C04398809114
:10845000CE06882381F481E08093CE0680E395E701
:1084600024EF31E0F9013197F1F70197D9F7089539
:10847000419A1092CE0608958091CE06882399F4F1
:108480008091BD17882311F082E0C7CF439881E027
:108490008093CE0680E395E724EF31E0F901319730
:1084A000F1F70197D9F708958091BD17882311F04E
:1084B00081E0B3CF439A1092CE060895EF920F93C6
:1084C0001F935BDF8091BD17882331F087B18360F4
:1084D00087B988B1847F88B982B1806F82B90C98DE
:1084E0008091DC0F813009F409988FEF84B988B14D
:1084F000806988B987B18C6E87B93C988091BD1727
:1085000043985E9A8AB1806F8AB9299A0E945AAEBE
:1085100011E01093311E84E190E00E9437C884E19D
:1085200090E00E940EC681E00E94506B80E084D1F2
:108530003CDB84E10E9479B278948091960F80931D
:10854000081E0E942BC68091960F0E9468C88091D9
:10855000240F833088F01093240F81E090E060E0D6
:1085600070E043E050E029E50CE0EE24E3940E9443
:1085700096998093240F66D981E05ED180E991E0DD
:1085800060E870E040E00E94B7B01092E7060E94F9
:108590008D4F0E9429908091BD17882349F082E079
:1085A00062E576E040E020E007E061D415E001C03C
:1085B0001BE08091C017813031F460E476E040E048
:1085C00020E0012F54D48091C017823039F481E02B
:1085D0006EE276E040E020E0012F49D487E090E0B1
:1085E0000E940B53BC0185E040E020E002E03FD454
:1085F00088E090E00E940B53BC0186E040E020E060
:1086000004E035D480E066E24FE728E101E092E043
:10861000E92E88D588E293E224EF31E0F901319721
:10862000F1F70197D9F70799299888EE93E024EF9D
:1086300031E0F9013197F1F70197D9F780E991E03D
:1086400060E870E040E00E94B7B080EF0E9476B032
:108650002BDF8091310F813049F48091330F8823D3
:1086600029F429D08091960F0E94FFDB8091320F70
:10867000813039F48091340F882319F41CD00E9482
:10868000A8370E9410318091310F813031F48091F0
:108690002F0F882311F485E001C086E00E94393A4B
:1086A0001F910F91EF9008952C988EBD0DB407FE89
:1086B000FDCF2C9A08951F93CF93DF9323EC37E1DE
:1086C000C90160E070E040E054E00E94E1EC10EB92
:1086D0002B98812FE9DF80E1E7DF8091CF06E4DF8F
:1086E0002B9AC0E8D0E080E0DFDF2197E1F71F5F41
:1086F000183B71F71092751C1092761CDF91CF9188
:108700001F910895A1E0B0E0E8E8F3E40C94CAE911
:108710008C012B989C01220F232F221F330B3195A4
:10872000822F80556983C0DF8091CF06102F1F777D
:10873000180F812F82958F70805FB6DF812F8F7029
:10874000B3DF2B9A6981862FAFDF2196E4E00C948A
:10875000E6E9CF93DF93C0E0D0E0FE01ED5BF74E9A
:108760008081FE01ED53F84E80836081CE01CADF27
:10877000219683E0C038D80781F7FE01ED53F84E0B
:108780001082CE0160E0BEDF219684E0C030D807C1
:10879000A1F7DF91CF910895282F87FD35C0603470
:1087A00098F5862F86958695869590E09695982FD4
:1087B000882797958795820F911D677021E030E09B
:1087C00001C0220F6A95EAF79370413061F04130A1
:1087D00018F04230A1F40DC0FC01ED53F84E308189
:1087E000209532230BC0FC01ED53F84E3081322B23
:1087F00005C0FC01ED53F84E308132273083FC0177
:10880000ED53F84E60817ECF089588E893E101979B
:10881000F1F708950F931F93CF93DF938C01C0E07E
:10882000D0E002C0F2DF2196C017D107D8F3DF9164
:10883000CF911F910F9108951F93182F1092751CBF
:108840001092761C8CE58CBD81E08DBD2C9A2A9807
:108850008AE090E0DFDF2A9A2C982B9880E424DFCE
:10886000113089F48091CF06882321F481EA1CDF3E
:1088700080EC03C080EA18DF88EC16DF80912B0FB4
:10888000882339F404C081EA0FDF80EC0DDF86EA2B
:1088900001C087EA09DF82EA07DF8FE205DF88EFA0
:1088A00003DF80E001DF87E2FFDE113029F481E899
:1088B000FBDE80912C0F03C081E8F6DE86E1F4DE5A
:1088C0008CEAF2DE80E0F0DE8FEAEEDE80919D0F32
:1088D0008823C9F41130A1F460912D0F70E088272E
:1088E00077FD8095982F0E9458E723E333E343E216
:1088F00050E40E9445E80E942AE76093B30003C059
:108900008FEF8093B300D7DE1F9108950F931F93CD
:10891000CF93DF93082F10E01695102F002717959F
:1089200007951370C0E0D0E0CE01800F911FFC01CD
:10893000ED53F84E2081DE01AC53B44E2C93608190
:10894000E1DE2196CE37D10579F7DF91CF911F91E6
:108950000F9108950F931F93CF93DF93082F10E08B
:108960001695102F0027179507951370C0E0D0E0DB
:10897000CE01800F911FFE01EC53F44E2081FC01CB
:10898000ED53F84E20836081BDDE2196CE37D105B0
:1089900079F7DF91CF911F910F9108958091761C07
:1089A0008F5F8093761C883020F0D3DE87E0809341
:1089B000761C0895A5E0B0E0E0EEF4E40C94BCE988
:1089C000602E082F10E0C62EDD24242E3324D10182
:1089D000A01BB10B422F50E05A8349837A01EC1857
:1089E000FD08B7FD08C0E1E08E2E912C109731F400
:1089F0008824992403C088248A94982CF7FC09C001
:108A000071E0472E512CE114F10431F44424552433
:108A100003C044244A94542C9D01B7FF03C03095F1
:108A200021953F4FF7FE04C0F094E194F108F394D0
:108A3000462D2C833D83B0DE2C813D81E216F3066A
:108A40003CF5C90162E070E00E946CE9AA24BB24F5
:108A5000A61AB70A982D782C700E16C0AE0CBF1C43
:108A6000080D191D1A141B0424F4C40CD51CA21AD9
:108A7000B30A872D6C2D462D2C833D839B838CDE82
:108A80009B81790E3D812C810215130539F726C093
:108A9000C70162E070E00E946CE9AA24BB24A61A18
:108AA000B70A342C742C7C0C14C0A20EB31EC40C58
:108AB000D51C1A141B0424F4080D191DAE18BF0888
:108AC000802F672D462D2C833D8366DE730C3D8100
:108AD0002C8189819A81C816D90639F72596E2E159
:108AE0000C94D8E9A0E0B0E0E8E7F5E40C94C5E91F
:108AF000182FB02E87FD1FE7603408F06FE3E42ED7
:108B0000FF24C62EDD24C20ED11CE10EF11C21E88B
:108B1000E216F10418F0A0E8EA2EF12C31E4C316B5
:108B2000D10418F0F0E4CF2ED12CC62FD0E007C02E
:108B3000812F6C2F4E2D2C2F0B2D3CDF2196CC1628
:108B4000DD06B0F7CDB7DEB7E9E00C94E1E9A1E0CE
:108B5000B0E0EDEAF5E40C94C2E9C82EB62E322F4F
:108B6000D02E4F3DE1F0403E38F4463D81F04C3D83
:108B700091F0443CA9F407C0463F59F04C3F69F0DE
:108B8000443E71F402C041E00BC042E009C043E042
:108B900007C044E005C045E003C046E001C04EE127
:108BA000142F1F77FC2CFF0CFC0CFF0CFD0C6B2D05
:108BB000660F660F660FAE2CA60EEE2009F051C0B0
:108BC000323011F0343039F48F2D45E027E001E0E8
:108BD000398388DF3981AB2CBB24B694BA2CAA2404
:108BE000B794A79446E02C2D249FC0011124A80E11
:108BF000B91E8D2D992787FD9095A80EB91E8FEF70
:108C000093E0A822B922149FA00111248A01045ADA
:108C1000194F82E6E82E86E0F82EE40EF51EF801E4
:108C20009491323011F0343039F4F501ED53F84EAF
:108C300080818927808304C0F501ED53F84E90832D
:108C4000F501ED53F84E6081C50139835BDD0F5F9F
:108C50001F4F0894A11CB11C39810E151F05F9F690
:108C60003AC006E0109F80011124BCE58B2EB6E0CF
:108C70009B2E800E911E0E59194FF401B490EA2CD0
:108C8000CC24C394DD248C2D8B2139F0323059F063
:108C900041E050E0343061F406C0323039F041E058
:108CA00050E0343029F040E050E002C041E050E0B4
:108CB0008F2D6E2D398370DD3981D394E394FD2D92
:108CC000F83011F0CC0CDFCF0894811C911CF39488
:108CD0008016910691F62196ECE00C94DEE9AF92B5
:108CE000BF92DF92EF92FF920F931F93CF93DF9388
:108CF000D62EF42E122FA82EE5015E01B92EE50125
:108D000019C04A30B1F04D3019F41092751C12C0E0
:108D10008091751C6091761C2D2D0F2DE12E17DF93
:108D20008091751C8F5F8093751C863118F01092AE
:108D3000751C34DE4991442321F7DF91CF911F91B7
:108D40000F91FF90EF90DF90BF90AF900895EF925A
:108D50000F93FA01402F8093751C6093761CCF010E
:108D6000622F2E2DBCDF0F91EF9008958093751C1C
:108D70006093761CCA01622F40E020E0B0CF0F93D1
:108D8000972FA62FB72FFD0101900020E9F731970B
:108D9000EA1BFB0B205CDF01AA0FBB1FAE0FBF1F3E
:108DA0002A1B1092751C8093761C862F642F422FED
:108DB000202F95DF0F910895A0E0B0E0E2EEF6E4F9
:108DC0000C94C8E9FE013F9664E4E62E6CE1F62EB1
:108DD00081E0B70148E22D853E858F010E9482D552
:108DE0008985B7014A852B850C85C9DF2096E6E089
:108DF0000C94E4E9A0E0B0E0E0E0F7E40C94C7E90B
:108E0000EC01D62EF42E122F1AC04A30B1F04D309C
:108E100019F41092751C12C08091751C6091761C1B
:108E20002D2D0F2DE12E93DE8091751C8F5F809389
:108E3000751C863118F01092751CB0DD2196FE016C
:108E40004491442311F7CDB7DEB7E7E00C94E3E992
:108E5000EF920F93FA01402F8093751C6093761C5C
:108E6000CF01622F2E2DC6DF0F91EF900895A2E063
:108E7000B0E0EDE3F7E40C94C8E9182F7B01C701DB
:108E80002A8349830E9496EC2A81422F405CFC0190
:108E9000EE0FFF1FE80FF91F4E1B1092751C109369
:108EA000761CC7016981202FA5DF2296E6E00C948D
:108EB000E4E98093751C6093761CCA01622F40E040
:108EC00020E098CF40E020E095CF8F929F92BF9214
:108ED000CF92DF92EF92FF920F931F93CF93DF9386
:108EE000182FF62EB22EC02EDE2C842EE4014E0159
:108EF000952EE40107C0812F6F2D2B2D0C2DED2C0D
:108F000026DE1F5F49914423B1F7DF91CF911F9176
:108F10000F91FF90EF90DF90CF90BF909F908F9038
:108F20000895EF920F9300E0EE24CFDF0F91EF90C2
:108F30000895EF920F9300E0EE2409DE0F91EF9079
:108F400008951F93CF93DF93EC01162F17C04A307B
:108F500019F04D3019F40FC021DD0FC08091751C40
:108F60006091761C212FE5DF8091751C8F5F8093C7
:108F7000751C863110F01092751C2196FE014491EB
:108F8000442329F7DF91CF911F9108958093751C99
:108F90006093761CCA01622FD4CF0F931F938093E6
:108FA000751C6093761C282F30E0240F311D26316C
:108FB00031051CF005E1081B01C0042F080F182F14
:108FC00007C0812F6091761C40E220E0B2DF1F5F76
:108FD0001017B8F31F910F9108957F928F929F926F
:108FE000AF92BF92CF92DF92EF92FF920F931F93B7
:108FF000182FF62EC42ED22EB02E74DD8E2D813079
:1090000091F1823009F044C0712E739401E0B110E7
:1090100000E0872D6F2D402FBFDBAF2CA394812F55
:109020006A2D402FB9DBEC2CE10E8E2C8A94882D12
:109030006F2D402FB1DB8E2D6A2D402FADDBAD2C77
:10904000AF0C9A2C9A94812F692D402FA5DB872D88
:109050006A2D402FA1DB882D6A2D402F9DDB8E2DA0
:10906000692D402F99DB01E0B11000E0812F6F2DB9
:10907000402F92DBC10E8C2D6F2D402F8DDBFD0C10
:10908000812F6F2D402F88DB8C2D6F2D402F84DB9F
:109090001F910F91FF90EF90DF90CF90BF90AF9016
:1090A0009F908F907F900895A0E0B0E0EAE5F8E40B
:1090B0000C94C7E9F82EE02E87FF02C0BFE7FB2E15
:1090C000162F603408F01FE3E42FF0E0C12FD0E04A
:1090D000C20FD11DEF0DF11DE138F10510F0E0E8F0
:1090E000F0E0DE2E8F2D612F4E2F212F0E2D62DC12
:1090F000C134D10510F0C0E4D0E08D2D612F4D2D8D
:109100002C2F0E2D57DC8D2D9E016C2F4F2D52DCF8
:109110008F2D6C2F4F2D212F4DDCCDB7DEB7E7E023
:109120000C94E3E97F928F929F92AF92BF92CF927D
:10913000DF92EF92FF920F931F93182FF62EB42E0B
:10914000C22ED02EB1DF8E2D813009F442C0823084
:1091500009F054C0912E939401E0D11000E0892DC4
:109160006F2D402F19DBEF2CE394812F6E2D402FB4
:1091700013DB892D6E2D4D2D0FDB8B2C810EA82C32
:10918000AA948A2D6F2D402F07DB882D6E2D402F3E
:1091900003DB8A2D6E2D4D2DFFDA7C2C7F0CE72C06
:1091A000EA94812F6E2D402FF7DA892D672D402FFD
:1091B000F3DA892D6E2D4D2DEFDA8A2D672D402F94
:1091C000EBDA882D6E2D402FE7DA8A2D6E2D4D2D8E
:1091D000E3DA01E0D11000E0812F6F2D402FDCDABF
:1091E000B10E8B2D6F2D402FD7DAFC0C812F6F2DF8
:1091F000402FD2DA8B2D6F2D402FCEDA1F910F9199
:10920000FF90EF90DF90CF90BF90AF909F908F90A6
:109210007F900895A0E0B0E0E0E1F9E40C94BCE9AF
:10922000C82ED62E7A01922EC1E0D0E0C41BD50BF9
:1092300000271127041B150B000F111F642F6D0D44
:10924000422FAADA6D2D6E198C2D492DA5DA8E2D9F
:109250008C0D6D2D492DA0DA8C2D8E196D2D492D7B
:109260009BDA83E0282E312CAA24BB2443C0D7FDEF
:1092700007C00894E108F1080E5F1F4FC00FD11F0F
:109280000894A11CB11CC20DD31D5A2C5C0C6E2C71
:109290006D0C852D662D492D7FDA4C2C4A18842DB6
:1092A000662D492D79DA6D2C6E18852D662D492D88
:1092B00073DA842D662D492D6FDA5E2C5C0C6A2CD6
:1092C0006D0C852D662D492D67DA8C2D8E19782E23
:1092D000662D492D61DA9D2D9A19892E852D692FCC
:1092E000492D5ADA872D682D492D56DA82E090E013
:1092F000280E391EAE14BF040CF4B9CFCDB7DEB7BB
:10930000E2E10C94D8E9A0E0B0E0E9E8F9E40C94DB
:10931000BCE9B82E162F6A01A22EC1E0D0E0C41B12
:10932000D50BEE24FF24E41AF50AEE0CFF1C642F83
:10933000610F212F241B4B2D0A2D3CDB4B2D4C198B
:109340008C2D8B0D612F212F35DB460123E0222E42
:10935000312C6624772437C0D7FD09C008948108D2
:10936000910882E090E0E80EF91ECE0DDF1D089412
:10937000611C711CC20DD31DC62C562C5B0C4B2CD2
:109380004618282D210F852D622F442D0A2D12DB22
:10939000212F2819852D622F442D0CDB582C5B0CB6
:1093A0009B2D9819D92E262D210F852D622F492FFF
:1093B00001DB212F2619852D622F4D2DFBDA82E04E
:1093C00090E0280E391E6814790434F2CDB7DEB768
:1093D000E2E10C94D8E9A1E0B0E0E1EFF9E40C940B
:1093E000BDE9882EF62E342ED22E9E2CB80180E0B8
:1093F00090E00E9456E72BED3FE049E450E40E94E4
:1094000045E820E030E044E353E40E94BDE6162F37
:10941000A72E082FE92E0E94BAE62B013C016D2DE4
:1094200070E080E090E00E9456E79B01AC01C30130
:10943000B2010E9445E80E94A8E82B013C01612F7F
:109440007A2D802F9E2D0E94C8E85B016C01632D50
:1094500070E080E090E00E9456E79B01AC01C601FD
:10946000B5010E9445E80E94A8E80E942AE7462F1D
:10947000480DC301B20149830E942AE72F2D261B04
:10948000882D6F2D4981092D95DA2196E1E10C9403
:10949000D9E9AEE0B0E0EFE4FAE40C94BCE9182FAF
:1094A000F62E6A015901449F9001459F300D549F4B
:1094B000300D11243A832983AA9CC001AB9C900DE6
:1094C000BA9C900D11249C838B83A29E4001A39E85
:1094D000900CB29E900C1124BC0168197909882760
:1094E00077FD8095982F0E9458E72B013C01E98178
:1094F000FA81BF01882777FD8095982F0E9458E751
:1095000020E030E040E85EE30E9445E89B01AC01CA
:10951000C301B2010E9452E60E94A8E80E9425E71A
:109520003B019401220F331F3A8729876A2D6F0D63
:10953000812F402F31D96F2D6A19812F402F2CD9BF
:109540008C2D810F6F2D402F27D9812F8C196F2DD6
:10955000402F22D989819A81909581959F4F880FBC
:10956000991F9E838D83EB81FC81EE0FFF1FF8878F
:10957000EF836F012B813C81C20ED31E44245524FE
:10958000882499247E866D8629853A853DC08D85FF
:109590009E8597FD0BC00894A108B108ED81FE815E
:1095A0002E0F3F1F821B930B9E878D870894411CB3
:1095B000511C8F819885880E991EED85FE85EC0DD6
:1095C000FD1DFE87ED87E42CE10E7A2C7F0C8E2D9D
:1095D000672D402F2B873C87DFD8FF2DFA196F2E80
:1095E0008E2D6F2F402FD8D8E12EE4188E2D672DA9
:1095F000402FD2D88E2D662D402FCED88F819885C2
:10960000C80ED91E3C852B85821693060CF4BFCF5D
:109610003A872987B201882777FD8095982F0E9485
:1096200058E720E030E040E05FE30E9452E6E62E9B
:10963000C72E782E692E1501089421083108EB8178
:10964000FC81BF01882777FD8095982F0E9458E7FD
:10965000F3012E2D3C2D4F2F5E2F0E9445E8F30184
:109660002E2D3C2D4F2F5E2F0E9445E85B016C0193
:10967000229CC001239C900D329C900D11242981C5
:109680003A81829FB001839F700D929F700D1124CB
:10969000882777FD8095982F0E9458E79B01AC01A1
:1096A000C601B5010E9452E65B016C018B819C8171
:1096B000E981FA818E9FB0018F9F700D9E9F700D82
:1096C0001124882777FD8095982F0E9458E79B01E9
:1096D000AC01C601B5010E9451E60E94A8E80E94B3
:1096E00025E751012D813E81309521953F4FC9805D
:1096F000DA808D819E81C81AD90AE985FA85CE1A49
:10970000DF0A7A836983190136C029813A811216EA
:1097100013065CF00894411C511C8F819885880EBB
:10972000991E280D391D3A832983E981FA81EC0DB0
:10973000FD1DFA83E983E42CE10E7A2C7F0C8E2D3B
:10974000672D402F4B8628D8FF2DFA196F2E8E2DAE
:109750006F2F402F21D89B85E12EE91A8E2D672D82
:10976000402F1AD88E2D662D402F16D80894A108A8
:10977000B108C20CD31CC5010196181619062CF2AB
:109780002E96E2E10C94D8E98A3010F4805D0895B9
:10979000895C0895A1E0B0E0E0EDFBE40C94C9E938
:1097A000F82E042F122F6093761C8F5F8093751C08
:1097B000842F82958F706983E7DF482F8F2D698111
:1097C000212FB7DB802F8F70DFDF482F8091751C32
:1097D0006091761C212FADDB2196E5E00C94E5E944
:1097E000FF920F931F93082F162FF090751C8F2D4B
:1097F0008F5F8093751C802F82958F70C5DF482FF7
:109800008F2D6091761C212F94DBF090751C8F2D8D
:109810008F5F8093751C802F8F70B6DF482F8F2D40
:109820006091761C212F85DB8091751C982F9F5F9E
:109830009093751C6091761C40E2212F7ADB1F917A
:109840000F91FF900895A0E0B0E0E9E2FCE40C94F1
:10985000C8E9FE017096A4E4EA2EACE1FA2E80E09D
:10986000B70148E22E853F858F010E9482D5898508
:109870008093751C8A858093761CC7016B854C8507
:109880002D852DDA2096E6E00C94E4E9A0E0B0E026
:10989000ECE4FCE40C94C8E9FE017096B4E4EB2E11
:1098A000BCE1FB2E81E0B70148E22E853F858F01A8
:1098B0000E9482D589858093751C8A858093761C49
:1098C000C7016B854C852D850ADA2096E6E00C945D
:1098D000E4E9A0E0B0E0EFE6FCE40C94C8E9FE01A6
:1098E0003E9604E4E02E0CE1F02E81E0B70148E260
:1098F0002C853D858F010E9482D589858093751CBA
:109900008A858093761CC7016B8540E020E0E7D90B
:109910002096E6E00C94E4E9EF92FF920F931F93F8
:10992000CF93DF93082FC3E0D0E020E014E68AE075
:10993000E82E802F612F0E944CE9F82E882321F415
:10994000222311F4113069F48091751C982F9F5FC8
:109950009093751C4F2D405D6091761C20E0E9DAF4
:1099600021E0812F6E2D0E944CE9219731F0F19E6C
:10997000102D1124011B182FDCCFCDB7DEB7E6E088
:109980000C94E4E98093751C6093761C842FC4CFFB
:10999000A0E0B0E0EEECFCE40C94C7E9D82ECB01DB
:1099A0007A0135E23093771C222331F020E32093B3
:1099B000781CC9E7DCE102C0C8E7DCE16EE67CE1C7
:1099C0004AE050E00E9447ED0EE61CE1F80101C0BC
:1099D000899381918823E1F71E141F0484F48EE299
:1099E0008993C7016EE67CE14AE050E00E9447EDB2
:1099F00001C08993F80181918F018823D1F7D88222
:109A00001982CDB7DEB7E7E00C94E3E9AF92CF92CD
:109A1000EF92FF920F931F93CF93DF93182FF62EA1
:109A2000EA01B901202F85E740E050E0B1DF8DB7B2
:109A30009EB709979EBF8DBFEDB7FEB73196ADB704
:109A4000BEB711961C93F182E282C382A48287E79B
:109A50009CE196838583D087C783F5DE8DB79EB75B
:109A600009969EBF8DBFDF91CF911F910F91FF90FF
:109A7000EF90CF90AF900895AF92CF92EF920F9367
:109A8000CC24AA24C3DF0F91EF90CF90AF9008951C
:109A9000AF92CF92EF92FF920F931F93CF93DF93EA
:109AA000182FF62EEA01B901202F84E640E050E09D
:109AB0006FDF8DB79EB709979EBF8DBFEDB7FEB71D
:109AC0003196ADB7BEB711961C93F182E282C38284
:109AD000A48287E79CE196838583D087C783B3DE22
:109AE0008DB79EB709969EBF8DBFDF91CF911F9115
:109AF0000F91FF90EF90CF90AF900895AF92CF92DB
:109B0000EF920F93CC24AA24C3DF0F91EF90CF9054
:109B1000AF900895AF92CF92EF92FF920F931F9361
:109B2000CF93DF93182FF62EEA01B901202F615051
:109B3000704085E741E050E02BDF8DB79EB7099775
:109B40009EBF8DBFEDB7FEB73196ADB7BEB71196CC
:109B50001C93F182E282C382A48287E79CE1968310
:109B60008583D087C7836FDE8DB79EB709969EBF6A
:109B70008DBFDF91CF911F910F91FF90EF90CF900C
:109B8000AF900895AF92CF92EF920F93CC24AA2476
:109B9000C1DF0F91EF90CF90AF900895AF92CF9229
:109BA000EF92FF920F931F93CF93DF93182FF62E10
:109BB000EA01B901202F6250704085E742E050E091
:109BC000E7DE8DB79EB709979EBF8DBFEDB7FEB795
:109BD0003196ADB7BEB711961C93F182E282C38273
:109BE000A48287E79CE196838583D087C7832BDE99
:109BF0008DB79EB709969EBF8DBFDF91CF911F9104
:109C00000F91FF90EF90CF90AF900895AF92CF92C9
:109C1000EF92FF920F931F93CF93DF93182FF62E9F
:109C2000EA01B901202F6150704084E641E050E024
:109C3000AFDE8DB79EB709979EBF8DBFEDB7FEB75C
:109C40003196ADB7BEB711961C93F182E282C38202
:109C5000A48287E79CE196838583D087C783F3DD61
:109C60008DB79EB709969EBF8DBFDF91CF911F9193
:109C70000F91FF90EF90CF90AF900895AF92CF9259
:109C8000EF920F93CC24AA24C1DF0F91EF90CF90D5
:109C9000AF900895CF92DF92EF920F931F93CF93DF
:109CA000DF93182F362F6A01CCE3D0E0CA01BE0142
:109CB0000E9458E98DB79EB70B979EBF8DBFADB779
:109CC000BEB71196EDB7FEB7118311963C9311976D
:109CD00012962C93129713960C9313971496EC925A
:109CE00014978DE391E016969C938E931597189692
:109CF0007C936E9317976C9FC0016D9F900D7C9F16
:109D0000900D1124F601E81BF90B1A96FC93EE93C3
:109D1000199799DD8DB79EB70B969EBF8DBFDF91CA
:109D2000CF911F910F91EF90DF90CF900895EF9218
:109D30000F9320E000E0EE24ADDF0F91EF90089547
:109D4000A0E1B0E0E6EAFEE40C94C0E9D82EB62E1D
:109D5000E986FA860B871C872D873E874F87588BAD
:109D6000F82CCE010196BE01675F7F4F0E94C1D8DB
:109D700069807A808B809C808DB79EB70D979EBF3F
:109D80008DBF0DB71EB70F5F1F4FEDB7FEB7D18266
:109D9000F801B182C282A382F48287E491E09683C3
:109DA0008583C401B30120E13EE040E050E00E9421
:109DB0007FE9F801278310869CE3C92ED12CE12C82
:109DC000F12CC401B301A70196010E947FE9662E20
:109DD000CA01B901A70196010E947FE9F8016187D4
:109DE0001286638614862FDD8DB79EB70D969EBFB3
:109DF0008DBF6096EEE00C94DCE9CF92EF920F936A
:109E0000CF93DF93EDB7FEB73B97FEBFEDBFCDB766
:109E1000DEB72196818369830A83EB82CC8285E653
:109E200091E09E838D83CA01B90124E630E040E0D1
:109E300050E00E94A1E92F83388749875A8703DDC4
:109E40008DB79EB70B969EBF8DBFDF91CF910F91BF
:109E5000EF90CF9008950F930E945B4388E068E0F5
:109E60004FE620E301E020D982E062E04CE759E0D0
:109E700022E01FD882E064E04BE659E020E019D8E8
:109E800082E065E04CE559E020E013D880E10E94D3
:109E900076B0882379F480E20E9476B0882351F46A
:109EA00080E40E9476B0882329F480E80E9476B08E
:109EB000882361F30F9108950F93CF93DF93EC0103
:109EC000662311F00E945B4380E060E04FE727E0EB
:109ED00001E00E947245CE010E9496EC813191050D
:109EE00008F409D181E060E0AE0122E00E94594708
:109EF000DF91CF910F9108950F93880F880F880FEE
:109F0000480F01E0662309F400E080E0642F4FE78A
:109F100027E00E9472450F91089509981198ECE787
:109F2000F0E080E480838081807E816080838FEE9A
:109F300080937A000895EF92FF920F931F93CF932F
:109F4000DF93F8946091880F7091890F80E090E022
:109F50000E9456E72091D0063091D1064091D2065A
:109F60005091D3060E9452E62FE832EC45E75FE3BA
:109F70000E9445E87B018C01762F272F3F2D402F33
:109F8000512FCA01B9010E9425E7CB0160E470E0BE
:109F90000E946CE9EC019093D9068093D8066E2D4F
:109FA0007F2D802F912F20E030E040E85CE30E947D
:109FB00045E8262F372F482F592F2093D00630936E
:109FC000D1064093D2065093D306C032D10574F027
:109FD00020E030E040E85FE30E9452E66093D00664
:109FE0007093D1068093D2069093D3066091D006E9
:109FF0007091D1068091D2069091D30620E030E096
:10A0000040EF50E40E94BDE6262F372F482F592FEE
:10A010002093D4063093D5064093D6065093D706A6
:10A020000E942AE77093DD066093DC061092DB063F
:10A030001092DA0680E090E0DC018093D0069093E5
:10A04000D106A093D206B093D3067894CDB7DEB7ED
:10A05000E6E00C94E4E91F920F920FB60F920BB654
:10A060000F9211242F933F934F935F936F937F939E
:10A070008F939F93AF93BF93EF93FF93609178007B
:10A080007091790080E090E00E9456E79B01AC015E
:10A090006091D0067091D1068091D2069091D3063E
:10A0A0000E9452E66093D0067093D1068093D20648
:10A0B0009093D3068091DA069091DB0601969093F7
:10A0C000DB068093DA0620E1803092070CF033DF64
:10A0D000FF91EF91BF91AF919F918F917F916F9180
:10A0E0005F914F913F912F910F900BBE0F900FBE3C
:10A0F0000F901F9018950F93CF93DF9388E660E041
:10A1000047E127E001E00E94544889E661E045E12B
:10A1100025E000E00E94544886E660E041E027E048
:10A120000E94724587E662E041E023E001E00E9480
:10A1300054486091DC067091DD066054714080E007
:10A1400090E00E9456E720918A0F222329F02AE905
:10A1500039E949E950E404C020E030E040E950E446
:10A160000E94BDE60E9425E7EB0177FD15C0653131
:10A1700071051CF4209791F002C0C4E1D0E04C2F8F
:10A1800041508EE78C1B62E023E001E00E947245A3
:10A19000C431D10559F002C0C0E0D0E043E14C1B0E
:10A1A0008AE662E023E000E00E947245DF91CF91F1
:10A1B0000F9108950E945E421092DF061092E00611
:10A1C0000E942A6480917E0F90917F0FA091800F52
:10A1D000B091810F181619061A061B067CF480919F
:10A1E000820F9091830FA091840FB091850F181664
:10A1F00019061A061B0614F40E94D48881E083D540
:10A20000D1D1FECF0F931F930E943BCB88EB9AE0F6
:10A210000E946FCB8091320F882369F08091310FBB
:10A22000882349F088E261E04FE15BE328E63AE009
:10A2300089010E945ECD8091BD17882369F08091CD
:10A240003010882349F08DE261E04AE45BE326E7C1
:10A250003AE089010E945ECD8091BD17882369F0A4
:10A260008091DF0F882349F08CE261E04FE35BE3EC
:10A2700024E83AE089010E945ECD8091310F882365
:10A2800049F089E261E047EA5BE322E93AE08901CB
:10A290000E945ECD8AE261E04EE95BE320EA3AE0AB
:10A2A00089010E945ECD8091320F882349F08BE2B4
:10A2B00061E045E05BE32CEA3AE089010E945ECD73
:10A2C00080E00E9403D20E9462CB1F910F910895FB
:10A2D0000F931F930E943BCB83EE9AE00E946FCBBB
:10A2E0008CE361E047E951E524EC3AE089010E9402
:10A2F0005ECD8091320F882349F08DE361E04BE71A
:10A3000055EC21ED3AE089010E945ECD8EE361E0DB
:10A310004CEF58EA2AED3AE089010E945ECD80E0D8
:10A320000E9403D20E9462CB1F910F9108958091E9
:10A33000DF06882319F481E00E94FB698091DF0623
:10A34000813019F482E00E94FB698091DF0682303F
:10A3500011F40C94FB6908950F931F9381E061E061
:10A360004BE055E828E53AE089010E945ECD82E0A5
:10A3700062E04DED5FE82EED39E008EE19E00E9455
:10A380005ECD8CE061E040E050E028E23AE08901F7
:10A390000E945ECD8091A11C882349F084E062E098
:10A3A0004DEF57E620E33AE089010E945ECD83E05D
:10A3B00061E04FEF5AE52CE33AE089010E945ECD5F
:10A3C00085E061E043E459E527E43AE000E51AE07E
:10A3D0000E945ECD86E061E048EF50E42CE53AE073
:10A3E00089010E945ECD8BE062E048E651E521EFF5
:10A3F00039E00DEF19E00E945ECD88E062E042E0B6
:10A4000051E529E03AE089010E945ECD89E062E0F1
:10A4100040E050E025E13AE089010E945ECD8AE00B
:10A4200061E046E052E92FE13AE089010E945ECD09
:10A430001F910F9108950F931F938CE061E040E00E
:10A4400050E028E23AE089010E945ECD8091A11C93
:10A45000882349F084E062E04DEF57E620E33AE0DC
:10A4600089010E945ECD83E061E04FEF5AE52CE365
:10A470003AE089010E945ECD85E061E043E459E560
:10A4800027E43AE000E51AE00E945ECD8BE062E04E
:10A4900048E651E521EF39E00DEF19E00E945ECD6D
:10A4A00088E062E042E051E529E03AE089010E945B
:10A4B0005ECD89E062E040E050E025E13AE08901CC
:10A4C0000E945ECD8AE061E046E052E92FE13AE089
:10A4D00089010E945ECD1F910F9108950F931F93E4
:10A4E00087E061E040E050E02EEB39E000ED19E05C
:10A4F0000E945ECD82E062E04DED5FE82EED39E036
:10A5000008EE19E00E945ECD8BE062E048E651E57E
:10A5100021EF39E00DEF19E00E945ECD09E01AE06D
:10A5200088E062E042E051E598010E945ECD05E1DD
:10A530001AE089E062E040E050E098010E945ECDC0
:10A540000FE11AE08AE061E046E052E998010E94DA
:10A550005ECD1F910F9108950E943BCB83E791E060
:10A560000E9488CB82E290E056D0BC0185E04CE1AD
:10A5700051E90E94B6CB88E660E070E042E051E528
:10A580000E94B6CB8091DF06882309F4A7DF809173
:10A59000DF06813009F4E0DE8091DF06823009F4C5
:10A5A0004ACF08951F931091320F0E94B5C6B5DCB3
:10A5B00080EF0E9476B088E791E06CE671E04CE0B5
:10A5C00050E00E9411ED81E00E946CCBC5DF80E07D
:10A5D0000E9403D20E9430CC873019F481E093D3DB
:10A5E00006C08C3051F480E090E061E08AD288238C
:10A5F00041F00E9462CBB0DF04C0893011F40E94A8
:10A60000DEA68091320F181711F30E9462CBA4DFEF
:10A610001091320FDCCF2091240F223018F021E06E
:10A620002093240F2091240F222351F4FC01EE0FDC
:10A63000FF1FEE0FFF1FE151F54F259134910BC025
:10A64000213059F4FC01EE0FFF1FEE0FFF1FEF50FA
:10A65000F54F25913491C9010895EFEEFAE0259167
:10A660003491C901089586E2EBE8FCE1DF011D9217
:10A670008A95E9F70895AF92CF92EF920F931F93C7
:10A68000DF93CF93CDB7DEB72A97DEBFCDBF8A2D3C
:10A69000002311F4112391F00E1531F41C1539F437
:10A6A0008156481739F40CC00E1560F405C01C150E
:10A6B00048F402C0481730F481E005C080E003C0D0
:10A6C00082E001C083E02A96DEBFCDBFCF91DF914B
:10A6D0001F910F91EF90CF90AF900895EF920F934D
:10A6E000413059F1423009F05BC030918D1C332369
:10A6F00029F490918E1C992309F44EC04DB75EB792
:10A700004D5050405EBF4DBFEDB7FEB73196ADB76F
:10A71000BEB711968C931197618322830383E482E1
:10A720008EE499E2968385833783108680918E1C10
:10A73000818712868091911C22C03091971C33230F
:10A7400021F49091981C992339F1ADB7BEB71D97AC
:10A75000BEBFADBFEDB7FEB7319611968C93618346
:10A7600022830383E4828DE399E296838583378392
:10A7700010868091981C8187128680919B1C90E0A6
:10A780008F599F4F9487838781D84DB75EB7435FBA
:10A790005F4F5EBF4DBF04C048E459E20E942847A6
:10A7A0000F91EF900895A2E1B0E0E9EDF3E50C948C
:10A7B000C8E9E82EF62E142F022F4091A31C442343
:10A7C000E1F400D000D00F92EDB7FEB73196CE0184
:10A7D0000196ADB7BEB712969C938E93119782E106
:10A7E000828383E399E2948383830E942FD80F901E
:10A7F0000F900F900F900F9042C08091A11C9E016E
:10A800002F5F3F4F882301F18DB79EB709979EBFF9
:10A810008DBFEDB7FEB73196ADB7BEB712963C937C
:10A820002E93119782E182838DE299E29483838350
:10A830004583168284EA9CE1908787830E942FD803
:10A840008DB79EB7099619C0ADB7BEB71797BEBFF3
:10A85000ADBFEDB7FEB7319612963C932E9311978C
:10A8600082E182832AE239E234832383458316829C
:10A870000E942FD88DB79EB707969EBF8DBF8E2D95
:10A88000BE016F5F7F4F4F2D212F0E94BF46629602
:10A89000E6E00C94E4E98BE10E948FC88BE10E9412
:10A8A0008FC885E50E948FC88AEA0E948FC880E021
:10A8B0000E948FC881E08093E00684EF91E024EF4E
:10A8C00031E0F9013197F1F70197D9F708951F9316
:10A8D0001092B11C8DB79EB707979EBF8DBFEDB785
:10A8E000FEB7319685E7ADB7BEB711968C9312E0EF
:10A8F000118381E0828381EB9CE19483838381E0F7
:10A9000090E0968385830E9496C81093E0068DB7E9
:10A910009EB707969EBF8DBF84EF91E024EF31E094
:10A92000F9013197F1F70197D9F71F910895A1E047
:10A93000B0E0EDE9F4E50C94C3E98983B62EC7DFF6
:10A9400081E58093DE061092710B91E7992EAA247F
:10A95000A3946E010894C11CD11C81E0E82EF12C57
:10A9600004E110E028C08DB79EB707979EBF8DBF4A
:10A97000EDB7FEB73196ADB7BEB711969C92A182E6
:10A98000A282D482C382F682E5820E9496C8109386
:10A990003F1E00933E1E8DB79EB707969EBF8DBF8C
:10A9A00080913E1E90913F1E009721F08091710B87
:10A9B0008823B1F3BA948091710B882311F4BB20E2
:10A9C00091F61092DE0680E090E00E94706980911E
:10A9D000710B882341F00E948AC98091730B90917A
:10A9E000740B0E9470698091A31C2196EBE00C947B
:10A9F000DFE9A1E0B0E0EFEFF4E50C94BFE9898373
:10AA0000862E8091A11C882309F469C083E5809378
:10AA1000DE061092710B992453E7552E6624639439
:10AA200042E0742E6E010894C11CD11C31E0E32E6B
:10AA3000F12C26E4A22EB12C45C00091730B10918D
:10AA4000740B0F5F1F4F0E94BD692DB73EB72B508F
:10AA500030403EBF2DBFEDB7FEB73196ADB7BEB7A4
:10AA600011965C9261827282D482C382F682E58200
:10AA700010870783818712860E9496C8B0923F1E76
:10AA8000A0923E1E2DB73EB7255F3F4F3EBF2DBF64
:10AA900080913E1E90913F1E009721F08091710B96
:10AAA0008823B1F38A948091710B882359F00E9416
:10AAB0008AC9E091730BF091740B9080992011F486
:10AAC0001092710B8091710B882329F4882019F062
:10AAD000992009F4B2CF8FEF6FE029DF01C09924EC
:10AAE000892D2196EFE00C94DBE91F93182F64E188
:10AAF0001EDF811719F462E37CDF01C080E01F9143
:10AB00000895A0E0B0E0E7E8F5E50C94C5E9EC01B4
:10AB1000F0908B1CB0908C1C009721F09093331E0A
:10AB20008093321E8EE591E09093411E8093401EEB
:10AB300001E011E1B4E1CB2EB9E2DB2E002309F4F0
:10AB4000ABC00E945B43D7DA80E060E045E628E0D6
:10AB500001E00E94724581E060E042E259E222E0B9
:10AB600000E0EE240E94284780918B1C882329F462
:10AB700080918C1C882309F473C080E06EE14FE75C
:10AB800026E101E0A2E0EA2E0E94ED4780E062E0CB
:10AB90004EE159E220E004E0FBEFEF2E0E9428474F
:10ABA00084E062E042E020E002E098DD8CE062E0D8
:10ABB00049E159E220E005E00E9428478DB79EB7A1
:10ABC00009979EBF8DBFEDB7FEB73196ADB7BEB743
:10ABD00011961C9382E08183128283838BEF84839E
:10ABE000D682C5828091A21C878310860E94464C23
:10ABF0008DB79EB709969EBF8DBF8091A11C8823FB
:10AC000051F48BE063E04AE059E222E0ECEFEE2EF3
:10AC10000E94284707C087E464E146E328E000E09B
:10AC20000E94724580E063E046E059E220E004E0E3
:10AC30007DEFE72E0E94284784E063E041E020E0BA
:10AC400002E04CDD84E06BEF78E242E020E001E0DE
:10AC50000E94374785E062E040E023E0A4DD0AC0BF
:10AC600085EF90E0D8DC60E040E050E021E000E0DB
:10AC70000E94F6918EE090E0CEDCAC018CE067E0C3
:10AC800020E00E945947209739F480E067E043EFC5
:10AC900058E220E00E9459472EDA80E80E9476B000
:10ACA000882331F0209721F480E02DD001E001C00D
:10ACB00000E080E20E9480B0882371F40E9412912B
:10ACC000811101E0209709F439CF8091321E9091D3
:10ACD000331E009709F032CF80EF0E9476B080914A
:10ACE0008B1CF81649F481E090E020918C1CB21680
:10ACF00029F480E090E002C081E090E0CDB7DEB7BB
:10AD0000E9E00C94E1E9A0E0B0E0E9E8F6E50C94B4
:10AD1000C7E9182FA8DCBFDD84EF91E024EF31E014
:10AD2000F9013197F1F70197D9F7B5DD86E5809301
:10AD3000DE061092710BEE2491E046E7F42EC0E19E
:10AD4000D0E06CC0992361F10E945B430E9429907E
:10AD50008DEF90E060DCBC0182E040E020E002E0AA
:10AD60000E9437478DE090E056DCAC0180E063E064
:10AD700020E000E038E0E32E0E9428478EE090E0DB
:10AD80004ADCAC018CE067E020E00E94594780E09B
:10AD90006AE24EE728E001E00E94544822E0E22EF9
:10ADA000AAD900D00F92EDB7FEB73196ADB7BEB7B6
:10ADB0001196FC92118212820E9496C8D093331E83
:10ADC000C093321E0F900F900F908091321E909181
:10ADD000331E0097D1F782E06CE24E2D24E001E0B3
:10ADE0000E947245B2E0EB0E8E2D8D3740F082E06E
:10ADF0006CE24BE724E000E00E947245EE2480E222
:10AE00000E9476B0882321F01092DF0600E0BEC0D9
:10AE10000E94129191E0882309F490E08091710BD7
:10AE2000882309F48FCF8091710B882309F486C0A1
:10AE30000E948AC98091A51E8236C1F482E0809367
:10AE4000DF068093E00681E080938B1CADE8BCE1D7
:10AE50003091730B2091740B832F922FFC018AE0A9
:10AE600001900D928150E1F701E001C000E0809176
:10AE7000A51E8336B1F481E08093DF068093E0065F
:10AE800080938C1CA7E9BCE13091730B2091740B6B
:10AE9000832F922FFC018AE001900D928150E1F7FF
:10AEA00001E08091DF06813009F049C010DD86E5C0
:10AEB0008093DE061092710B98E2F92E86E7D82E69
:10AEC000EE24E394C4E1D0E01BC000D00F92EDB7B4
:10AED000FEB73196ADB7BEB71196DC92E182128211
:10AEE0000E9496C8D093331EC093321E0F900F90CD
:10AEF0000F908091321E9091331E0097D1F7FA94F3
:10AF00008091710B882311F4FF20F9F68091710B69
:10AF10008823A9F00E948AC981E080938B1CADE848
:10AF2000BCE19091730B8091740B292F382FF9019C
:10AF30008AE001900D928150E1F701C000E08FEFAF
:10AF40006FE0F5DC1092DE061092710B8091A11C6F
:10AF5000882361F089E190E06FEF7FEF40E00E948D
:10AF6000B7B0112381F084EF91E00BC088EE93E03D
:10AF70006FEF7FEF40E00E94B7B0112321F080E433
:10AF800096E061E0BEDD80EF0E9476B0802FCDB705
:10AF9000DEB7E7E00C94E3E9A1E0B0E0E2EDF7E52D
:10AFA0000C94BFE9E091E006F0E0E052F94F8081B7
:10AFB00089830E945B4380E062E04FE859E220E031
:10AFC0000E94594781E064E040E859E220E00E9495
:10AFD000594784E090E01FDBAC018CE067E020E0A3
:10AFE0000E94594783E167E04DE759E220E00E9463
:10AFF000594781E48093DE0680ED97E024EF31E04D
:10B00000F9013197F1F70197D9F71092710B84E1AB
:10B0100090E09093331E8093321E11E000E0B1E681
:10B02000FB2E552453945E010894A11CB11CA1E091
:10B030008A2E912CF4E1CF2ED12CE4EF6E2EE1E09C
:10B040007E2EC1C08DB79EB707979EBF8DBFEDB74F
:10B05000FEB73196ADB7BEB71196FC9211825282FF
:10B06000B482A382968285820E9496C88DB79EB7CD
:10B0700007969EBF8DBF11E006C080E20E9476B0A9
:10B0800011E0811110E08091710B882341F48091CF
:10B09000321E9091331E009711F0112371F78091A9
:10B0A000321E9091331E009709F467C00E948AC92E
:10B0B0004981E091730BF091740B8081481709F07E
:10B0C0004EC08FE064E050E022E030E000E0EE248B
:10B0D0000E943C4D2091E00630E02150304075E068
:10B0E000220F331F7A95E1F78981280F311DC9019D
:10B0F00064E0880F991F6A95E1F7820F931FA09172
:10B10000B21CB091B31CE091730BF091740BA80FBB
:10B11000B91F319680E101900D928150E1F7809145
:10B12000E00690E00197298155E0880F991F5A9514
:10B13000E1F7820F911D9C0144E0220F331F4A95D5
:10B14000E1F7280F391FE091B21CF091B31CE20F18
:10B15000F31F108A89818F5F898300E007C088EE22
:10B1600093E0F3013197F1F70197D9F7D092331EAD
:10B17000C092321E1092710B26C01123D9F00F5FBE
:10B18000D092331EC092321E0233E0F080E062E0C3
:10B190004EE659E220E00E94594784E690E0909301
:10B1A000331E8093321E8091321E9091331E009781
:10B1B000D1F712C080E20E9476B011E0882319F026
:10B1C00010E001C011E08981803220F4112309F0E0
:10B1D00039CF0AC0112341F0E091E006F0E0E052DF
:10B1E000F94F8981808311E0812F2196EFE00C9443
:10B1F000DBE9FF920F931F93CF93DF93F82E0E940A
:10B200005B4307E02F2D209F80011124C0E0D0E098
:10B210006C2F9F2D943041F4C43030F080E06C2FBF
:10B2200045E10E94CD4720C02091E00630E021504A
:10B23000304055E0220F331F5A95E1F7200F311FA0
:10B240002C0F3D1FC90144E0880F991F4A95E1F773
:10B25000820F931F4091B21C5091B31C480F591F8D
:10B2600080E020E00E94B6462196C730D10581F6E5
:10B27000CDB7DEB7E5E00C94E5E98091B21C909182
:10B28000B31C0C9493EAA3E0B0E0E9E4F9E50C9474
:10B29000BCE90E945B4380E494E00E94F9E990934A
:10B2A000B31C8093B21C009719F40E942B4FA3C1CA
:10B2B000E82FF92F80E494E0DF019C011D922150DA
:10B2C0003040E1F71092E1061092E2060E940ECAA9
:10B2D00088EC90E09093331E8093321EE091E0065C
:10B2E000F0E0E052F94F8081803220F455DE88236F
:10B2F00009F480C18091321E9091331E009709F4A9
:10B3000079C184E48093DE061092710B08EC10E0A2
:10B310001093331E0093321E8AE089838DB79EB747
:10B3200007979EBF8DBFEDB7FEB7319684E6ADB7E8
:10B33000BEB711968C93118281E082835E010894DE
:10B34000A11CB11CB482A38281E090E09683858326
:10B350000E9496C81093351E0093341EEDB7FEB7B9
:10B360003796FEBFEDBF80E044DF10E0B8ECCB2E97
:10B37000D12CAAE09A2EF4E66F2E552453948A2CF1
:10B380007B2CE1E0AE2EB12C74E4472E8091710B42
:10B39000882309F467C00E948AC92091730B3091F9
:10B3A000740B3B832A8383E090E035D9AC0180E0C5
:10B3B00067E020E00E945947412F4F5F85E067E03A
:10B3C0000E94C24C8091E006823011F483E001C0FB
:10B3D00083E167E04BE659E220E00E945947809103
:10B3E000E006823011F483E101C083E067E048E6C3
:10B3F00059E220E00E94594787E0189F100111246C
:10B40000FF2416C0220D331D2F5F3F4F220F331F25
:10B410008A819B81280F391FD9014D915C918FE062
:10B420006F2D26E030E000E0EE240E947E4DF39484
:10B430002F2D30E0143019F484E090E002C087E052
:10B4400090E028173907F4F21092710B8CEA9DE016
:10B45000E4EFF1E03197F1F70197D1F7D092331E85
:10B46000C092321E8091341E9091351E0097E1F4F7
:10B470009982EDB7FEB73797FEBFEDBF3196ADB7F6
:10B48000BEB711966C921182528283827482B68208
:10B49000A5820E9496C8D092351EC092341EEDB788
:10B4A000FEB73796FEBFEDBF80E80E9476B08823D6
:10B4B00029F01150153058F014E009C080E40E94C2
:10B4C00076B0882331F01F5F153008F010E0812F2F
:10B4D00090DE8091DF06813009F040C080E10E945B
:10B4E00076B08823D9F18091E006813019F40E946A
:10B4F0000ECA02C00E94E5C9E091E006F0E0E05209
:10B50000F94F8081803220F447DD882309F472C02E
:10B510004092DE061092710BD092331EC092321E02
:10B5200099822DB73EB7275030403EBF2DBFEDB7B3
:10B53000FEB73196ADB7BEB711966C9211825282AA
:10B5400083827482B682A5820E9496C8EDB7FEB748
:10B550003796FEBFEDBF80E04CDE10E080E20E9437
:10B5600076B0882339F48091321E9091331E009773
:10B5700009F00CCF19822DB73EB7275030403EBF9F
:10B580002DBFEDB7FEB7319684E6ADB7BEB71196C5
:10B590008C93118281E08283CE0101969483838310
:10B5A00081E090E0968385830E9496C81092DE0623
:10B5B0001092710B8091321E9091331EEDB7FEB741
:10B5C0003796FEBFEDBF0097A9F40E945B4380E071
:10B5D00062E049E559E220E00E94594784E690E0A4
:10B5E0009093331E8093321E8091321E9091331EB1
:10B5F0000097D1F742DE2396E2E10C94D8E9A1E06E
:10B60000B0E0E5E0FBE50C94BCE988E48093DE065D
:10B610001092710B84EF91E09093331E8093321E51
:10B620008FEF898301E010E0F8E6FF2E5E010894B9
:10B63000A11CB11CE1E08E2E912C33243A9474EFBE
:10B64000C72E71E0D72E64EF662E61E0762E5EEF96
:10B65000252E42E3442E512C002319F18091E0065F
:10B66000813019F489EC99E202C086EC99E261E03C
:10B670000E945C4F84E060E04EEB59E222E00E94C1
:10B68000594780E06BE04FE729E201E032E0E32E2A
:10B690000E94924882E067E04CEA59E220E00E9472
:10B6A00059470E947B508DB79EB707979EBF8DBFAD
:10B6B000EDB7FEB73196ADB7BEB71196FC921182C9
:10B6C00081E08283B482A382968285820E9496C89A
:10B6D00039828DB79EB707969EBF8DBF84EF91E0EC
:10B6E000F6013197F1F70197D9F78091710B882313
:10B6F00009F441C00E948AC91091BB1E1092BB1E62
:10B7000080E062E047EA5EE120E005E0EE24EA94B2
:10B710000E94A7461093BB1E1091CF1E1092CF1E01
:10B7200080E063E04BEB5EE120E0EE240E94A74660
:10B730001093CF1E1091E31E1092E31E80E064E090
:10B740004FEC5EE120E0EE24E3940E94A7461093C4
:10B75000E31E1092F71E80E065E043EE5EE120E01C
:10B7600092E0E92E0E94A7461092710B7092331E50
:10B770006092321E11E00E94129101E0882309F4C8
:10B7800000E080E80E9476B0882329F480E862E037
:10B790000E94A0B08111298280E40E9476B08823A3
:10B7A00031F480E462E00E94A0B0882311F09DEFA4
:10B7B000998380E20E9480B0882311F0ABEFA983C7
:10B7C00080E10E9480B0882311F0B7EFB9838091A7
:10B7D000DF06813031F580E10E9495B0882309F1C0
:10B7E00089E190E06FEF7FEF40E00E94B7B0809179
:10B7F000E006813011F46BD809C04DD884EF91E098
:10B80000F6013197F1F70197D9F745D850923F1ECD
:10B8100040923E1E80913E1E90913F1E0097D1F7B0
:10B8200001E080E20E9495B0882341F089E190E038
:10B830006FEF7FEF40E00E94B7B007C08091321EEB
:10B840009091331E009709F007CF1092DE061092F8
:10B85000710B8091321E9091331E0097B9F4112321
:10B8600011F00E945B4380E062E048E959E220E089
:10B870000E94594784E690E09093331E8093321ED5
:10B880008091321E9091331E0097D1F70E94ACB088
:10B890002196E2E10C94D8E9A1E0B0E0E2E5FCE514
:10B8A0000C94C9E9F82E162F8DB79EB707979EBF47
:10B8B0008DBFEDB7FEB731968EED9CE1ADB7BEB74B
:10B8C00012969C938E93119784E1828389E092E390
:10B8D00094838383F582168249830E942FD8EDB723
:10B8E000FEB73796FEBFEDBF4981442309F463C01C
:10B8F0000E945B4381E061E072E342E020E00DEFF3
:10B900000E94374782E062EF71E340E020E000E010
:10B910000E9437478DB79EB707979EBF8DBFEDB783
:10B92000FEB73196ADB7BEB711961C9284E0818305
:10B93000128225EE31E334832383F58216820E943E
:10B94000694CEDB7FEB73196ADB7BEB711961C92F4
:10B9500085E0818312828AED91E39483838315834A
:10B9600016820E94694CEDB7FEB73796FEBFEDBF59
:10B970008EE090E00E940B53AC018BE067E020E08A
:10B980000E94594784EF91E06FE070E040E00E9430
:10B99000B7B004EF11E009C08CED95E0F8013197E4
:10B9A000F1F70197D9F70E94129180E20E9476B0D8
:10B9B000882391F307C080EA90E06FE070E040E0F8
:10B9C0000E94B7B02196E5E00C94E5E91F936CEC7A
:10B9D00079E2FB011491181729F01F3F19F0655FF8
:10B9E0007F4FF7CF84EB9CE14BE050E00E947BEC73
:10B9F0006091B71C7091B81C8AEC9CE144E150E066
:10BA00000E949FEC81E01F3F09F480E01F910895A0
:10BA10008091240F882329F44091BB1C5091BC1CB9
:10BA200004C04091BD1C5091BE1C80E062E020E04B
:10BA30000C945947A0E0B0E0E0E2FDE50C94C4E9C5
:10BA4000182F062FC3DF8091B41C8F3F41F441E0D3
:10BA5000013009F040E08CE0612F1EDFDCC0812F57
:10BA60000E94FB68F82EDD24D39486FFDD248F2D01
:10BA70008F77DD2041F081958F77C82FD0E0D0956A
:10BA8000C195DF4F02C0C82FD0E0013001F18DB762
:10BA90009EB707979EBF8DBFEDB7FEB731968EED6F
:10BAA0009CE1ADB7BEB712969C938E93119784E13B
:10BAB000828382E891E394838383D683C5830E9443
:10BAC0002FD88DB79EB707969EBF8DBFA4C00E948A
:10BAD0005B4302E094E0C92E85E7A82E81E3B82EEF
:10BAE000023031F580E060E04FE727E001E00E949E
:10BAF000724581E060E04BE751E322E000E0EE2494
:10BB00000E94284782E090E00E940B53AC0180E045
:10BB100067E020E00E94594786E090E00E940B53C6
:10BB2000AC018BE067E020E00E94594771DF01E043
:10BB30000E947B500130B9F4ADB7BEB71797BEBFB6
:10BB4000ADBFEDB7FEB7319611961C92C18212823D
:10BB5000B482A382D683C5830E94694C8DB79EB7F9
:10BB600007969EBF8DBF80E20E9480B0882309F0B7
:10BB700052C080E10E9480B08823B1F06C2F91E028
:10BB8000C6FF90E0FF1CFF24FF1CFD1419F081E0AC
:10BB9000892701C0892F882311F0606801C06F7761
:10BBA000812F0E942D6937C080E80E9480B08823D1
:10BBB00031F480E862E00E94A0B0882339F0BFEF42
:10BBC000C53CDB072CF0219701E005C000E003C075
:10BBD00001E0CCE3D0E080E40E9480B0882331F41F
:10BBE00080E462E00E94A0B0882349F0CC33D10504
:10BBF0001CF4219601E003C001E0C4ECDFEF80EF0C
:10BC000062E00E94A0B00E941291882309F468CFDC
:10BC10000E945B4367CFCDB7DEB7EAE00C94E0E962
:10BC2000A1E0B0E0E6E1FEE50C94BCE9F82E698302
:10BC3000CDDE8091B41C69818F3F41F441E06130D9
:10BC400009F040E08CE06F2D27DE0AC1613021F160
:10BC50008F2D0E94FB682DB73EB7275030403EBF66
:10BC60002DBFEDB7FEB731962EED3CE1ADB7BEB7B7
:10BC700012963C932E93119794E1928327EC31E333
:10BC800034832383858316820E942FD8EDB7FEB7B5
:10BC90003796FEBFEDBFE4C00E945B438F2D0E942C
:10BCA000FB68D82E10E002E0BFE0CB2EA4E94A2EBC
:10BCB000A1E35A2EF7E08F2E912CE1E06E2E712C2D
:10BCC0000230E1F580E060E04FE727E001E00E940C
:10BCD000724581E060E040EC51E322E000E0EE24B8
:10BCE0000E94284781E067E04BEA51E320E00E9490
:10BCF000594786E090E00E940B53AC018BE067E06F
:10BD000020E00E94594787E066E049EA51E320E0DD
:10BD10000EEF72E0E72E0E942847FF2DF03411F05D
:10BD2000F23451F48AE065E04DE951E320E000E0AF
:10BD300032E0E32E0E9428476BDE01E00E947B5038
:10BD4000013009F045C02224332408E0AD2CBB2487
:10BD5000C501022C02C0959587950A94E2F780FFF1
:10BD600002C041E301C040E3802F64E020E00E9474
:10BD7000994701500894211C311C002349F780E0A9
:10BD800068E24BE327E00E947245812F8F5F65E0F8
:10BD90004BE951E320E00E9459472DB73EB72750A9
:10BDA00030403EBF2DBFEDB7FEB73196ADB7BEB741
:10BDB0001196CC9284E08183128254824382B682AF
:10BDC000A5820E94694CEDB7FEB73796FEBFEDBF66
:10BDD00080E20E9480B0882309F042C080E10E9486
:10BDE00080B0882329F08F2D6D2D0E942D6938C0D9
:10BDF00080E40E9480B0882321F0173021F01F5F7B
:10BE000003C000E002C010E001E080E40E9495B0B1
:10BE1000882331F0112311F0115001C017E001E027
:10BE200080E80E9480B0882379F0812F992787FDD0
:10BE300090959401281B390BD30102C0AA0FBB1F98
:10BE40002A95E2F7DA2601E080EF62E00E94A0B0D6
:10BE50000E941291882309F433CF0E945B4332CFB2
:10BE60002196E2E10C94D8E9682F80E02BE030E0E5
:10BE700001C08F5F482F50E0429FF001439FF00DBB
:10BE8000529FF00D1124E757FE4F9081961719F439
:10BE90006F3F41F402C09F3F61F78EE140E0FCDC60
:10BEA00080E00895AFEBBCE18BE001900D928150F2
:10BEB000E1F781E00895A0E0B0E0E1E6FFE50C9451
:10BEC000C6E9F82EEB018A0169018091B41C8F1537
:10BED00011F08F2D7BDD8091B41C8F3F19F48FE121
:10BEE0006F2D24C08F2D0E94FB6888838AECE82E7A
:10BEF0008CE1F82E8BE090E0D7016D917D0120E080
:10BF000001C02F5F422F50E0489FF001499FF00D84
:10BF1000589FF00D1124E757FE4F3081361719F462
:10BF20006F3F41F402C03F3F61F780E240E0B4DC84
:10BF300080E045C0663749F43091B91CF801308380
:10BF40003091BA1CD6013C9306C03181D8013C9394
:10BF50003281F6013083D8014C91F601508138814D
:10BF6000541728F0341738F0531728F00CC0351741
:10BF700010F0431740F4D7012C91222309F0BCCFD5
:10BF800081E26881D3CF30E08BE090E0289FF00120
:10BF9000299FF00D389FF00D1124AFEBBCE1E7575E
:10BFA000FE4F8BE001900D928150E1F7F801808106
:10BFB0008093C01CD6018C918093C11C81E0CDB7C9
:10BFC000DEB7E8E00C94E2E99091240F833061F44D
:10BFD000992329F48091C61C9091C71C08958091E3
:10BFE000C81C9091C91C0895992329F48091C21C02
:10BFF0009091C31C08958091C41C9091C51C089514
:10C00000A0E0B0E0E6E0F0E60C94C6E9F82E062FDA
:10C01000DDDC8091B41C8F3F41F441E0013009F038
:10C0200040E08CE06F2D38DCBFC08F2D0E94FB6894
:10C03000DD24D39486FFDD24182F111F1127111F33
:10C040001D25013011F1112311F081E301C080E3BE
:10C050000BDF802FB9DF00D000D00F92EDB7FEB715
:10C0600031962EED3CE1ADB7BEB712963C932E93C0
:10C07000119724E12283948383830E942FD80F9009
:10C080000F900F900F900F908FC00E945B4302E0C3
:10C0900094E0C92EC6E8D1E3023031F580E060E0DB
:10C0A0004FE727E001E00E94724581E060E04DE843
:10C0B00051E322E000E0EE240E94284782E090E075
:10C0C0000E940B53AC0180E067E020E00E945947DA
:10C0D00086E090E00E940B53AC018BE067E020E02B
:10C0E0000E94594795DC01E00E947B50013019F510
:10C0F000112311F081E301C080E3B6DE83E064DF49
:10C100002DB73EB7275030403EBF2DBFEDB7FEB72D
:10C110003196ADB7BEB711961C92C1821282D483FC
:10C12000C383968385830E94694C2DB73EB7295FF0
:10C130003F4F3EBF2DBF80E20E9480B08823A1F513
:10C1400080E10E9480B08823A1F0112319F011E052
:10C150001D2501C01D2D8F2D0E94FB68112319F094
:10C16000682F606802C0682F6F778F2D0E942D693D
:10C170001BC080E40E9480B0882329F480E80E94DC
:10C1800080B0882321F081E0182701E001C000E0A1
:10C1900080EF62E00E94A0B00E941291882309F40F
:10C1A0007BCF0E945B437ACFCDB7DEB7E8E00C943B
:10C1B000E2E9A3E0B0E0EFEDF0E60C94CBE9162F56
:10C1C000BE016F5F7F4FAE014E5F5F4F9E012D5FDF
:10C1D0003F4F71DE8823E1F19091BF1C2B818A8152
:10C1E000963739F4281780F489E2698140E054DBFE
:10C1F0002FC09981281718F0981B998302C0891BBA
:10C20000898389818F5F8983812FDEDE2DB73EB7D9
:10C21000275030403EBF2DBFEDB7FEB731962EED13
:10C220003CE1ADB7BEB712963C932E93119724E133
:10C230002283948383838981858316820E942FD8E9
:10C240002DB73EB7295F3F4F3EBF2DBF81E001C0F4
:10C2500080E02396E3E00C94E7E9A3E0B0E0E3E3B9
:10C26000F1E60C94CAE9182F062FBE016F5F7F4FCD
:10C27000AE014E5F5F4F9E012D5F3F4F1CDE882356
:10C2800009F485C0298130E04091BF1C8AEC9CE113
:10C29000FC01508101965417D9F75A814B814517FB
:10C2A00008F40195602F772767FD7095620F731F63
:10C2B000852F90E0451720F06817790724F031C0EA
:10C2C00086179707A4F58CE1EA3CF80741F401C012
:10C2D000FC01CF01019621812223D1F701C03197C2
:10C2E000408150E08BE090E001C05F5F252F30E09F
:10C2F000289FF001299FF00D389FF00D1124E7577A
:10C30000FE4F2081241719F44F3F21F440C02F3FE6
:10C3100061F73DC0463719F46091BA1C34C06281A0
:10C3200032C0842F90E08617970734F02CC0842FFA
:10C3300090E0681779073CF5DF0111968181882329
:10C3400011F4AAECBCE14C9150E08BE090E001C00C
:10C350005F5F252F30E0289FF001299FF00D389F67
:10C36000F00D1124E757FE4F2081241719F44F3F99
:10C3700021F40DC02F3F61F70AC0463719F46091D0
:10C38000B91C01C06181812F68D781E001C080E0C4
:10C390002396E4E00C94E6E9A0E0B0E0E2EDF1E6FB
:10C3A0000C94C2E9182F613011F003DFB3C00EDB2B
:10C3B0008091B41C8F3F29F48BE0612F41E06CDA4F
:10C3C000A9C00E945B43812F16D7882EFF2402E06C
:10C3D00044E0942ECCECD1E33EEDC32E3CE1D32ED1
:10C3E00024EFA22E21E0B22E023031F580E060E091
:10C3F0004FE727E001E00E94724581E060E043EDF5
:10C4000051E322E000E0EE240E94284782E090E021
:10C410000E940B53AC0180E067E020E00E94594786
:10C4200086E090E00E940B53AC018BE067E020E0D7
:10C430000E945947EDDA01E00E947B50013089F5F6
:10C44000812F63E0B6DE2DB73EB7275030403EBFA8
:10C450002DBFEDB7FEB73196ADB7BEB711961C92A2
:10C4600091821282D483C383D682C5820E94694C92
:10C470008091C11C90E02091C01C821B91094496C0
:10C480002DB73EB7295F3F4F3EBF2DBF8932910583
:10C4900038F480ED97E0F5013197F1F70197D9F77E
:10C4A000FF2480E20E9476B0882321F0812F682D3E
:10C4B000D4D630C080E10E9476B0882359F580E45C
:10C4C0000E9476B0882331F480E462E00E94A0B03C
:10C4D000882311F0FF24F39480E80E9476B088232B
:10C4E000B1F480E862E00E94A0B0882381F4FF20CC
:10C4F00029F0812F6F2DB1DE01E001C000E00E9424
:10C500001291882309F470CF0E945B436FCFFF2400
:10C51000FA94EFCFCDB7DEB7ECE00C94DEE9A1E002
:10C52000B0E0E5E9F2E60C94C6E97C016B018A0112
:10C530000E943BCB8091240F882311F4C60101C0D7
:10C54000C8010E946FCB80E00E946CCB4E2D5F2D06
:10C550008A0118C06E3F19F40E94D9CD13C0862FEE
:10C56000698334DA8091B41C69818F3F21F481E0C2
:10C5700041E092D91FC028D6882321F08091B41CB5
:10C580000E94B0CDF80161918F016F3F19F780E0F3
:10C590000E9403D20E9418CC853061F00E9430CCFA
:10C5A000082F14DAE091B51CF091B61C802F61E0E1
:10C5B0000995EDCF0E9462CB2196E8E00C94E2E968
:10C5C0000F931F93CF93DF93EB010E943BCBCE01E0
:10C5D0000E9488CB80E00E946CCB82E061E040E06A
:10C5E00050E02CE530E303E610E30E945ECD83E0EB
:10C5F00061E040E050E02BE630E309E710E30E9401
:10C600005ECD84E061E040E050E027E830E389015E
:10C610000E945ECD85E061E040E050E02DE830E32F
:10C6200089010E945ECD86E061E040E050E025E9AE
:10C6300030E30AE910E30E945ECD87E061E040E06C
:10C6400050E023EA30E30AEA10E30E945ECD88E07E
:10C6500061E040E050E021EB30E389010E945ECDD3
:10C6600089E061E040E050E02BEB30E304EC10E3C4
:10C670000E945ECD8AE061E040E050E02CEC30E3C7
:10C680000AED10E30E945ECD8BE061E040E050E0F7
:10C6900028EE30E389010E945ECD8CE061E040E04D
:10C6A00050E02DEE30E306EF10E30E945ECD8DE00A
:10C6B00061E040E050E02BEF30E308E011E30E943E
:10C6C0005ECD8FE061E040E050E023E131E389019D
:10C6D0000E945ECD80E00E9403D20E9418CC85307B
:10C6E00009F46AC00E9430CC90E002978E30910528
:10C6F00008F058C087599F4FFC010C94F3E98AE574
:10C7000092E06CE570E343E650E34AC08DE692E0C8
:10C710006BE670E349E750E343C086E792E067E8E1
:10C7200070E33DC08CE792E06DE870E338C087E8C5
:10C7300092E065E970E34AE950E332C08BE992E0A8
:10C7400063EA70E34AEA50E32BC081EB92E061EBCD
:10C7500070E325C087EC92E06BEB70E344EC50E3B0
:10C760001FC088ED92E06CEC70E34AED50E318C016
:10C770008FEE92E068EE70E312C080E093E06DEE21
:10C7800070E346EF50E30CC089E093E06BEF70E399
:10C7900048E051E305C08EE093E063E171E3AB0153
:10C7A000BEDE98CF8EE191E360E048EC50E021E0FE
:10C7B00001E00E94F6918ECF0E9462CBDF91CF9173
:10C7C0001F910F910895AF92BF92DF92EF92FF9267
:10C7D0000F931F93CF93DF93D82E7B01CED5C82F15
:10C7E000D0E02196CE010E94F9E98C01009751F426
:10C7F00084E590E361E040E253E021E001E00E9443
:10C80000F6911DC06091730B7091740BAE010E9484
:10C81000D8EC8D2DB701D4DE6091730B7091740B41
:10C82000C801AE010E94CBECE82EE7015E01B92EF3
:10C83000E501C8010E9493EA81E0209709F480E0B5
:10C84000DF91CF911F910F91FF90EF90DF90BF90FC
:10C85000AF90089583E0EEE5FDE1DF011D928A953A
:10C86000E9F78CE49DE16BE173E00C94FCEC8091C2
:10C870005F1D9091601D009711F00E9493EAEACF2E
:10C88000FF920F931F93182F062F77D5F82E409104
:10C890005F1D5091601D4115510551F4482F50E026
:10C8A000CA0101960E94F9E980935F1D9093601D73
:10C8B00040915F1D5091601D4115510559F489E764
:10C8C00090E461E040E253E021E001E00E94F69153
:10C8D00080E01FC02F2D30E06091730B7091740BBE
:10C8E000163061F48091A21C80935E1D2F5F3F4F34
:10C8F000CA01A9010E94D8EC86E00BC02F5F3F4F10
:10C90000CB01BA01A9010E94D8EC812F602F0E94AF
:10C91000F9541F910F91FF900895A0E0B0E0E3E972
:10C92000F4E60C94C7E902EF1CE1C0E0D0E090E12E
:10C93000D92E8AE2E82E83E0F82E9E012F5F822F07
:10C9400064E10E949754882309F456C021968BE62F
:10C9500043D4ADB7BEB71997BEBFADBFEDB7FEB7F5
:10C96000319612961C930E931197D282F482E38231
:10C97000D683C583908787830E941BD80E5E1F4F86
:10C980002DB73EB7275F3F4F3EBF2DBFC530D10506
:10C99000A1F680915F1D9091601D009741F130914B
:10C9A0005E1D2091A21C321711F061DF20C098D4C7
:10C9B0008BE612D4ADB7BEB71797BEBFADBFEDB70C
:10C9C000FEB731962CE43DE112963C932E931197DD
:10C9D000D28222E333E034832383968385830E94CB
:10C9E0001BD82DB73EB7295F3F4F3EBF2DBF8FEFFE
:10C9F00064E10E94975401C080E0CDB7DEB7E7E064
:10CA00000C94E3E91F93182F0E943BCB80E00E9417
:10CA10006CCB81E00E94A0CB212F30E02150304030
:10CA2000220F331FC90143E0880F991F4A95E1F790
:10CA3000820F931F8E50934E0E9488CB8EEFC4D3EB
:10CA4000882359F48AEF90E00E940B539C0184E103
:10CA500061E040E050E00E947ECD163059F081E860
:10CA600090E00E940B539C0185E161E040E050E0C2
:10CA70000E947ECD85E190E00E940B539C0186E1EF
:10CA800061E040E050E00E947ECD80E00E9403D251
:10CA90000E9418CC853021F00E9430CC182F01C0A4
:10CAA00010E00E9462CB81E00E946CCB812F1F912D
:10CAB00008951F93182F0E943BCB80E00E946CCBFF
:10CAC00081E00E94A0CB212F30E021503040220F86
:10CAD000331FC90163E0880F991F6A95E1F7820F40
:10CAE000931F8E50934E0E9488CB82E190E00E946B
:10CAF0000B539C018EE161E040E050E00E947ECD4E
:10CB000084E190E00E940B539C018FE161E040E0E2
:10CB100050E00E947ECD80E00E9403D20E9418CC9B
:10CB2000853021F00E9430CC182F01C010E00E9407
:10CB300062CB81E00E946CCB812F1F910895A0E011
:10CB4000B0E0E5EAF5E60C94C1E9C82E0E945B432B
:10CB50008C2D90E00197880F991FEC01E3E0CC0F3A
:10CB6000DD1FEA95E1F7C80FD91FCE50D34E1C2D1B
:10CB7000DD24FF24F39475E0972E63E0862E54E7BE
:10CB8000A52E50E4B52E44E0742EFF2009F480C099
:10CB900080E060E04FE727E001E00E94724585E811
:10CBA00090E00E940B53AC0181E060E022E00E9423
:10CBB00059478BEF90E00E940B53AC0180E062E09C
:10CBC00020E000E0EE24EA940E9428478DB79EB74B
:10CBD00009979EBF8DBFEDB7FEB73196ADB7BEB713
:10CBE00011969C9282E08183128283828FEF8483EC
:10CBF000B682A582D087C7830E94464C8DB79EB768
:10CC000009969EBF8DBF8EE169E14AE527E00E944B
:10CC100072458CEF90E00E940B53AC0180E064E021
:10CC200020E039EFE32E0E942847ADB7BEB7199731
:10CC3000BEBFADBFEDB7FEB7319611969C92718223
:10CC40001282838289EF8483B682A582812F90E04D
:10CC50000197880F991F9C01B3E0220F331FBA95EB
:10CC6000E1F7280F391F2E50334E308727830E945B
:10CC7000464C8DB79EB709969EBF8DBF82E090E06F
:10CC80000E940B53AC0180E067E020E00E9459470E
:10CC900080E20E9476B0882309F0B4C080E40E944C
:10CCA00076B0882321F0163021F01F5F03C0FF24E7
:10CCB00003C011E0FF24F39480E80E9476B088233B
:10CCC00039F0113011F0115001C016E0FF24F39437
:10CCD00080E10E9476B0882309F48CC088E890E057
:10CCE0000E940B53BC0185E040E020E001E00E947F
:10CCF000374780E065E24FE72EE0A2E0EA2E0E948F
:10CD0000924880E068E34FE727E000E00E94724528
:10CD100086E290E00E940B53AC018CE067E020E0DB
:10CD20000E94594789E190E06FEF7FEF40E00E9459
:10CD3000B7B080E10E9476B0882311F004E001C012
:10CD400000E080E20E9476B0811105E00E9412911D
:10CD5000002379F3043009F047C09C2D9630A1F0F0
:10CD60008C2D64E10E949754D82E8C1569F087EFC2
:10CD700090E00E940B5361E040E253E021E001E0CB
:10CD80000E94F691DD2440C0163021F486E06AE06E
:10CD900077DD3AC080E060E240E820E200E00E94F7
:10CDA000724583E190E00E940B53BC0184E040E0B7
:10CDB00020E009E00E94374780E065E24FE72EE07F
:10CDC00001E0F2E0EF2E0E949248AC2DA63021F453
:10CDD000812F6EE155DD06C0163060F4812F6EE1C3
:10CDE0000E94F954D82E10C0053021F40E945B43F4
:10CDF000FF24F3940E941291882309F4C6CE0E9466
:10CE00005B43C6CEE3E6DE2E8D2DCDB7DEB7EDE07B
:10CE10000C94DDE9EF92FF920F931F9388EF90E05F
:10CE20000E940B5360E040E050E021E001E00E94EE
:10CE3000F69173DD182F882359F487EF90E00E9454
:10CE40000B5361E040E253E021E00E94F691CFC035
:10CE50000E943BCB88E690E40E946FCB20E002E189
:10CE60000EC0F22EF394209F900111242E50334EC9
:10CE70008F2D62E040E050E00E9497CD2F2D822F51
:10CE800090E040915F1D5091601D4115510519F0D2
:10CE900046E050E002C045E050E0841795070CF3EF
:10CEA000812F0E9458CC812F61E00E949ECC80E0AF
:10CEB0000E9403D20E9418CC853009F496C00E94CB
:10CEC00030CC182F8150863090F7812F9BDD843134
:10CED00009F048C0812F69E10E949754812F90E0AA
:10CEE0000197880F991FBC01B3E0660F771FBA95B1
:10CEF000E1F7680F791F6E50734E812F64DC882331
:10CF0000B1F21630A1F2812FD4DD8E3181F680E0AE
:10CF100068E340E827E000E00E94724583E190E08A
:10CF20000E940B53BC0184E040E020E009E00E9435
:10CF3000374780E065E24FE72EE001E0A2E0EA2E0D
:10CF40000E949248812F62E30E94F954882309F0DD
:10CF5000AECF87EF90E00E940B5361E040E253E0D8
:10CF600021E01CC0853139F589EF90E00E940B5318
:10CF700060E040E050E021E001E00E94F691812F66
:10CF80000E947555082F882361F487EF90E00E9476
:10CF90000B5361E040E253E021E001E00E94F69192
:10CFA00086CF11E0812F60E00E949ECC1F5F16307B
:10CFB000C9F7802F79CF863109F079CF812FBFDD76
:10CFC000882361F487EF90E00E940B5361E040E218
:10CFD00053E021E001E00E94F69103C0833609F49A
:10CFE00066CF0E9462CB81E003C00E9462CB80E0EA
:10CFF0001F910F91FF90EF9008950F931F93109141
:10D00000DF06113009F045C00E94E5C98DB79EB713
:10D0100007979EBF8DBFEDB7FEB731968FE6ADB7D0
:10D02000BEB711968C9382E0818312838AE090E0F0
:10D030009483838381E090E0968385830E9496C8E1
:10D040008FE48093DE061092710B88EC90E0909351
:10D05000331E8093321E8DB79EB707969EBF8DBF3D
:10D060008091710B882331F48091321E9091331E90
:10D070000097B1F78091710B882379F00E948AC9DB
:10D08000E091730BF091740BED5BFF4F808180FD9D
:10D0900004C0C0DE8130E9F30BC089E190E00E945A
:10D0A0000B5360E040E951E021E001E00E94F6917D
:10D0B0001F910F910895CF93DF93DB01EA011C923A
:10D0C0001882F90110824DEE54E4FA0194919817F8
:10D0D00009F534968491FA013596E491882321F07C
:10D0E0009091A21C9817D8F4EE2321F08091A21CF5
:10D0F000E817A8F4FA013196E491EC93FA0132961C
:10D10000E491E8834D5F5F4FFA014491F901408358
:10D1100081E006C09F3F19F04A5F5F4FD6CF80E0A5
:10D12000DF91CF910895A1E0B0E0E9E9F8E60C9431
:10D13000CBE98983162FFA011082F90110828091C0
:10D14000A11C882321F18981982F905A9F3548F49A
:10D15000BE016F5F7F4FAFDF882319F41123E1F029
:10D160001EC02091611D3091621D498190E0F9013E
:10D17000549131968491541731F05F3F31F0980FFC
:10D180002E5F3F4FF4CF4F3F21F44F3F11F080E02F
:10D190009FEF112319F003C08FEF01C0892F219653
:10D1A000E3E00C94E7E9A2E0B0E0E9EDF8E60C94E6
:10D1B000CCE9AE014F5F5F4F9E012E5F3F4FB3DF63
:10D1C0002296E2E00C94E8E961E0EDDF91E088234B
:10D1D00009F490E0892F089560E0E5DF8F3F39F092
:10D1E0002091631D3091641D280F311D02C020E085
:10D1F00030E0C9010895A2E0B0E0E1E0F9E60C9466
:10D20000CCE960E0AE014F5F5F4F9E012E5F3F4F64
:10D210008ADF8F3FE9F0E091631DF091641DE80F14
:10D22000F11D80819981913029F49A81982381E0C0
:10D2300081F40EC0923029F49A81982381E049F05C
:10D2400007C0933031F48A81E80FF11D808101C05D
:10D2500080E02296E2E00C94E8E9A2E0B0E0E3E3AB
:10D26000F9E60C94CBE9162F60E0AE014F5F5F4FFB
:10D270009E012E5F3F4F57DF8F3F69F12981922F2B
:10D2800091509230B0F4E091631DF091641DE80F6D
:10D29000F11D9081223021F481E0111180E0182FDE
:10D2A0008A81112311F0892B02C080958923808304
:10D2B00010C090E0E091631DF091641D233031F4C3
:10D2C0002A81E80FF91FE20FF11D02C0E80FF91FD4
:10D2D000108381E001C080E02296E3E00C94E7E94E
:10D2E0001092621D1092611D1092641D1092631DB8
:10D2F0001092A11C1092A21C1092A31C1092A41CAC
:10D300000097B9F1DC012D912093A31CFC01218130
:10D310002093A21C30E0832F90E0FC01EE0FFF1F52
:10D32000E80FF91FE65CFC4F8081821721F08F3FE8
:10D3300001F13F5FF0CF2F3FF1F0B093641DA09358
:10D34000631D818192819093621D8093611D81E0B4
:10D350008093A11C8BE640DF009741F0A4EABCE17A
:10D36000FC018CE001900D928150E1F78091A11CAD
:10D37000089580E0089580E008958091A11C88239D
:10D3800019F08FEF60E00FCF80E00895AAE8BFE1C9
:10D3900090E1FD0111929A95E9F7882339F4CD01C6
:10D3A00070E040E150E00E94E1EC05C0E82FF0E0C1
:10D3B000E757F04E60838DB79EB707979EBF8DBF2E
:10D3C000EDB7FEB7319684E7ADB7BEB711968C9333
:10D3D00081E0818382838AE89FE19483838380E173
:10D3E00090E0968385830E9496C8EDB7FEB7379686
:10D3F000FEBFEDBF0895EF920F931F93CF93DF937E
:10D40000182F0E945B4381E08093661D8093681D06
:10D410001092671D0E945B4381E496E462E00E94E3
:10D42000624782E062E046E356E420E00E9459470A
:10D4300082E063E04BE256E420E00E94594788E036
:10D4400068E240E026E001E00E94724583E090E05F
:10D450000E940B53AC0180E067E020E00E94594736
:10D4600082E167E047E256E420E00E94594780E00D
:10D4700062E045E256E420E00E945947123051F440
:10D480008091DF06813031F48091E006813011F423
:10D490000E940ECACFEFD0E08091661D882369F507
:10D4A00080E40E9476B0882331F480E463E00E9437
:10D4B000A0B0882311F14091671D4E3FF0F44F5FFB
:10D4C0004093671D89E063E050E023E030E000E036
:10D4D000EE240E943C4D123081F48091671D20E7BC
:10D4E000829FC0011124BE010E946CE9462F88E092
:10D4F00068E226E001E00E9472458091661D882363
:10D5000009F040C080E80E9476B0882331F480E8BA
:10D5100063E00E94A0B08823A9F18091671D882351
:10D5200089F1123079F420E7829FC0011124BE01F5
:10D530000E946CE9862F885F68E240E026E000E008
:10D540000E9472454091671D41504093671D89E0DC
:10D5500063E050E023E030E000E0EE240E943C4D28
:10D56000123081F48091671D20E7829FC001112451
:10D57000BE010E946CE9462F88E068E226E001E0E7
:10D580000E9472458091661D8130D9F480E40E942A
:10D5900076B0882331F480E461E00E94A0B0882353
:10D5A00081F04091681D403160F44F5F4093681DE9
:10D5B00089E062E050E023E030E000E0EE240E94E9
:10D5C0003C4D8091661D813041F580E80E9476B027
:10D5D000882331F480E861E00E94A0B08823E9F05C
:10D5E0004091681D4423C9F041504093681D442375
:10D5F00049F089E062E050E023E030E000E0EE2412
:10D600000E943C4D8091681D882339F489E062E0D6
:10D6100041E256E420E00E94594780E10E9476B042
:10D62000882329F18091661D882389F462E04FE107
:10D6300056E420E00E94594780E063E04DE156E463
:10D6400020E00E94594781E08093661D10C080E071
:10D6500062E04BE156E420E00E94594780E063E03D
:10D6600049E156E420E00E9459471092661D8091DE
:10D67000681D6091671D8ADE80E20E9476B0882373
:10D6800009F40ACF80EF0E9476B0123019F480E0DE
:10D6900060E07CDEDF91CF911F910F91EF900895B4
:10D6A00008951092911D1092921D08951F93CF938B
:10D6B000DF93EA011091921D1F30B0F58823E1F04D
:10D6C00021E030E002C0220F331F8A95E2F7C90142
:10D6D000AA2797FDA095BA2F2091F70F3091F80F48
:10D6E0004091F90F5091FA0F82239323A423B5237D
:10D6F0000097A105B105C1F0E12FF0E0DF01AA0F0D
:10D70000BB1FAA0FBB1FAF56B24E13967C936E93EE
:10D710001297EE0FFF1FEE0FFF1FEB56F24ED18355
:10D72000C0831F5F1093921DDF91CF911F910895C9
:10D730001092911D9091921D891710F48093911D64
:10D7400008958091911D8F5F8093911D9091921DFE
:10D75000891710F01092911D81E08093D01D0895DB
:10D760008091911D882311F48091921D81508093A6
:10D77000911D81E08093D01D0895E091911DF0E00E
:10D78000EE0FFF1FEE0FFF1FEB56F24E0190F081E0
:10D79000E02D09950895FC011082118212821382F6
:10D7A00020E021C0822F90E0DC01AA0FBB1FA80F50
:10D7B000B91FAA0FBB1FA25DBB4E3C91418143170D
:10D7C00010F431832083DC01AA0FBB1FA80FB91FFF
:10D7D000AA0FBB1FAF5CBB4E8C919381981710F4BE
:10D7E000838322832F5F80912B142817D8F208950A
:10D7F000EF920F93DF93CF9300D000D0CDB7DEB779
:10D80000CE010196C8DF81E990E00E940B53AC0184
:10D8100080E060E020E00E94594760910B14709115
:10D820000C14882777FD8095982F0E9458E720E0F8
:10D8300030E040EA51E40E94BDE60E9425E79B01EA
:10D84000AC018EE060E0A90124E030E000E0EE24CD
:10D850000E947E4D82E160E04DE620E002E00E9401
:10D86000A74582E990E00E940B53AC0180E061E0A3
:10D8700020E00E945947209111143091121440E089
:10D8800050E0CA01B901E3E0660F771F881F991FB6
:10D89000EA95D1F7620F731F841F951F2AEF30E0BE
:10D8A00040E050E00E947FE98FE061E0A90123E0C1
:10D8B00030E000E00E943C4D82E161E04EE457E43C
:10D8C00020E002E00E94284783E990E00E940B5389
:10D8D000AC0180E062E020E00E945947809117147B
:10D8E000909118146AE070E00E9458E9AB018EE054
:10D8F00062E024E030E000E00E943C4D82E162E022
:10D900004DE620E002E00E94A74584E990E00E94F5
:10D910000B53AC0180E063E020E00E945947409146
:10D9200029144F3F41F48EE063E049E457E420E0DE
:10D930000E94594709C08EE063E050E023E030E0E8
:10D9400000E0EE240E94C24D82E163E046E520E063
:10D9500002E0EE240E94A74587E990E00E940B5365
:10D96000AC0180E064E020E00E945947409123141C
:10D97000509124148EE064E024E030E000E00E9446
:10D980003C4D82E164E045E457E420E002E00E947F
:10D99000284786E990E00E940B53AC0180E065E0E7
:10D9A00020E00E94594740911B1450911C148DE0B7
:10D9B00065E024E030E000E00E94C24D82E165E0D5
:10D9C00041E420E002E00E94A74580E066E047E3F2
:10D9D00057E420E00E945947498150E04F5F5F4F74
:10D9E00086E066E021E030E000E00E943C4D4A81A4
:10D9F0008EE066E050E023E030E00E94C24D82E11C
:10DA000066E041E420E002E00E94A74580E067E094
:10DA100049E257E420E00E9459474B8150E04F5FB4
:10DA20005F4F86E067E021E030E000E00E943C4D7F
:10DA30004C818EE067E050E024E030E00E943C4DF5
:10DA400082E167E046E257E420E002E00E942847D6
:10DA50002496DEBFCDBFCF91DF910F91EF90089557
:10DA6000A1E0B0E0E6E3FDE60C94C9E9F82EFF0C76
:10DA7000FF0CFF0C9FE39F19692F685080E04FE770
:10DA800023E000E099830E9472459981192F145078
:10DA90002F2D2C5F80E0612F4FE701E00E9472453F
:10DAA00080E0612F40E00E94CC438FE7612F40E08F
:10DAB0000E94CC439981935081E0612F40E0292F4F
:10DAC00000E099830E94DA448EE7612F4FE7998145
:10DAD000292F0E94DA442196E5E00C94E5E989E6D5
:10DAE000E3EFF3E1DF011D928A95E9F78FEF809371
:10DAF0002914809320148EE7809326148093281491
:10DB0000089584E591E0E6E5F5E1DF019C011D92D1
:10DB100021503040E1F70895A2E0B0E0E2E9FDE6EF
:10DB20000C94CCE9813089F58A830E94E5C9198279
:10DB30002DB73EB7275030403EBF2DBFEDB7FEB7E3
:10DB4000319694E6ADB7BEB711969C9311828A8147
:10DB50008283CE0101969483838381E090E0968353
:10DB600085830E9496C883E090E09093331E809353
:10DB7000321E2DB73EB7295F3F4F3EBF2DBF80916C
:10DB8000321E9091331E0097D1F78AE089838DB7BA
:10DB90009EB707979EBF8DBFEDB7FEB731968FE654
:10DBA000ADB7BEB711968C9382E0818381E082830A
:10DBB000CE0101969483838381E090E096838583F0
:10DBC0000E9496C883E090E09093331E8093321EAB
:10DBD0002DB73EB7295F3F4F3EBF2DBF8091321E0C
:10DBE0009091331E0097D1F787E089838DB79EB758
:10DBF00007979EBF8DBFEDB7FEB731968BE6ADB7E9
:10DC0000BEB711968C93118281E08283CE0101967A
:10DC10009483838381E090E0968385830E9496C8F5
:10DC20008FE48093DE0688EC90E09093351E80931D
:10DC3000341E1092710B2DB73EB7295F3F4F3EBF88
:10DC40002DBF2296E2E00C94E8E9A2E0B0E0EBE21E
:10DC5000FEE60C94C6E994E59093DE0691E0998384
:10DC60002DB73EB7275030403EBF2DBFEDB7FEB7B2
:10DC7000319624E7ADB7BEB711962C9322E02183ED
:10DC800092839E012F5F3F4F3483238321E030E056
:10DC9000368325838A830E9496C81092710B8A81ED
:10DCA00090E09093331E8093321EEDB7FEB7379607
:10DCB000FEBFEDBF8091321E9091331E0097D1F7C9
:10DCC0008091710B882309F44BC00E948AC900918E
:10DCD000730B1091740BD8018D919C911197815DFC
:10DCE0009740873C910508F03DC0F894F8016481A5
:10DCF00070E080E090E020E13EE040E050E00E94F3
:10DD00002DE96B017C01D80115966C91159770E097
:10DD100080E090E02CE330E040E050E00E942DE90C
:10DD2000C60ED71EE81EF91EF8018681C80ED11C4A
:10DD3000E11CF11CC092361ED092371EE092381EB4
:10DD4000F092391E838180933A1E828180933B1E1C
:10DD50008081918190933D1E80933C1E789402C0F7
:10DD600080E001C081E090E02296E8E00C94E2E9D6
:10DD7000A0E0B0E0EEEBFEE60C94BEE9E091EC1D15
:10DD8000F091ED1DED5BFF4FD0808091401E909192
:10DD9000411E009751F50091971C1091981C2091FD
:10DDA000991C30919A1C40919B1C50919C1C609135
:10DDB0009D1C70919E1C80919F1C9091A01CEE2434
:10DDC000FEE1CF2EE7E6AE2E0E943B53823068F094
:10DDD00084E13BDF009719F482E390E002C080E722
:10DDE00097E19093411E8093401E8091491E90912F
:10DDF0004A1E009709F0ACC08BE48093DE061092B7
:10DE0000710B84E190E09093331E8093321EAD2C11
:10DE1000BB2481E0A822BB2490C08091710B882391
:10DE200009F48BC00E948AC9A091730BB091740B46
:10DE3000DC909D2D983008F07EC085E0989FF00121
:10DE40001124E759F24E0D9001928150E1F70D2D0A
:10DE500010E0F801EE0FFF1FEE0FFF1FE00FF11FA4
:10DE6000E759F24E8481807F09F465C0A114B104A2
:10DE700009F461C0E801CC0FDD1FC00FD11FCC0F2A
:10DE8000DD1FCF5DD04FDE01A55FBA4FED90FC9056
:10DE900011970894E11CF11CED92FC929EE0492E32
:10DEA00095E0592E4C0E5D1ED2016D907C9011971D
:10DEB00088249924C1806C2D70E080E090E024E6F5
:10DEC00030E040E050E00E942DE9661977098809AA
:10DED0009909970140E050E00E94A1E9260D371D05
:10DEE000481D591DF20131832083C35FDA4F8881B9
:10DEF0008C1508F4C882F801EE0FFF1FEE0FFF1F0C
:10DF0000E00FF11FE759F24E8281F801EE0FFF1F7B
:10DF1000E00FF11FEE0FFF1FEF5CFB4E9081981793
:10DF200008F4808380912B1490E0081719071CF0E7
:10DF3000D394D0922B141092710B8091321E909139
:10DF4000331E009709F069CF10924A1E1092491EA5
:10DF50008FE48093DE061092710B8CE291E0909337
:10DF6000331E8093321ECDB7DEB7E0E10C94DAE9C0
:10DF7000E091EC1DF091ED1DDF01AD5BBF4F8C9189
:10DF800080FF6AC0DF01A65BBF4F8C9181FF64C038
:10DF900085A996A997FF29C01092E8068091EA0604
:10DFA0008F5F8093EA069091E906992399F4909106
:10DFB0006303891778F080919D0F882339F48CE2F0
:10DFC00091E06FEF7FEF40E00E94B7B08091630374
:10DFD0008093EA068091E9068F5F8093E90690912D
:10DFE0006203891711F41092E906E091EC1DF0919B
:10DFF000ED1D85A996A9009719F41092EA060895D7
:10E00000181619064CF51092E9068091EA068F5F02
:10E010008093EA069091E806992399F4909163031E
:10E02000891778F080919D0F882339F484E690E079
:10E030006FEF7FEF40E00E94B7B080916303809361
:10E04000EA068091E8068F5F8093E806909161036D
:10E05000891711F41092E80608955091220F523357
:10E0600030F56091F006633020F582E08093EE0693
:10E07000E091EC1DF091ED1D42E07BE20BC0A42F7E
:10E08000AF5F21AD30E0479FC00111242817390749
:10E090001CF04A2F473098F34093EE06459F402DE1
:10E0A00011244093EF066F5F6093F00602C0509317
:10E0B000EF06E091EC1DF091ED1D91AD8091EF0622
:10E0C0009817A0F48091F106853020F48F5F80933B
:10E0D000F1060895ED5BFF4F808180FF07C088EE59
:10E0E00093E060E270E041E00C94B7B00895CF9304
:10E0F000DF93C091EC1DD091ED1D8EAD9FADE8E694
:10E10000F1E0BF010E946CE99C018EA59FA5BF01B3
:10E110000E946CE9281B390B37FF02C028593E4F7B
:10E120003093EF1D2093EE1DDF91CF9108959C0158
:10E13000285130402C32310528F19C0124543040C4
:10E140002D32310508F19C01215730402D32310527
:10E15000E8F09C012E5930402D323105C8F09C0169
:10E160002B5C30402D323105A8F09C01285F3040F7
:10E170002D32310588F0855291408D32910570F431
:10E1800086E0089580E0089581E0089582E0089592
:10E1900083E0089584E0089585E0089587E0089578
:10E1A000A0E0B0E0E6EDF0E70C94C4E9382FF62EDD
:10E1B000CA01D22E102F66E170E00E9458E96D5E10
:10E1C00070E0EB012497A5E0AA2EB12CA60EB71E95
:10E1D00001C03C2DC32EC394FE01E755F94B449179
:10E1E000832F6F2D20E00D2DE12E0E94A745219653
:10E1F000CA15DB0571F7CDB7DEB7EAE00C94E0E9AC
:10E20000A0E0B0E0E6E0F1E70C94C5E9F82EE62ED8
:10E21000D42EC22EE801822F8695B62EB81A8F2DE5
:10E220006B2D01E00E9454481F2D1F5F6B2D6F5F07
:10E230004D2D42502C2D2250812F00E00E9472451E
:10E240004D2D4F0D8F2D6E2D2E2D01E00E94DA44A5
:10E250001C161D060CF04FC0CE0165E070E00E9458
:10E260006CE9FB016130710569F062307105B9F04C
:10E270002E2D21508F2D8C5F4F2D4A5F309721F529
:10E28000622F52C02E2D21504F2D4A5F8F2D8C5F53
:10E29000622F01E00E94DA446E2D635054C02E2D8F
:10E2A00021504F2D4A5F8F2D8C5F622F01E00E941D
:10E2B000DA446E2D63508F2D8D5F44E021E00E9483
:10E2C00072456E2D655057C0622F01E00E94DA44FE
:10E2D0006E2D63508F2D8D5F44E021E00E947245CA
:10E2E0006E2D65508F2D8E5F46E021E00E947245B5
:10E2F0006E2D66505AC0209709F45CC0CE016BEFBA
:10E300007FEF0E946CE9FB016130710581F06230A2
:10E310007105E9F08F2D8C5F4F2D4A5F2E2D2F5FF9
:10E32000309769F5622F01E00E94DA4443C02E2D38
:10E330002F5F4F2D4A5F8F2D8C5F622F01E00E946F
:10E34000DA446E2D6E5F8F2D8D5F44E030C02E2D30
:10E350002F5F4F2D4A5F8F2D8C5F622F01E00E944F
:10E36000DA446E2D6E5F8F2D8D5F44E021E00E94B8
:10E3700072456E2D6C5F8F2D8E5F46E018C0622F48
:10E3800001E00E94DA446E2D6E5F8F2D8D5F44E0B8
:10E3900021E00E9472456E2D6C5F8F2D8E5F46E0EE
:10E3A00021E00E9472456E2D6B5F812F48E021E0D5
:10E3B0000E947245CDB7DEB7E9E00C94E1E98F9297
:10E3C0009F92AF92BF92CF92DF92EF92FF920F9304
:10E3D0001F93F62E182F110F180F110FFF0CFF0CA3
:10E3E000FF0C47E0A42EAF0C33E0932E9F0C812F3F
:10E3F000692D41E00E94CC4326E0B22EBF0CD12E05
:10E40000D39492E0892E8F0C8D2D6B2D4D2D282DC0
:10E4100001E00E94DA44EF2CE394812F8E5F6E2D91
:10E4200041E00E94CC4383E0C82EC10E8C2D6F2D9D
:10E4300041E00E94CC43812F8C5F6E2D41E00E9411
:10E44000CC43B5E0EB2EE10E8E2D6B2D4E2D282DFD
:10E450000E94DA44812F8A5F692D41E00E94CC43FB
:10E460008C2D6B2D41E00E94CC436F2D6B5F8C2D6A
:10E4700041E00E94CC438D2D6A2D4E2D2A2D0E9405
:10E48000DA441F910F91FF90EF90DF90CF90BF90F3
:10E49000AF909F908F900895A0E0B0E0E2E5F2E7A2
:10E4A0000C94C6E9F62E182F110F180F110FFF0C40
:10E4B000FF0CFF0C57E0E52EEF0CC12FD0E02396A8
:10E4C000CE2CDD248DEF9FEFC80ED91ECE01B601F4
:10E4D00044E050E021E00E940A492F2D2C5F412F9B
:10E4E0004A5F812F622F01E00E94DA44412F4D5F85
:10E4F0002F2D2F5F842F6E2D0E94DA44CE01B6019E
:10E5000042E050E021E00E940A49CDB7DEB7E8E0E2
:10E510000C94E2E98F929F92AF92BF92CF92DF92DA
:10E52000EF92FF920F931F93982E862ECA01B90186
:10E53000D02EBE2CAC2C0E9458E77B018C0120E031
:10E5400030E048E453E40E9441E8181654F0C80152
:10E55000B70120E030E048E453EC0E94B6E687FFC4
:10E5600017C0C801B70120E030E040EA51E40E9442
:10E57000BDE60E9425E79B01AC01892D682DA9010C
:10E5800024E030E000E0ED2CCB2C0E94484D16C07A
:10E59000C801B70120E030E040E05FE30E9445E8B9
:10E5A0000E9425E79B01AC01892D682DA90123E07C
:10E5B00030E000E0ED2CCB2C0E94064E1F910F9115
:10E5C000FF90EF90DF90CF90BF90AF909F908F9093
:10E5D000089529E936E1D901F901719791E1019096
:10E5E0000D929150E1F72151304095E126353907E0
:10E5F00091F780935615D9011196E6E3FEE188E084
:10E6000001900D928150E1F70895CF92EF920F9310
:10E610008CE790E00E940B53AC0180E060E022E0C8
:10E620000E9459478DE790E00E940B53AC0180E0B7
:10E6300062E020E00E9459478EE790E00E940B5371
:10E64000AC0180E063E020E00E9459478AE090E05E
:10E650000E940B53AC0180E065E020E00E94594726
:10E660002091820F3091830F4091840F5091850F3C
:10E6700081E066E000E0EE24CC240E94FD4E209173
:10E680007E0F30917F0F4091800F5091810F8CE071
:10E6900066E00E94FD4E0F91EF90CF9008951F937A
:10E6A000182F2CE231E03093331E2093321E10924B
:10E6B000DE068091EB1D883229F088E28ADF88E24D
:10E6C0008093EB1D112371F080E090E060E070E03A
:10E6D00042E00E94B7B00E945B438AEF90E060E4A2
:10E6E00070E008C080918B0F813039F488EC90E0A5
:10E6F00060E870E040E00E94B7B087DF81E00CDAAC
:10E700001F910895EF92FF920F931F93CF93DF9382
:10E71000EC01FB01122FCA01880F991F840F951F6E
:10E72000880F991F62E070E00E946CE99B012296BD
:10E73000BE01660F771F6C0F7D1F660F771FA3E06A
:10E74000EE0FFF1FAA95E1F76E5F7F4F802F99278D
:10E7500087FD90953B96FF24E7FCF094EE0DFF1D9E
:10E76000A9014250504025503040860F971FBF01ED
:10E77000012F0E94494ACDB7DEB7E6E00C94E4E9E8
:10E78000AF92CF92EF920F931F93CF93DF93FB0142
:10E79000D901202F0296EC01CC0FDD1FC80FD91F25
:10E7A000CC0FDD1F53E0EE0FFF1F5A95E1F7842FCA
:10E7B000880F840F880F63E00E944CE9280F22968F
:10E7C0003B96AE0EAE014C0D842F6A2D422F8D016B
:10E7D0000E94EB49DF91CF911F910F91EF90CF9065
:10E7E000AF900895DF92EF92FF920F931F93182F2F
:10E7F000F62EF5E0EF2EE60E6E2D4AE028E001E061
:10E800000E945448E5E0DE2ED10E8D2D6F2D412F54
:10E810002E2D0E94DA44412F465F8D2D6F2D2E2D17
:10E820000E94DA446F2D665F812F8C5F42E023E007
:10E830000E9454481F910F91FF90EF90DF90089530
:10E84000CF92DF92EF92FF920F931F93182FF62E25
:10E8500092E0E92EE60E6E2D44E022E001E00E94F7
:10E860005448812F885F6E2D44E022E00E94544876
:10E87000812F8C5F6F2D44E026E00E94544886E093
:10E88000C82EC10EB7E0DB2EDF0CABE0EA2EEF0C9A
:10E89000412F4E5F8C2D6D2D2E2D0E94DA44412F7D
:10E8A000465F8C2D6D2D2E2D0E94DA442F2D245F76
:10E8B000412F455F812F8F5F622F0E94DA441F91A5
:10E8C0000F91FF90EF90DF90CF900895FF920F93FC
:10E8D0001F93182FF62E8E5F42E022E001E00E9487
:10E8E00054486F2D6E5F812F46E02FE00E94544800
:10E8F0001F910F91FF900895EF92FF920F931F9336
:10E90000062F182F110F180F110F000F000F000FF7
:10E91000F02EF394E12EE394602F6B5F812F8C5FD8
:10E9200041E00E94CC43202F2D5F412F4B5F812F70
:10E930008D5F622F01E00E94DA44412F4A5F8E2DE5
:10E940008F5F6F2D2F2D0E94DA441F910F91FF9042
:10E95000EF900895ACE2B0E0E0EBF4E70C94C6E988
:10E96000F82ED62EC42E322F102F87E098E49A83EB
:10E97000898384E098E49C838B8381E098E49E8380
:10E980008D838EEF97E498878F838BEF97E49A8738
:10E99000898788EF97E49C878B8785EF97E49E872C
:10E9A0008D8782EF97E4988B8F878FEE97E49A8B11
:10E9B000898B8CEE97E49C8B8B8B89EE97E49E8BF6
:10E9C0008D8B86EE97E4988F8F8B83EE97E49A8FEA
:10E9D000898F80EE97E49C8F8B8F8DED97E49E8FCF
:10E9E0008D8F8AED97E498A38F8F87ED97E49AA394
:10E9F00089A384ED97E49CA38BA381ED97E49EA368
:10EA00008DA38EEC97E498A78FA38BEC97E49AA73D
:10EA100089A788EC97E49CA78BA7662331F0660F43
:10EA2000660F660F615028E002C027E060E0FF201B
:10EA300039F08F2D880F8F0D880F82504EE002C065
:10EA40004CE080E0810F6E0D332391F001E00E94D5
:10EA50007245EC2DF0E0EE0FFF1FEC0FFD1F418122
:10EA600052818F2D6D2D22E0012F0E94284703C077
:10EA700000E00E947245AC96E8E00C94E2E9EF9267
:10EA80000F93922FE02EE42FF0E0E631F10508F02D
:10EA90005FC0E958FF4FA091EC1DB091ED1D0C94A3
:10EAA000F3E9A65BBF4F02C0AC5BBF4F2C91227055
:10EAB00050C0AC5BBF4F0EC0A65BBF4F13C0A65B80
:10EAC000BF4F34C0A65BBF4F36C0AD5BBF4F38C031
:10EAD000AD5BBF4F2C9124703CC0AD5BBF4F26C0D7
:10EAE000AD5BBF4F2C91217034C0AD5BBF4FDECF0B
:10EAF000AD5BBF4F20C0A65BBF4FECCFAC5BBF4F41
:10EB00000DC0AC5BBF4F2C912095221F2227221FE6
:10EB100020C0AD5BBF4F19C0AD5BBF4F2C912078BB
:10EB200018C0AC5BBF4FDECFAC5BBF4F2C912870E1
:10EB300010C0AC5BBF4F2C9120710BC0AC5BBF4FC2
:10EB40002C91207206C0AC5BBF4F2C91207401C089
:10EB500020E0092FFFDE0F91EF900895A1E0B0E0D3
:10EB6000E4EBF5E70C94CBE9182FE091EC1DF09164
:10EB7000ED1DE65BFF4F808181FF03C08FE990E0D0
:10EB800002C08EE990E069830E940B53AC01812F93
:10EB9000698120E00E9459472196E3E00C94E7E95F
:10EBA000DF92EF92FF920F931F93142FF22E982F64
:10EBB000990F980F990F190F660F660F660FF60ED3
:10EBC000812F6F2D46E027E000E00E947245E09122
:10EBD000EC1DF091ED1D05A8F6A9E02DE330F1053F
:10EBE0009CF062E0D62ED10E52E0E52EEF0C8D2D7A
:10EBF0006F2D412F2E2D01E00E94DA44412F4C5FF2
:10EC00008D2D6F2D2E2D18C08FEFEE3FF807B4F429
:10EC100042E0D42ED10E36E0E32EEF0C84E0F80E65
:10EC20008D2D6E2D412F2F2D01E00E94DA44412FB2
:10EC30004C5F8D2D6E2D2F2D0E94DA441F910F9168
:10EC4000FF90EF90DF900895BF92CF92DF92EF9206
:10EC5000FF920F931F93182FB62E423039F443ECD6
:10EC600057E420E00E9459471C5F05C08B5F49E0D4
:10EC700020E00E949947E091EC1DF091ED1D63A901
:10EC800074A9882777FD8095982F0E9458E76B011B
:10EC90007C0120E030E048E453E40E9441E818168B
:10ECA00054F0C701B60120E030E048E453EC0E9484
:10ECB000B6E687FF16C0C701B60120E030E040EAA3
:10ECC00051E40E94BDE60E9425E79B01AC01812F23
:10ECD0006B2DA90124E030E000E0EE240E947E4D7F
:10ECE00015C0C701B60120E030E040E05FE30E94BC
:10ECF00045E80E9425E79B01AC01812F6B2DA901FE
:10ED000023E030E000E0EE240E943E4E812F8C5F35
:10ED10006B2D41EC57E420E00E9459471F910F9161
:10ED2000FF90EF90DF90CF90BF900895A0E0B0E00B
:10ED3000ECE9F6E70C94C5E9182FB62EE091EC1D2E
:10ED4000F091ED1D91AD8091EF06981710F492E0CF
:10ED500001C090E09093CF1D4091EE06442309F44A
:10ED6000CAC0812F8A5F6B2D50E021E030E000E0C7
:10ED7000E92E0E943C4D812F895F6B2D4FEB57E4AC
:10ED80002091CF1D0E9459478091EE06833009F0F3
:10ED90004EC0F12EFF0CF10EFF0CEB2CEE0CEE0C26
:10EDA000EE0C8F2D6E2D4CE127E001E00E945448BF
:10EDB0002091EE0630E0309521953F4F55E0220F2F
:10EDC000331F5A95E1F7E091EC1DF091ED1D81ADF7
:10EDD000280F311DC901880F991FB3E0220F331F7F
:10EDE000BA95E1F7820F931F6CE070E00E946CE926
:10EDF0006B01EB01CB0101978B31910540F46E2D36
:10EE00006F5F8F2D8F5F4C2D25E00E9472452BE1A7
:10EE1000C216D10470F48C2DF3946E2D6F5F4AE10D
:10EE20004C198F0D25E000E00E94724502C0C0E041
:10EE3000D0E08091EE068450823008F05CC0F12E64
:10EE4000FF0CF10EFF0CBB0CBB0CBB0C8F2D6B2D04
:10EE50004EE127E001E00E9454488091EE068430A4
:10EE6000A9F4E091EC1DF091ED1D21AD30E02058AA
:10EE70003040C901880F991FF3E0220F331FFA9524
:10EE8000E1F7820F931F6FE070E016C08530B9F490
:10EE9000E091EC1DF091ED1D21AD30E0205A3040A5
:10EEA000C901880F991F73E0220F331F7A95E1F78C
:10EEB000820F931F63E170E00E946CE9EB01CE01C9
:10EEC00001978D31910548F46B2D6F5F8F2D8F5F0A
:10EED0004C2F25E001E00E947245CC31D10558F459
:10EEE0008C2FF3946B2D6F5F4CE14C1B8F0D25E045
:10EEF00000E00E947245CDB7DEB7E9E00C94E1E98D
:10EF00009F92AF92BF92CF92DF92EF92FF920F93B8
:10EF10001F93D82EB62EC42E122FE091EC1DF09127
:10EF2000ED1D41AD8091EF06481718F472E0E72E11
:10EF300001C0EE24E092CF1D80912F1064E0962E48
:10EF40009D0CFC2CF3948823B9F08AE0489FC00103
:10EF500011246091EE0670E00E946CE9AB018D2DEA
:10EF60006B2D23E030E000E0A12E0E94CE4D892DD4
:10EF70006B2D4DEB57E40DC08D2D6B2D50E023E034
:10EF800030E000E0A12E0E948A4D892D6B2D4BEBC5
:10EF900057E42091CF1D0F2DE12E0E9428474D2DC3
:10EFA000440F4D0D440F485E6B2D660F660F660FC4
:10EFB000262F295F01E08091CF1D823009F000E00B
:10EFC000842F0E94DA441F910F91FF90EF90DF9001
:10EFD000CF90BF90AF909F900895AF92CF92EF9255
:10EFE0000F938091D01D813079F581E260E041E29C
:10EFF00029E001E00E94DA448DE560E04DE529E07A
:10F000000E94DA4480E06AE04FE72AE00E94DA4496
:10F010008CE060E04AE557E420E00FEFEE240E9428
:10F02000284780E06AE040E02FE301E00E94DA44F4
:10F030008FE76AE04FE72FE30E94DA4480E06FE356
:10F040004FE72FE30E94DA4480E060E040E020E0F8
:10F0500057DFE091EC1DF091ED1DE05BFF4F40812B
:10F0600051818091920F9091930F8417950710F41E
:10F0700092E001C090E09093CF1D87E060E025E032
:10F0800030E000E0E92EEDEFCE2EAA240E94064DDE
:10F09000E091EC1DF091ED1D47A950AD80E160E0DD
:10F0A00020E002E0EE240E944A4E83E162E042E06A
:10F0B00029EF0EEFE4DC83E164E040E029EF0BEFA1
:10F0C000DEDC83E166E041E029EF08EFD8DC83E194
:10F0D00067E043E029EF0DEFD2DC80E162E046E03B
:10F0E00022EF0EEFCCDC80E164E04BE022EF0BEF8F
:10F0F000C6DC80E166E042E122EF08EFC0DC80E19F
:10F1000067E04EE022EF0DEFBADC8CE062E047E012
:10F1100021EF0EEFB4DC8CE064E048E021EF0BEF70
:10F12000AEDC8CE066E049E021EF08EFA8DC8CE083
:10F1300067E04AE021EF0DEFA2DC89E062E044E005
:10F140002BEE0EEF9CDC89E064E045E02BEE0BEF4C
:10F1500096DC89E066E044E12BEE08EF90DC89E084
:10F1600067E045E12BEE0DEF8ADC86E062E04FE0E0
:10F1700025EE0EEF84DC86E064E040E125EE0BEF47
:10F180007EDC86E066E041E125EE08EF78DC86E093
:10F1900067E043E125EE0DEF72DC0F91EF90CF9029
:10F1A000AF900895A1E0B0E0E8EDF8E70C94BCE979
:10F1B0008091D01D813071F581E260E041E229E06B
:10F1C00001E00E94DA448DE560E04DE529E00E940F
:10F1D000DA4480E069E04FE729E00E94DA4480E009
:10F1E0006AE040E02FE30E94DA448FE76AE04FE7ED
:10F1F0002FE30E94DA4480E06FE34FE72FE30E94A1
:10F20000DA4486E060E040E657E420E002E0EE24E5
:10F210000E94284780E060E040E020E071DE8CE062
:10F2200060E04EE025E000E02ADCE091EC1DF0918A
:10F23000ED1D47A950AD80E160E020E002E0EE2442
:10F240000E944A4E94E6692E94E1792E82E0B82E0F
:10F250009BE04424552409E1202E312C1CEFD12EB3
:10F26000D40C420180E0692F4FE727E001E0998349
:10F270000E9472450894411C511C80E06B2DA20134
:10F2800021E030E000E0B2E0EB2EA4E0CA2EAD2C8D
:10F290000E94064D829CF001839CF00D929CF00D23
:10F2A0001124E45AFB4E84E06B2DE080F180028152
:10F2B00013812481358146815781F2E0CF2EAA2423
:10F2C0008D2C0E94A04E84E16B2D4EE557E422E088
:10F2D00000E0ED2C0E942847F30120813181442772
:10F2E00037FD4095542F80E16B2D02E0EE24CD2CAC
:10F2F00011D99981292F285F81E0622F4DE700E025
:10F300000E94DA441B2D1F5FF30120853185428561
:10F31000538581E0612F0E94FD4EF30124813581E8
:10F32000468157818CE0612F0E94FD4E99819F5E3E
:10F33000F2E0BF0E29E130E0620E731E9E3309F049
:10F340008DCF2196E2E10C94D8E9EF92FF920F93D2
:10F350001F93182FF62EE091EC1DF091ED1D21ADBD
:10F360008091EF06281710F492E001C090E090938E
:10F37000CF1D423009F41D5F812F6F2D422F50E0C9
:10F3800023E030E000E0E92E0E94C24D812F8C5F27
:10F390006F2D49EB57E42091CF1D0E9459471F91D3
:10F3A0000F91FF90EF900895CF92DF92EF92FF922E
:10F3B0000F931F93E82EF62ED42E122F6091EE0697
:10F3C000E42FF0E042E2649F402D112450E0A09130
:10F3D000EC1DB091ED1DD9962C91D99730E0241BEE
:10F3E000350BE29FC001E39F900DF29F900D112419
:10F3F0002AE2629F602D112470E0641B750B0E944D
:10F400006CE9C62E67FDCC248C2D992787FD90953D
:10F41000E817F9070CF4CD2C113009F410E02D2D6C
:10F420002C19013069F48E2D6F2D412F00E00E94C0
:10F4300072456D2D6F0D6C198E2D412F2C2D0CC02A
:10F440008C2D8E0D6F2D422F212F00E00E947245D2
:10F450008E2D6F2D4C2D212F01E00E9472451F91A2
:10F460000F91FF90EF90DF90CF900895A0E0B0E073
:10F47000ECE3FAE70C94C1E98091D01D813009F0EA
:10F4800056C080E063E14FE723E101E00E94DA44E7
:10F4900080E069E24FE729E20E94DA4480E06FE30E
:10F4A0004FE72FE30E94DA4481E260E041E223E18A
:10F4B0000E94DA448DE560E04DE523E10E94DA44E4
:10F4C00080E063E140E020E40E94DA448FE763E1FA
:10F4D0004FE720E40E94DA448CE060E046E557E420
:10F4E00020E00FEFEE240E9428478CE061E044E525
:10F4F00057E420E012E0E12E0E9428474091EE06FA
:10F5000083E161E050E021E030E000E0EE24B2E091
:10F51000CB2EA2E0AA2E0E94064D84E161E042E5D6
:10F5200057E420E002E0F2E0EF2E0E94284780E05E
:10F5300060E040E020E0E4DC80E069E04EE121E0D2
:10F5400002E032DFE091EC1DF091ED1DE05BFF4F3A
:10F55000408151818091920F9091930F841795076C
:10F5600010F492E001C090E09093CF1D87E060E03E
:10F5700025E030E000E0E92EEDEFCE2EAA240E9437
:10F58000064DE091EC1DF091ED1D47A950AD80E1D5
:10F5900060E020E002E0EE240E944A4EE091EC1D83
:10F5A000F091ED1DE25BFF4F4081518187E061E00A
:10F5B00024E030E000E072E0A72E0E948A4D88240B
:10F5C000992455E0D52EBB24BB2019F447EFF42E27
:10F5D00002C03DEFF32E7D2C7A94E401CC0FDD1FA9
:10F5E000CC0FDD1FC80DD91DC659D24E11E08B813D
:10F5F000807F19F149814423A1F0812F672D50E0CC
:10F6000023E030E000E0EE24CC24AF2C0E94064D35
:10F61000812F8D5F672D4BE020E001E0EF2C0E94F1
:10F62000A7454881812F6D2D50E023E030E000E0B8
:10F63000EE24CC24AF2C0E948A4D25961B5F1531F9
:10F64000B1F6B39482E0D80E84E090E0880E991E63
:10F650009B2D923009F0B8CFCDB7DEB7EDE00C941A
:10F66000DDE9AF92CF92EF920F93CF93DF9380912A
:10F67000D01D813009F06DC080E06CE14FE72CE1D6
:10F6800001E00E94DA4480E063E34FE723E30E9455
:10F69000DA4481E460E041E422E30E94DA4480E05D
:10F6A00064E014D987E062E046E857E420E000E037
:10F6B00092E0E92E0E9428478CE060E041E857E4A0
:10F6C00020E0EE240E9428478CE061E04CE757E4FC
:10F6D00020E0EE24E3940E94284784E161E04BE0BF
:10F6E00020E001E00E94A7458CE062E047E757E494
:10F6F00020E000E0B2E0EB2E0E94284784E162E0C7
:10F7000041E420E002E00E94A74580E061E298D851
:10F7100086E065E042E757E420E000E0EE24E39471
:10F720000E94284786E460E25DD884E164E04DE60B
:10F7300020E002E0EE240E94A74584E165E04BE072
:10F7400020E001E0EE24E3940E94A74584E167E015
:10F75000D3D882E068E04BE022E001E025DE82E0E1
:10F7600060E040E020E0CCDB88E060E046E020E0C4
:10F7700000E085D9E091EC1DF091ED1D47A950AD59
:10F7800082E061E020E0EE24E3940E944A4EE091A2
:10F79000EC1DF091ED1DE05BFF4F408151818091A8
:10F7A000920F9091930F8417950710F492E001C087
:10F7B00090E09093CF1D82E062E025E030E000E031
:10F7C000E92ECC24A2E0AA2E0E94064DE091EC1D69
:10F7D000F091ED1D23A934A9442737FD4095542FFE
:10F7E00080E160E0EE240E948A7284E160E042E001
:10F7F00020E0D6D9E091EC1DF091ED1D86AD97ADDE
:10F8000068E671E00E946CE9AC0181E161E023E00F
:10F8100030E0AA24A3940E94064DE091EC1DF091E3
:10F82000ED1DE25BFF4F80819181CAE0D0E0BE0117
:10F830000E9458E9AB0181E162E023E030E0F2E0B0
:10F84000AF2E0E94064DE091EC1DF091ED1D42A9F6
:10F8500084E064E050E022E030E00E943C4D88E02B
:10F8600064E04EE02FEF0BD9E091EC1DF091ED1D1F
:10F8700022AD33AD40E050E0CA01B901E3E0660FCC
:10F88000771F881F991FEA95D1F7620F731F841F96
:10F89000951F2AEF30E040E050E00E947FE983E0CE
:10F8A00065E0A90123E030E0AA24A3940E94064D5C
:10F8B000E091EC1DF091ED1D84A595A5BE010E947F
:10F8C00058E9AB0181E164E023E030E00E943C4D67
:10F8D0004091EE1D5091EF1D80E165E024E030E0A5
:10F8E0000E94064D81E067E042E020E0C8D884E055
:10F8F00067E040E020E0C3D887E067E041E020E037
:10F90000BED88AE067E043E020E0B9D88DE067E048
:10F910004BE020E0B4D8E091EC1DF091ED1DEE5BE2
:10F92000FF4F408181E167E050E023E030E00E943A
:10F930003C4DDF91CF910F91EF90CF90AF90089514
:10F940009091950F992309F0F1C9FFCCEF92FF92A6
:10F950000F931F93F82E162FE091EC1DF091ED1DE3
:10F96000E05BFF4F408151818091920F9091930F06
:10F970008417950710F492E001C090E09093CF1D9A
:10F980008F2D612F25E030E000E0E92E0E943C4DF4
:10F990008F2D8B5F612F45EB57E42091CF1D0E9487
:10F9A00059471F910F91FF90EF900895A1E0B0E0AB
:10F9B000ECEDFCE70C94CBE9182FE091EC1DF091F5
:10F9C000ED1DE65BFF4F808180FF03C021EA30E040
:10F9D00002C020EA30E0C90169830E940B53AC01E8
:10F9E000812F698120E00E9459472196E3E00C9421
:10F9F000E7E9EF92FF920F931F93182FF62E4230F4
:10FA000018F0423059F515C0E091EC1DF091ED1D54
:10FA100086AD97AD68E671E00E946CE9AC01812F7C
:10FA20006F2D23E030E000E0EE240E943C4D1D5F8E
:10FA300015C0E091EC1DF091ED1D86AD97AD68E627
:10FA400071E00E946CE9AC01812F8B5F6F2D23E088
:10FA500030E000E0EE240E943C4D185F812F6F2DB6
:10FA60004EE120E00E9499471F910F91FF90EF9087
:10FA700008950F931F93082F162FE091EC1DF0911E
:10FA8000ED1D86AD97AD68E671E00E946CE90E94BD
:10FA90009770E82FF0E0EE0FFF1FE752F94B25912A
:10FAA0003491802F612FA90120E00E9459471F91B6
:10FAB0000F910895A0E0B0E0E0E6FDE70C94C5E901
:10FAC000E091EC1DF091ED1D86A597A588599E4FFC
:10FAD00026AD37AD821B930BC8E6D1E0BE010E9474
:10FAE0006CE9C82EB92E8AE160E244E620E201E02A
:10FAF0000E94DA448FE360E04FE32FE30E94DA4490
:10FB00008DE36BE041E42BE00E94DA4488E26EE191
:10FB100048E222E20E94DA4486E56EE146E522E20E
:10FB20000E94DA448DE365E341E425E30E94DA4470
:10FB300085E790E00E940B53AC0189E060E020E093
:10FB40000E94594787E790E00E940B53AC0183E085
:10FB500063E020E00E94594788E790E00E940B5341
:10FB6000AC0181E163E020E00E94594786E790E024
:10FB70000E940B53AC0189E067E020E00E945947E6
:10FB800089E790E00E940B53AC0180E060E020E048
:10FB90000E945947E091EC1DF091ED1DE05CFF4F94
:10FBA0004081552747FD509582E060E023E030E03A
:10FBB00000E0EE240E947E4D85E060E04BE020E016
:10FBC0000E9499478AE790E00E940B53AC0180E0C5
:10FBD00067E020E00E945947E091EC1DF091ED1D97
:10FBE000EF5BFF4F4081552747FD509582E067E06E
:10FBF00023E030E00E947E4D85E067E04BE020E0AE
:10FC00000E9499478BE790E00E940B53AC018DE076
:10FC100060E020E00E945947E091EC1DF091ED1D5D
:10FC200086AD97ADBE010E946CE9AC018FE060E04B
:10FC300023E030E00E943C4D82E160E04BE020E0B8
:10FC40000E94994783E160E014DFE091EC1DF091A0
:10FC5000ED1DDF01A05CBF4F8C91992787FD90952A
:10FC600022E030E0B9010E946CE9709561957F4F08
:10FC700040E2F42EF60EEF5BFF4F8081992787FD5F
:10FC80009095B9010E946CE9709561957F4F3FE3B3
:10FC9000D32ED60E6091E3068091E40690E070E0EA
:10FCA00049E050E028E030E00E94494A0091E50632
:10FCB0001091E6068091E4066091E30648E027E0B3
:10FCC0000E94EB498D2D90E06F2D70E049E050E0EF
:10FCD00028E030E001E00E94494A8D2D6F2D48E078
:10FCE00027E00C2D1B2DEE24E3940E94EB49C092DB
:10FCF000E506B092E606F092E306D092E406CDB7B0
:10FD0000DEB7E9E00C94E1E90F931F93082F162F5B
:10FD1000E091EC1DF091ED1D26AD37ADC90168E60F
:10FD200071E00E946CE9AC01802F612F20E000E0BF
:10FD30000E94D0701F910F910895EF92FF920F9340
:10FD40001F93F82E162FE091EC1DF091ED1DE25B54
:10FD5000FF4F4081518123E030E000E0EE240E941B
:10FD6000C24D8F2D8C5F612F43EB57E420E00E9442
:10FD700059471F910F91FF90EF9008950F931F9394
:10FD8000082F162FE091EC1DF091ED1D47A950AD05
:10FD90000E94974E802F8B5F612F41EB57E420E04C
:10FDA0000E9459471F910F910895EF92FF920F9370
:10FDB0001F93F82E162FE091EC1DF091ED1D22AD52
:10FDC00033AD40E050E0CA01B901E3E0660F771FB0
:10FDD000881F991FEA95D1F7620F731F841F951F23
:10FDE0002AEF30E040E050E00E947FE98F2D612F44
:10FDF000A90123E030E000E0EE240E943C4D8F2D6D
:10FE00008D5F612F4DEA57E420E00E9459471F9112
:10FE10000F91FF90EF9008958F929F92AF92BF92B3
:10FE2000CF92DF92EF92FF920F931F93B82E962EF0
:10FE3000842ED22E102FFE2C0E9477708B2D90E0F6
:10FE4000692D70E0482D50E021E00E9482732091DE
:10FE5000E5063091E6062C543F4F8B2D90E0692D3E
:10FE600070E0482D0D2DEE24C12EAF2C0E94C073E2
:10FE70002091EE1D3091EF1D2C543F4F8B2D90E0C3
:10FE8000692D70E0482DEE24E3940E94C0738091A8
:10FE9000EE1D9091EF1D9093E6068093E5061F916D
:10FEA0000F91FF90EF90DF90CF90BF90AF909F9019
:10FEB0008F9008958F929F92AF92CF92EF920F936F
:10FEC0001F93CF93DF938091D01D813031F581E274
:10FED00060E041E22BE001E00E94DA448FE560E05F
:10FEE0004FE52BE00E94DA4480E06CE04FE72CE025
:10FEF0000E94DA4480E062E04DE657E420E000E052
:10FF0000A2E0EA2E0E94284780E065E047E657E439
:10FF100020E0F3E0EF2E0E94284780E060E040E020
:10FF200020E00E94807780E069E04EE121E002E07D
:10FF30003BDAE091EC1DF091ED1D86AD97ADE8E662
:10FF40008E2EE1E09E2EB4010E946CE9AC0186E0A9
:10FF500060E022E000E00E94D070E091EC1DF091A2
:10FF6000ED1D47A950AD80E160E020E002E0EE2405
:10FF70000E944A4EE091EC1DF091ED1D23A934A999
:10FF8000442737FD4095542F80E063E000E073E0A4
:10FF9000C72E0E948A7284E063E041E023E00E9461
:10FFA000D075E091EC1DF091ED1D84A595A56AE05A
:10FFB00070E00E9458E9AB0180E066E024E030E0A8
:10FFC000CC2494E0A92E0E94064D84E066E045E62C
:10FFD00057E420E002E014E0E12E0E94284788E088
:10FFE00063E049E024E0B3E0EB2E16DF85E361E255
:10FFF00046E12AE000E00E94724584E360E248E1C5
:020000021000EC
:100000002CE001E00E9454488FE36CE342E022E0E0
:100010000E947245C091EE1DD091EF1DC43BD105E9
:1000200034F0C4018C1B9D0BEC0110E001C011E009
:1000300089E064E0AE0123E030E000E0EE24A3E0DC
:10004000CA2EF3E0AF2E0E94064D112349F02097EF
:1000500039F086E366E247E326E201E00E94DA44F3
:1000600080E162E046E02DEF00E00E943F7583E111
:1000700062E042E020E00E943F7583E164E040E0FE
:1000800020E00DEF0E943F7583E166E041E020E053
:100090000AEF0E943F7583E167E043E020E00FEF45
:1000A0000E943F7580E167E04EE02DEF0E943F75B2
:1000B000DF91CF911F910F91EF90CF90AF909F90D4
:1000C0008F900895EF92FF920F931F93F82E162FA3
:1000D0004091EE1D5091EF1D23E030E000E0EE2452
:1000E0000E943C4D8F2D8D5F612F4EE120E00E94DC
:1000F00099471F910F91FF90EF900895EF92FF9213
:100100000F931F93F82E162F423020F0423009F043
:1001100042C020C0E091EC1DF091ED1D84A595A595
:100120006AE070E00E9458E9AB018F2D612F23E057
:1001300030E000E0EE240E943C4D8F2D8D5F612F5A
:100140004DE620E00E9499478F2D8C5F612F0E9421
:10015000DF7121C048EA57E420E00E945947E0914E
:10016000EC1DF091ED1D84A595A56AE070E00E945C
:1001700058E9AB018F2D8B5F612F23E030E000E069
:10018000EE240E943C4D8F2D885F612F44EA57E496
:1001900020E00E9459471F910F91FF90EF90089522
:1001A0000F931F93CF93DF93E091EC1DF091ED1D22
:1001B000E65BFF4F9081492321E009F420E0909114
:1001C0008C0F992311F091E0292706E0809F800190
:1001D00011240B5F1F4FC62FD0E0B3E0CC0FDD1F03
:1001E000BA95E1F7239640918D0FC801BE0150E00A
:1001F0000E948349C801BE0143E050E021E00E9413
:100200000A49DF91CF911F910F91089548E0C8CF1F
:1002100040E1C6CFA1E0B0E0E0E1F1E80C94CBE929
:10022000182FE091EC1DF091ED1DEC5BFF4F8081EC
:1002300080FF03C085EA90E009C081FF03C086EA21
:1002400090E004C082FF0BC087EA90E069830E94BF
:100250000B53AC01812F698120E00E945947219600
:10026000E3E00C94E7E9EF92FF920F931F93F82ECF
:10027000162FE091EC1DF091ED1DEE5BFF4F4081DC
:1002800050E023E030E000E0EE240E943C4DE0919D
:10029000EC1DF091ED1DEC5BFF4F90818F2D8D5F7C
:1002A00094FF04C0612F41EA57E403C0612F4EE977
:1002B00057E420E00E94C6471F910F91FF90EF90F6
:1002C0000895EF92FF920F931F93F82E162FE0914F
:1002D000EC1DF091ED1DDF01AC5BBF4FEC90E094A5
:1002E000EE1CEE24EE1CEE0CE092CF1D423018F016
:1002F000423009F510C042A950E022E030E000E0B1
:100300000E943C4D8F2D8E5F612F48E02091CF1DC4
:100310000E94994710C042A950E022E030E000E07E
:100320000E943C4D8F2D8E5F612F49E957E420914B
:10033000CF1D0E9459471F910F91FF90EF90089594
:10034000A1E0B0E0E6EAF1E80C94CBE9182FE091E7
:10035000EC1DF091ED1DED5BFF4F808182FF03C02E
:1003600089EA90E01BC083FF03C08AEA90E016C0D0
:1003700080FF03C08BEA90E011C081FF03C08CEACC
:1003800090E00CC084FF03C08DEA90E007C085FFB9
:1003900003C08EEA90E002C088EA90E069830E9480
:1003A0000B53AC01812F698120E00E9459472196AF
:1003B000E3E00C94E7E90F931F93660F660F660F57
:1003C000982F990F980F695FE091EC1DF091ED1D4A
:1003D00005A916A9892F880F4AE02EE00E94007116
:1003E0001F910F910895EF92FF920F931F93F82E94
:1003F000162F423000F5E091EC1DF091ED1D838D3C
:10040000948D6AE070E00E9458E9AB018F2D612F56
:1004100023E030E000E0EE240E943C4D8F2D8D5F04
:10042000612F4DE620E00E9499478F2D8C5F612F50
:100430000E944C7221C044E957E420E00E945947D1
:10044000E091EC1DF091ED1D838D948D6AE070E0DC
:100450000E9458E9AB018F2D8B5F612F23E030E0C4
:1004600000E0EE240E943C4D8F2D885F612F40E913
:1004700057E420E00E9459471F910F91FF90EF90A1
:100480000895EF92FF920F931F93182FF62EE0918D
:10049000EC1DF091ED1D85A996A997FF05C08095EB
:1004A00090918F0F981710F080E001C082E0809348
:1004B000CF1D8091900F882311F00E94B86F80911A
:1004C000CF1D823059F480919D0F882339F488EE36
:1004D00093E060E670E040E00E94B7B0E091EC1D70
:1004E000F091ED1D45A956A9812F6F2D23E030E035
:1004F00000E0E090CF1D0E943E4E812F8C5F6F2D5B
:100500004DE857E42091CF1D0E94C6471F910F91DF
:10051000FF90EF900895EF920F9381E061E041E04A
:100520000E94247680E067E041E00ADA8DE067E02F
:100530000DDA88E067E001DC8DE060E041E059DA47
:1005400082E160E096DA8CE061E0DEDB87E066E085
:1005500015DC80E060E029DC81E063E047E020E03A
:1005600000E0EE2459DC88E063E0ACDD87E062E087
:1005700041E0C4DD88E065E04DDE8FE066E073DEDB
:100580008FE062E07EDF88E064E041E09ADE89E0AF
:1005900060E011DF0F91EF900895EF92FF920F93BB
:1005A0001F93F82E162FE091EC1DF091ED1D40A940
:1005B00081E090E02091EB06222311F080E090E0B2
:1005C000242F30E08217930729F44093EB0681E053
:1005D0008093EC068091EC06813071F4EC5BFF4F68
:1005E000808185FF09C084EF91E060E870E040E021
:1005F0000E94B7B01092EC06E091EC1DF091ED1D59
:1006000040A98F2D8E5F612F50E022E030E000E0A6
:10061000EE240E943C4D8F2D612F4AE857E420E0E4
:100620000E9459471F910F91FF90EF900895EF920C
:100630000F9380E063E00E94AE758BE063E040E0E2
:100640000E94247680E067E040E07AD98DE067E0A0
:100650007DD988E067E071DB80E065E0A7D98DE0B7
:1006600060E040E0C6D982E160E003DA8CE061E05E
:100670004BDB80E061E082DB80E060E096DB80E1E4
:1006800064E045E020E000E0EE24C6DB8CE064E0BE
:1006900019DD8AE065E040E031DD8AE066E040E0B7
:1006A000A2DE85E066E079DF80E066E0AFDD83E032
:1006B00066E0AEDD80E064E0ADDD8CE062E0E1DECE
:1006C00082E162E040E0FDDD80E062E039DE89E069
:1006D00060E071DE0F91EF900895EF92FF920F931B
:1006E0001F93F82E162FE091EC1DF091ED1D858DD6
:1006F000968D6AE070E00E946CE9AB018F2D612F4E
:1007000023E030E000E0EE240E943C4D8F2D8D5F11
:10071000612F4EE120E00E9499471F910F91FF90B9
:10072000EF900895EF920F9380E061E00E94AE7524
:1007300080E064E042E00E9424768DE067E042E0E1
:10074000FFD880E067E002D988E067E0F6DA80E071
:1007500063E02CD98CE063E042E04BD98FE065E0A8
:100760000DDB80E160E045E020E000E0EE2454DBBA
:100770008BE065E0A7DC80E065E042E0BFDC80E084
:1007800066E042E030DE8BE066E0A7DF8CE062E00E
:100790003DDD8EE062E03CDD80E062E03BDD8FE04D
:1007A00064E06FDE8AE060E042E08BDD80E060E0E4
:1007B000C7DD0F91EF900895EF920F9383E00E94B1
:1007C000306D87E062E04EE157E420E00EEFEE246A
:1007D0000E94284785E066E043E157E422E004E018
:1007E00098EFE92E0E9428478FEF6FE00E94975400
:1007F00087E062E040E02CEF0E94D3538FEF0E942D
:1008000076B08AEF90E09093331E8093321E8091F1
:10081000321E9091331E009729F08FEF0E9476B020
:100820008823A9F380EF0E9476B00E945B430F916A
:10083000EF900895AF92CF92EF920F931F93CF93C3
:10084000DF93182F83E00E94306D82E066E041E084
:1008500057E422E002E0A9EFEA2E0E942847C12FC8
:10086000D0E08EE066E0AE0122E030E001E0F2E0B0
:10087000EF2EE2E0CE2E79EFA72E0E94064DFE016C
:10088000EE0FFF1FE95AF94B2591349187E0B9012A
:1008900042E020E00EEF0E943747DF91CF911F9199
:1008A0000F91EF90CF90AF900895AF92CF92EF92CB
:1008B0000F931F93CF93DF93182FEB0185E00E94D6
:1008C000306D83E061E24CE721E200E00E94DA440F
:1008D00083E065E34CE725E30E94DA4480E063E0CF
:1008E000412F50E022E030E001E092E0E92E15E0F7
:1008F000C12EAA24AA940E94064D82E063E04FEF25
:1009000056E422E005E0EE24EA940E94284785E0C0
:1009100063E0AE0122E00CEF0E94284780E064E033
:1009200043EF56E422E006E0B4E0EB2E0E942847B5
:1009300081E165E04EEE56E422E000E00E942847A7
:1009400083E090E00E940B53AC0180E067E022E07E
:100950000E94594781E167E049EE56E422E00E9497
:100960005947DF91CF911F910F91EF90CF90AF90AA
:100970000895CF93DF93FC01A091EC1DB091ED1D84
:10098000D3968D919C91D497918780879C968D91D9
:100990009C919D9793878287EF012C9611968DE00D
:1009A0000D9009928150E1F7A6E3BEE188E00D9039
:1009B00001928150E1F7DF91CF9108958AEFECE544
:1009C000F4E1DF011D928A95E9F70895E091EC1DAD
:1009D000F091ED1DEC5BFF4F808187FF15C08DE32B
:1009E00095E1DC01FC01799729E101900D922150FC
:1009F000E1F7499724E18C35920799F7BADF80EA4D
:100A000090E06FEF7FEF04C088E592E06FE070E068
:100A100040E00C94B7B0A3E0B0E0E1E1F5E80C945D
:100A2000BCE90E945B438091DF068230B9F48AE919
:100A300090E00E940B53AC0180E063E020E00E9454
:100A4000594784E690E09093331E8093321E809144
:100A5000321E9091331E0097D1F706C380912A0F62
:100A6000882309F0A9DE81E00E948C6D11E01093CB
:100A7000E7061092F0061092EE061092F106109220
:100A8000EB061092EC061092EB1D1092D11D0E9405
:100A9000516B8BEE90E00E940B53BC0180E041E370
:100AA0005BE70E94566B8CEE90E00E940B53BC01FA
:100AB00081E04AE55FE70E94566B8DEE90E00E9470
:100AC0000B53BC0182E046E35AE70E94566B8EEE60
:100AD00090E00E940B53BC0183E04DEE57E70E946B
:100AE000566B8FEE90E00E940B53BC0184E042ED08
:100AF00058E70E94566B80EF90E00E940B53BC01B8
:100B000085E04AE55DE70E94566B81EF90E00E9428
:100B10000B53BC0186E048EF5BE60E94566B82EF08
:100B200090E00E940B53BC0187E047E153E80E942C
:100B3000566B83EF90E00E940B53BC0188E04BE8BA
:100B400052E80E94566B84EF90E00E940B53BC0168
:100B500089E042E953E80E94566B8091940F0E940D
:100B6000986B1093D01D8CE291E09093331E80938C
:100B7000321E8DE290E090934C1E80934B1E10929B
:100B80004A1E1092491E1092501E10924F1E109233
:100B9000411E1092401E10E0EE2490E05CE2652EB3
:100BA00051E0752E01E040E9442E41E0542E3CEB2B
:100BB000232E32E0332E8091710B882309F41BC25F
:100BC0000E948AC9E091730BF091740BF093ED1DB4
:100BD000E093EC1D8091EE068823B9F482E08093C7
:100BE000EE0642E00CC0542F5F5F21AD30E06BE2B7
:100BF000469FC0011124281739071CF0452F4730A4
:100C000090F34093EE0640932A140E94777082ED91
:100C10009DE1AFDE8091E21D9091E31DA091E41D66
:100C2000B091E51D8093820F9093830FA093840F62
:100C3000B093850F8091DE1D9091DF1DA091E01D86
:100C4000B091E11D80937E0F90937F0FA093800F52
:100C5000B093810F8091EB1D883211F41092EB1D3F
:100C60008091EC1D9091ED1D9B838A83FC01ED5BCF
:100C7000FF4F808180FFF6C080913C1E90913D1E09
:100C8000009799F08091F9139091FA13009769F405
:100C9000A3EFB3E1E6E3FEE188E02A813B81019026
:100CA0000D928150E1F73B832A83EA81FB8187A97A
:100CB00090AD9093061480930514E0900714F09083
:100CC00008140894E11CF11CF0920814E092071437
:100CD00080901D1490901E14AA24BB24E25BFF4F49
:100CE000C080D180B60180E090E024E630E040E0B2
:100CF00050E00E942DE9681979098A099B0997013A
:100D000040E050E00E94A1E9280D391D4A1D5B1DFD
:100D100030931E1420931D14EA81FB8183A994A9AA
:100D200020910B1430910C142817390724F4909358
:100D30000C1480930B14EA81FB8182AD93AD20915A
:100D40001114309112142817390720F490931214BB
:100D500080931114EA81FB8184A595A52091171435
:100D6000309118142817390720F4909318148093A1
:100D7000171480911B1490911C148C159D0520F460
:100D8000D0921C14C0921B14EA81FB81E05BFF4FE0
:100D900080819181209123143091241428173907E0
:100DA00020F49093241480932314EA81FB8181AD75
:100DB00090912914891710F480932914EA81FB81FA
:100DC000E95BFF4F808191812091151430911614B9
:100DD0002817390724F49093161480931514EA8188
:100DE000FB81EE5BFF4F808190911F14981710F4E8
:100DF00080931F14EA81FB81EE5BFF4F808190910D
:100E00002014891710F480932014EA81FB81E05CA0
:100E1000FF4F808190912614891714F48093261433
:100E2000EA81FB81E05CFF4F808190912514981747
:100E300014F480932514EA81FB81EF5BFF4F8081DE
:100E400090912814891714F480932814EA81FB8167
:100E5000EF5BFF4F8081909127149817B4F4809333
:100E6000271413C0EE2099F080913C1E90913D1EF6
:100E7000009769F0ABEFB3E1E6E3FEE188E00190B3
:100E80000D928150E1F7EE2402C0EE24E3940E941B
:100E90002D701123C1F480914B1E90914C1E009730
:100EA00021F08091D01D813071F48091D01D81306E
:100EB00011F40E945B430E94BD6B8DE290E0909321
:100EC0004C1E80934B1E1092D01DE091EC1DF091B2
:100ED000ED1DEB5BFF4F80819091D11D891739F19A
:100EE000833228F58823B9F00E94E972E091EC1D65
:100EF000F091ED1DEB5BFF4F80819CDC88EE93E071
:100F00006FE070E040E00E94B7B030923F1E209248
:100F10003E1E12E003C00093D01D10E0E091EC1DD6
:100F2000F091ED1DEB5BFF4F80818093D11D80E23E
:100F30000E9495B0C82E80E10E9495B0882329F4C4
:100F400091E0CC2021F490E002C040DD91E080E10E
:100F500099830E9480B099818823B9F01123A1F46C
:100F60008091911DE82FF0E0EE0FFF1FEE0FFF1FA5
:100F7000EF56F24E6281738198DC50923F1E409290
:100F80003E1E11E090E001C091E080E899830E944C
:100F900076B09981882319F00E94B06B91E080E4CB
:100FA00099830E9476B09981882319F00E94A16BE1
:100FB00091E0112331F0992309F44EC00093D01D24
:100FC00009C0992339F403C00093D01D10E00E949A
:100FD000B86E03C01092710B10E08091341E909196
:100FE000351E009719F482E00E948C6D7092331EBA
:100FF0006092321E91E02091321E3091331E2115F5
:10100000310551F4892F0E944F737092331E609204
:10101000321E0093D01D90E08091911D8093940F1B
:1010200080E299830E9480B09981882309F4C3CD1E
:10103000EE2079F080913C1E90913D1E009749F082
:10104000ABEFB3E1E6E3FEE188E001900D92815061
:10105000E1F71092E70608C080913E1E90913F1E76
:10106000009709F4B1CFB3CF2396E2E10C94D8E90D
:10107000EF920F931F93182F0E94ACB08CE390E077
:101080006FEF7FEF40E00E94B7B00E945B4380E0CB
:1010900060E04FE727E001E00E94724585EE90E0B6
:1010A0000E940B53AC0181E060E022E000E0EE24FE
:1010B0000E9428470E947B5080E064E14FE72BE1CB
:1010C00001E092E0E92E0E949248133091F0143032
:1010D00028F4113041F01230E9F408C0143061F006
:1010E0001530C1F40CC080EE90E00BC081EE90E0B2
:1010F00008C082EE90E005C083EE90E002C084EE6E
:1011000090E00E940B53BC0182E040E020E009E047
:101110000E94374785EE90E00E940B53BC0184E0AB
:1011200040E020E004E00E9437478BE090E00E941E
:101130000B53AC0180E067E020E00E9459470E9419
:101140001291082F80E80E9476B0882321F00E9437
:10115000ACB081E00CC080E10E9476B0882321F41D
:10116000002309F092CFEBCF0E94ACB080E01F913A
:101170000F91EF90089585E07BDF8823A1F00E9416
:101180006F6D0E94816D1ADC60E070E0CB0120E0A1
:1011900030E0A9010E94113C80E991E06FEF7FEF00
:1011A00040E00C94B7B00895CF92EF920F931F9345
:1011B0000E94ACB011E0112309F463C00E945B43AC
:1011C00048D789E090E00E940B53AC0183E061E0D6
:1011D00020E000E0F4E0EF2E0E9428478CE090E051
:1011E0000E940B53AC0183E062E020E00E9428479C
:1011F00080E060E24FE727E001E00E9472458AE06C
:1012000090E00E940B53AC0181E063E022E000E03B
:10121000E8E0EE2E0E9428472091820F3091830F44
:101220004091840F5091850F81E064E0EE247AE0D4
:10123000C72E0E94FD4E20917E0F30917F0F40916E
:10124000800F5091810F8CE064E0EE24EA940E94BC
:10125000FD4E80E06FE14FE724E101E00E94544839
:1012600084E090E00E940B53AC018CE067E020E04A
:101270000E94594782E167E04AED5AE420E00E946B
:1012800059470E947B5080E20E9476B0882309F57E
:1012900080E10E9476B08823A1F084E0E9DE882313
:1012A00091F080E991E06FEF7FEF40E00E94B7B0EE
:1012B00060E070E0CB0120E030E0A9010E94113C29
:1012C00008C010E001C011E0ADD7882309F076CF47
:1012D00072CF0E94ACB01F910F91EF90CF90089504
:1012E0001F93162F882371F400D00F92EDB7FEB72D
:1012F000118221E73DE4338322830E9446D40F907C
:101300000F900F9084E064E673E00E9458D40E942E
:1013100011D58430F1F4812FABDE8823A9F012308F
:1013200039F0133041F0113039F40E946F6D04C070
:101330000E94816D01C042DB80E991E06FEF7FEF99
:1013400040E00E94B7B007C00E945B430E946DD48A
:10135000DECF8823E1F61F910895A9E0B0E0E3EB2A
:10136000F9E80C94BCE90E945B4383E50E94B3D387
:10137000882309F4C3C000D00F9282E0ADB7BEB796
:1013800011968C9311978DE09BE413969C938E930A
:1013900012970E9446D426E5C22E25E1D22E0F9048
:1013A0000F900F90EE24FF2480E01E010894211C72
:1013B000311C9CE3492E512C612C712CF60190813B
:1013C000992309F487C00E94F9D3B701B4E0660FEE
:1013D000771FBA95E1F76E0D7F1D695A7A4EC101EC
:1013E0000E94C1D889809A80AB80BC802DB73EB75F
:1013F0002F5030403EBF2DBF0DB71EB70F5F1F4FA0
:10140000ADB7BEB711961C922EEE3AE4F8013283C6
:101410002183C501B40120E13EE040E050E00E949C
:101420007FE9D80114963C932E931397C501B4011C
:10143000A30192010E947FE94B015C01CA01B9013D
:10144000A30192010E947FE9F8017683658390866B
:1014500087828D81818712868E81838714868F8112
:101460009885968785870E9446D42DB73EB7265F1C
:101470003F4F3EBF2DBFEDB7FEB73196ADB7BEB7FC
:1014800011961C9223EE3AE432832183D6018C918B
:10149000838314820E9446D4D601EC91F0E0EE0FD3
:1014A000FF1FE95AF94B85919491EDB7FEB731963C
:1014B000ADB7BEB711961C922EED3AE4328321836C
:1014C000838394830E9446D40F900F900F900F90C7
:1014D0000F9081E00894E11CF11CA1E1B0E0CA0E7C
:1014E000DB1EB4E1EB16F10409F068CF89870E9496
:1014F000F9D3898562E0F4DE0E94ECD32996E2E11B
:101500000C94D8E9A9E0B0E0E8E8FAE80C94BCE96A
:101510000E945B438DE20E94B3D3882309F4F7C095
:1015200000D00F9282E0EDB7FEB7818383E59BE4A4
:10153000938382830E9446D444E6E42E44E1F42E51
:101540000F900F900F908824992480E01E0108943A
:10155000211C311C3CE3432E512C612C712C870142
:10156000F8012085318542855385211531054105D6
:10157000510509F4BAC00E94F9D389E190E0889E30
:10158000B001899E700D989E700D1124645A7B4E97
:10159000C1010E94C1D8A980BA80CB80DC80EDB7A0
:1015A000FEB73F97FEBFEDBFEDB6FEB60894E11C57
:1015B000F11C118284E39BE4F701928381838D8186
:1015C000838314828E81858316828F81988590878C
:1015D0008783C601B50120E13EE040E050E00E9473
:1015E0007FE9F70132872187C601B501A301920186
:1015F0000E947FE95B016C01CA01B901A30192015C
:101600000E947FE9F70174876387B686A5860E94EA
:1016100046D40F900F900F900F90EDB6FEB6089441
:10162000E11CF11CEDB7FEB7118285E29BE4F701E6
:1016300092838183F801648575858685978528EE78
:1016400033E040E050E00E94A1E9F70123833483B6
:1016500045835683F80160817181882777FD8095E5
:10166000982F0E9458E720E030E040E05FE30E94BE
:1016700045E8F70167837087818792870E9446D487
:10168000EDB6FEB60894E11CF11CEDB7FEB7118271
:1016900088E19BE4F70192838183F801608571857D
:1016A000828593852AE030E040E050E00E94A1E985
:1016B000F7012383348345835683F8016481758160
:1016C000868197812AE030E040E050E00E94A1E965
:1016D000F70127833087418752870E9446D48DB710
:1016E0009EB70B969EBF8DBF81E00894811C911C14
:1016F000075E1F4F9AE08916910409F031CF898760
:101700000E94F9D3898563E0EBDD0E94ECD3299632
:10171000E2E10C94D8E9A8E0B0E0E1E9FBE80C9440
:10172000BEE963EF662E63E1762E2E010894411C1C
:10173000511CC201B3010E94C1D8C980DA80EB807C
:10174000FC808DB79EB70B979EBF8DBF0DB71EB7A0
:101750000F5F1F4FEDB7FEB7118284E59DE4F801DE
:1017600092838183C701B60120E13EE040E050E072
:101770000E947FE9F801348323835CE3852E912C5A
:10178000A12CB12CC701B601A50194010E947FE9EB
:10179000CA01B901A50194010E947FE9F80176838D
:1017A00065838D81878310868E81818712860E9452
:1017B00046D48DB79EB70B969EBF8DBFB301685FB1
:1017C0007F4FC2010E94C1D8C980DA80EB80FC80C3
:1017D000EDB7FEB73B97FEBFEDBF0DB71EB70F5F6E
:1017E0001F4F118287E39DE4F80192838183C70133
:1017F000B60120E13EE040E050E00E947FE9F801C0
:1018000034832383C701B601A50194010E947FE9B7
:10181000CA01B901A50194010E947FE9F80176830C
:1018200065838D81878310868E81818712860E94D1
:1018300046D48DB79EB70B969EBF8DBF0E94F9D33D
:101840002896E0E10C94DAE92F923F924F925F9252
:101850006F927F928F929F92BF92CF92DF92EF9280
:10186000FF920F931F93DF93CF9300D000D0CDB79B
:10187000DEB70E945B4380912B14880F880F865F30
:101880000E94B3D3882309F420C1CE0101960E949F
:10189000CB6B00D00F9232E0E32EADB7BEB71196FE
:1018A000EC9211978EEE9BE413969C938E93129775
:1018B0000E9446D40F900F900F902DDFEDB7FEB72A
:1018C0003797FEBFEDBF3196ADB7BEB711961C92EC
:1018D0008DED9BE4928381830DE010E014830383FC
:1018E00080911B1490911C14968385830E9446D48A
:1018F000EDB7FEB73196ADB7BEB711961C928CEC22
:101900009BE4928381838AE090E094838383809137
:101910001D1490911E1464E670E00E9458E96583DE
:1019200016820E9446D400D0EDB7FEB73196ADB70F
:10193000BEB711961C9285EB9BE49283818314833E
:101940000383898190E00196968385838A818783CA
:1019500010860E9446D400D0EDB7FEB73196ADB7E1
:10196000BEB711961C928FE99BE492838183148306
:1019700003838B8190E00196968385838C81878396
:1019800010868EE190E0928781870E9446D4EDB761
:10199000FEB73B96FEBFEDBF0E94F9D380912B149A
:1019A000882309F48DC000D00F92ADB7BEB7119651
:1019B000EC92119786E99BE413969C938E93129771
:1019C0000E9446D40F900F900F90BB2421E8C22EA6
:1019D0002BE4D22E9DE0E92EF12C8EE6882E8BE4AE
:1019E000982E0AE0602E712C14E6412E512CBDE594
:1019F0002B2EBBE43B2E5FC08B2D90E0EDB7FEB7E6
:101A00003997FEBFEDBF3196ADB7BEB711961C92A8
:101A1000D282C1829C012F5F3F4F34832383F682A1
:101A2000E5828C01000F111F080F191F000F111FF5
:101A30000F5D104FD801A35FBA4F8C91878310863A
:101A40000E9446D40F900F90EDB7FEB73196ADB718
:101A5000BEB711961C929282818274826382D801F1
:101A6000A25FBA4F8D919C91B2010E9458E96583A3
:101A700016820E9446D400D0EDB7FEB73196ADB7BE
:101A8000BEB711961C9232822182F482E382D80181
:101A9000A05FBA4F8C91858316822EE130E03087AB
:101AA00027830E9446D48DB79EB709969EBF8DBFEF
:101AB0000E94F9D3B39480912B14B81608F49CCFEC
:101AC00081E061E00DDC0E94ECD32496DEBFCDBF47
:101AD000CF91DF911F910F91FF90EF90DF90CF900A
:101AE000BF909F908F907F906F905F904F903F90AE
:101AF0002F900895A4E0B0E0E0E8FDE80C94C6E97A
:101B00000E945B4389E10E94B3D3882309F451C248
:101B1000CE0101960E94CB6B00D00F9282E0ADB750
:101B2000BEB711968C93119788E29DE413969C930F
:101B30008E9312970E9446D40F900F900F90EBDD7A
:101B40008091051490910614EDB7FEB73797FEBF4C
:101B5000EDBF3196ADB7BEB711961C922FE03DE4B4
:101B6000328321836CE370E00E9458E974836383BD
:101B7000968385830E9446D4EDB6FEB60894E11C98
:101B8000F11CEDB7FEB711828FEF9CE4D7011296DE
:101B90009C938E9311970DE010E014961C930E9376
:101BA000139760910B1470910C14882777FD809522
:101BB000982F0E9458E720E030E040EA51E40E946C
:101BC000BDE60E9425E7F701768365830E9446D42F
:101BD000EDB7FEB73196ADB7BEB711961C928FEE3A
:101BE0009CE49283818314830383809117149091E2
:101BF00018145AE0C52ED12CB6010E9458E97683FC
:101C000065830E9446D4EDB6FEB60894E11CF11C33
